:020000040000FA
:080000000002040000000000F2
:020000040000FA
:10040000CF2521000E7F22000E0188000000000091
:100410000C000700E0EC2D00010020001100070097
:10042000000020000000E000020032000000020096
:1004300000000000AED30200000000000040DA001F
:100440000000FE004440A900805021000000E000B0
:100450000300320000002000A00188004440A800F2
:100460000000060091018800800078000000EB0089
:1004700015003700E280400032A0B4009101BA00BC
:10048000E280400032A0B4009102BA00E280400055
:1004900032A0B4000002EB00472BDE00F507B200EB
:1004A000602CE10004003A000059EB008301E900F0
:1004B000FDFF3E00040037006128E100010032002A
:1004C0000082EB00040007001101BA000200E00006
:1004D000E8FF3A00000006003159BA008301E90044
:1004E0000C0032002159BA008301E90008003200F3
:1004F0000400E00003003A00E280400032A0B400B3
:10050000F5FF370011D9BA008301E900FAFF3A007C
:100510008100E800E180400032A0B4000000060045
:1005200048F5040000000000CEF5040000000000C3
:1005300046F60400000000000CEA04000000000081
:10054000A2EA04000000000010EB0400000000001C
:100550007E93040000000000889304000000000067
:10056000A693040000000000B8FB04000000000097
:1005700012FC04000000000024FC04000000000045
:100580003CFC04000000000058FC040000000000D7
:10059000D6FB04000000000018CB0400000000009F
:1005A0003ACB0400000000004ECB04000000000025
:1005B00062CB04000000000074CB040000000000C7
:1005C00016CC04000000000036CC0400000000003F
:1005D00048CC0400000000005ECC040000000000D5
:1005E000B8CC04000000000012CD040000000000A0
:1005F0006CCD040000000000C6CD04000000000027
:100600008ACB040000000000ECCD040000000000D4
:1006100000CE0400000000000040DA000000FE00F0
:100620001004B100030035009001B10001003C004E
:100630001000050000000500800078001104B100E2
:10064000030035009101B10001003C000050A00002
:10065000000006001004B100070035009001B10051
:10066000040034007000B100030035009001B100B7
:1006700001003C0010000500000005006900E100D9
:10068000040035006D00E100030034000002B100F9
:100690000100320000000500100005002002E20009
:1006A00004003D002342AB00020032002302AB00F5
:1006B000FEFF32000040DA00FEFF37000A00FA00B9
:1006C00080017800E20F500028003E00C08E8000BC
:1006D000E10F500008003200802320000000E000FD
:1006E000050032000423200025232000462320009B
:1006F0008001780004003700042220002522200019
:100700004622200083222000144090000004E000D4
:10071000040035008009EB00144090000074A00034
:1007200010429800154090000028A30003003A00F2
:10073000154090000024A000904298008001EB003A
:1007400007003700154090000008A300FDFF3200AD
:1007500063C078000000FB00000B78008301E80014
:10076000828F5100F7FF3A00080037003000200068
:10077000B0BF9F00C3BF9F00D1BF9F00E2BF9F00DB
:100780006A80570000C0DA006FB997000200780055
:100790000080FA00000006000A00FA0011002000A4
:1007A000B1BF9F00C0BF9F006A80570000C0DA0041
:1007B0004FB897000080FA00000006000A00FA0017
:1007C00051002000B1BF9F00C0BF9F006A8057004A
:1007D00000C0DA005FB897000080FA000000060051
:1007E0000A00FA00881F7800800178000000E0000D
:1007F00029003A00C08E8000E10F5000080032004E
:10080000802320000000E0000500320004232000C7
:100810002523200067232000800178000400370092
:1008200004222000252220006722200083222000AD
:10083000144090000004E000040035008009EB0043
:10084000144090000074A000104298000002EB00D9
:100850000C003700130A2000154478006140640042
:1008600002003A008301E900FBFF3A000402E800BD
:100870009541780061C061000500320017007800E2
:100880008058780004035100820F5200F1FF3A00B3
:10089000060051000800370020002000A0BF9F0084
:1008A000B3BF9F00C1BF9F00D2BF9F006C805700A5
:1008B00000C0DA005FB897004F0478000080FA00AB
:1008C00000000600889FBE0080047800D08E800063
:1008D0000000E00003003A00100007000000E00004
:1008E0000A003500D08E80000900E00002003A00C6
:1008F000000478000600370000047800090040007A
:10090000060007000000E00001003D000084EB004D
:10091000080078004F04BE00000006008000780048
:100920000000E00004003A00C01D2100D08E8800C5
:1009300001017800060037000081EB00C02521008E
:10094000808F500002003E00D18E88000001EB0035
:100950000200780000000600020AB900001BB9007E
:100960000200B80081004200810043000000060040
:100970006022B800060220000000D0008180D20072
:100980000482D2008582D2000000A0000202520040
:1009900083825A00030031000202420083824A002F
:1009A0000000A1000603E900F3FF3A000000060082
:1009B000EFFF07000400BE0000000600889FBE0095
:1009C0008A9FBE008C1F78000205BE000004BE0096
:1009D0000006EB00E00F5000E08F5800E00F5900D8
:1009E000E08F590007003D006000B8006011B800BA
:1009F00008045000898458000A0559008B85590065
:100A00001C002000E00F5200E08F5A00E00F5B0056
:100A1000E08F5B0002003D000F0007000C00A20009
:100A20000800BE000A01BE001D0107000203BE004F
:100A30000002BE000C00E0000100320006000700CA
:100A40000400BE000601BE004F0678004F05BE0040
:100A50004F04BE00000006006000B8006011B8003E
:100A6000040250008582580006035900878359000C
:100A700000000600881F7800000478005001BE00C6
:100A80004000BE0004004000858048000601490087
:100A900087814900009CBE000294BE000400E10072
:100AA0000588E1000690E1000798E10002003100AE
:100AB000680044001008E8004F04780000000600B9
:100AC000F4874700889FBE008A9FBE008C9FBE00AF
:100AD0008E1F78000205BE000004BE00D4B79F0040
:100AE000E5B79F00F6B79F0087BF9F000000EB00AF
:100AF000C0B79F00B0B79F00A0B79F0090B79F00FE
:100B000080B79F000D042000BFB097004FB0970042
:100B1000000140000000E0000F003D004F08DE0033
:100B200000007100C0B79F009E00070001003D005B
:100B300012002000A100070001003D00120020006B
:100B4000A6000700B1000700B60007000F00400034
:100B5000C8FF0700220037004F08DE0000067100C2
:100B6000CCB79F008F00070001003D00120020005D
:100B70009200070001003D001200200097000700CE
:100B8000A20007000FB297009FB297002FB3970003
:100B9000BFB39700A90007000000520081805A00EF
:100BA00002015B0083815B0080B79F0091B79F00CB
:100BB000A2B79F00B3B79F000007EB009F0007009C
:100BC0000020E10001A8E10002B0E10003B8E1006B
:100BD000010031001E0020000E005600C0B79F002B
:100BE0004FB297000400E00007003500100020001D
:100BF000010020006011B8000804700089847000B2
:100C00000A0571008B8571008D06E900BEFF3A0070
:100C10000400E00003003D00820007000F004000D8
:100C200094FF07004FA897000000E00004003A007E
:100C30000FB497009FB497002FB59700BFB59700EA
:100C4000940007004F0778004F06BE004F05BE0016
:100C50004F04BE004F01B10000000600881F78005D
:100C600018002000881F780095FF07008F87E90093
:100C70004F04780000000600801FEB0090FF070083
:100C80008F87E90000000600889FBE008A9FBE0093
:100C90008C1F78006E00070007003D0073000700FE
:100CA000E00F5B00E08F5B0007003D0032000700B3
:100CB0000006EB00040037003400070002003D008E
:100CC0002A0007001C00200072000700E3FF070055
:100CD0000203BE000002BE000C00E0000100320072
:100CE000220007000400BE000601BE004F06780087
:100CF0004F05BE004F04BE0000000600889FBE00E6
:100D00008A9FBE008C1F78005100070005003D003F
:100D100056000700E00F5B00E08F5B0006003D001F
:100D2000040037001900070003003D006000B80010
:100D30006011B8001000070056000700CEFF070042
:100D40000203BE000002BE000C00E0000100320001
:100D5000060007000400BE000601BE004F06780032
:100D60004F05BE004F04BE00000006006000B80042
:100D70006011B8000000370004025000858258005E
:100D80000603590087835900000006000006EB00A7
:100D9000E00F5200E08F5A00E00F5B00E08F5B0035
:100DA000000006000180400090B79F000001EB00AA
:100DB0008FB097000100E000000006000200700004
:100DC00090B79F000180400080B79F000001EB00BA
:100DD000FFA897000100E00000000600020070007C
:100DE00080B79F00018040006FAA9700CF20DE00EF
:100DF00001007000F0AF9F000402420025000700D0
:100E00004F18DE000002720000000600E4AF9F00F1
:100E10000804440089844C000A054D008B854D0070
:100E2000000006003FB29700CFB297005FB3970073
:100E3000EFB3970000FE2F00000006003FB09700C0
:100E4000CFB097005FB19700EFB1970000000600A8
:100E50000205BE000004BE00E00F5000E08F580005
:100E6000E00F5900E08F5900000006006000B80054
:100E70006011B80008045000898458000A05590020
:100E80008B8559001C002000E00F5200E08F5A00B3
:100E9000000006000800BE000A01BE0000000600B7
:100EA000889FBE008A9FBE008C9FBE000404B800CD
:100EB0000506B8008904460060854E000606B800A5
:100EC0000A054600E0854E000706B8008B0546007F
:100ED000040EB800890446000A854E00E0854D00E6
:100EE000050EB8000A0546008B854E00060EB800B8
:100EF0008B0546000416B8000A0546008B854E0097
:100F00000516B8008B054600041EB8008B05460088
:100F10000800BE000A01BE004F06BE004F05BE001D
:100F20004F04BE00000006000400FA00E0BF9F006E
:100F3000E4815700812978000002EB000F003700A0
:100F40006FB89700904078007FB897001040780005
:100F50000402E80080CF5000040032008180FB00D2
:100F60000080FB0000805000070037006FB897003A
:100F70000000E800E0BF9F009309E800820F5200E4
:100F8000EFFF3A000000EB000080FA0000000600CE
:100F900010417800B141510003003A000000E80020
:100FA0000204E000FAFF3A000300FB000000060024
:100FB0008001EB0002003700817178008301E800B6
:100FC000828F5100FCFF3A00000006000000FA008A
:100FD000CFB8970068815700D40007000080FA005E
:100FE00000000600810178000000E9000081EB00AC
:100FF000E50F500004003E0080004000C01B2100AF
:101000006081780003B078000200780000000600DC
:10101000000178000000E900E50F50000F003E00DD
:1010200080004000C01B2100E08078000100E0004B
:1010300002003A001000200071030700E18F400019
:10104000060032000000EB00E18F50000400320087
:101050000200780001000100000005000080EB00A4
:101060000000060010002000E9FF0700100020002B
:1010700063030700800278008001780001003700D8
:101080008301E8001304E000FDFF3A000002EB00DA
:10109000820F52000600320064C078008059780048
:1010A0000402E8000004E00002003200F8FF37000C
:1010B0008049EB0005007800000006000C00FA00F3
:1010C000889FBE0000047800CFB09700F0FF270093
:1010D000D0BF9F008004EB0099BF9F0088BF9F0096
:1010E000A8BF9F00200C2000B0BF9F007881570050
:1010F000708057008D0007000FB8970009487800EE
:101100000FB8970008045000080078004F04BE0094
:101110000080FA0000000600810178000002EB0068
:101120000B003700E44078000104E00003003200C7
:101130000402E80093CF5000040032008180FB00DD
:101140001380FB0000805000000006008301E800CF
:10115000820F5200F3FF3A00000005000C00FA0075
:10116000A0BF9F00C0BF9F000A000700B0BF9F0044
:10117000F0BF9F00100C2000D0BF9F00748157006B
:10118000EFB097006C8057004D0307000080FA0015
:1011900000000600800078003004E000FEFF3A0006
:1011A000010050000000E900000006001041780036
:1011B000814F5100040032000000E8000204E0000A
:1011C000FAFF3A000000EB00000006008001780002
:1011D0000001780031407800005978000004E000F8
:1011E000FCFF3A0003007800000006008001EB00DD
:1011F0000200370061F079008301E800828F51001E
:10120000FCFF3A0000000600889FBE008A9FBE00D7
:101210008000780000C2B300010037008900780028
:101220008104780039447800804F5400FBFF32007D
:10123000E94F5400F9FF3200D0C2B300804F540090
:1012400004003A00194478008184E8001AC0B30011
:10125000060037000045EB00B0C2B300804F5400D9
:1012600002003A00194478008184E8006022B80046
:101270000A003700A2002000030020000400BE0086
:10128000B5FD07000B4144000281FB000300200074
:101290000002410081824900394478000880FB0047
:1012A0000BFD2F000B004000E90F5000F1FF36004E
:1012B0000A04E0000200320060021200E0821A001C
:1012C0000400BE004F05BE004F04BE000000060033
:1012D0000003780080027800020278008001EB00B1
:1012E000080037000402E90063C07800805A7800E3
:1012F0008301E8000004E00002003A008000EB00F7
:1013000006003700828F5100F6FF3A00FBFF3700DE
:101310000040EB0080F07A008100E800848F5000EC
:10132000FBFF3A000600780000000600FE87470039
:10133000889FBE008A9FBE008C9FBE008E1F7800D3
:10134000F0B79F000107780082BF9F000000EB000C
:10135000A0B79F009F0237008006EB0050C2B30089
:1013600080CF5000090032000100FB00FFB0970061
:10137000F4030700E10F400096023200AFB097007F
:101380008100E800A1B79F00920237009E407800DC
:10139000D0C2B30080CF50000C00320007003C00E8
:1013A0006D40500080CF50000A0032006B4040007A
:1013B00080CF50000E003A000800370000C3B30091
:1013C00080CF50000A003A00060037000D30A00020
:1013D000050037000D00A000030037000D10A0002D
:1013E000010037000D20A0000E07E800E7FF3700DE
:1013F0000D18A300010032000D00A1000D38A3005C
:10140000010032000D20A1000100FB0002FD2F00B1
:1014100002004000E90F50000E003E000002EB0009
:10142000C4B79F0082017800CFB297006A28B90044
:101430001E01FB000001410003014100C2B79F00F3
:101440005E00FB0003004000E90F50000B003E006F
:10145000F5FF37000006EB00CCB79F00A0C2B30039
:1014600080CF500005003A000FB89700C000780008
:1014700080BF9F00C1B79F000E07E8000001EB008E
:10148000B2B79F00E0C2B3009E4F100018003A00B0
:101490000DE0A0008E00E80064405000914F100065
:1014A00002003200010778000C0037000FBA9700E5
:1014B000C402780084BF9F00B5B79F000E87E80084
:1014C0000B0037003FB697006A60B900000041008A
:1014D00003004000B0B79F000E07E8001E01FB00AC
:1014E00003FD2F0003004100E90F5000F5FF360017
:1014F000BE407800E1D79F00C0C6B30080CF500047
:10150000220032000F003C006940500080CF5000A4
:101510007700320004003C000104E0003102320098
:101520006B4050000F00370040C6B30080CF500022
:10153000930032006540400080CF50008B003A009D
:101540008F00370030C7B30080CF50001A00320040
:1015500007003C006440500080CF50001100320072
:101560000040E80080CF500080003A000F003700B4
:1015700050C7B30080CF500080003200634040006D
:1015800080CF500079003A000900370000002800A1
:101590000D48A30001003A0000012000808676007B
:1015A000D3FF37000D60A000750037000D50A0007C
:1015B0000D70A000720037008FB8970041007800CE
:1015C00081BF9F00000478000000E00001003A00A5
:1015D000C81621008004EB00010037008104E800F8
:1015E00089007800088044001004E000FBFF3A0006
:1015F0003FB197000200E00003003200890F510064
:1016000001003100820478000002EB00E4AF9F008B
:10161000CFB29700898F5200020036000980520035
:10162000E0AF9F004368DE00E10660001B003A0067
:101630000D06780009003700FFB097000002200077
:1016400040030700E10F4000030032002FB0970075
:101650000000E800A0B79F000C06E800EFA8970084
:10166000810F5600F4FF3A000081EB00E2AF9F00CB
:101670000A003700880078003100FB000104780080
:10168000FFB097002F030700E10F40000300320076
:101690002FB297000402E800A4B79F000900E900F8
:1016A00080047800E10F4000F2FF3A000006EB00F2
:1016B0000D00E0000A003A00C6013700FFB09700B5
:1016C000000220001F030700E10F4000030032006A
:1016D000AFB297008502E800A5B79F000C06E800AE
:1016E0006FA89700800F5600F4FF3A00B901370049
:1016F0008FB897004100780081BF9F00CF80DE0047
:1017000001017800820178000205BE000004BE00DD
:101710000203BE000002BE004822DE00482EDD00AB
:1017200004027600E4D79F000D48A3000A003200AF
:101730000404E00008003200E14F420006003200DD
:1017400071FD2F0001804700044878001840980080
:101750002900200002003700F0D79F001900200068
:1017600072FD2F0002844700A1FF370064FD2F00A7
:1017700004844700190020009DFF37000D0CB300C2
:101780000D007800000CB20028003A000D00E000C7
:1017900005003D008FBA97004505BE004504BE0018
:1017A00085BF9F00140037000D48A3000B003200D6
:1017B0000FBE97004C00BE008CBF9F004F89DE001B
:1017C000CF91DE000002BE000203780082037800A1
:1017D0000605BE000404BE00070037008FB897005E
:1017E0004100780081BF9F0000047800CFC4DE0074
:1017F000090578008A057800E00F5400E08F5C004E
:10180000E00F5D00E08F5D001F003D003D00B30074
:101810006000B8006011B8000804500089845800C6
:101820000A0559008B855900170037000D00E000AC
:1018300005003D000FB997004205BE004204BE00FE
:1018400082BF9F00100037000D48A3000700320040
:101850000FBA97004400BE0084BF9F006011B8001B
:101860000205BE000004BE00070037008FBA9700D3
:101870004500780085BF9F00000478000900200023
:101880000A0020000B0020003FB697000C00E0008B
:1018900007003A00E00F5400E08F5C00E00F5D00AD
:1018A000E08F5D0002003A0010002000B0B79F00FA
:1018B0008D007800010CB200E1B79F000004200009
:1018C000808F50003000320003003C000100E00037
:1018D0000800320040003700000820006FB1970078
:1018E000800F510014003200000C2000800F5100C6
:1018F00039003A0014C0B300C50C21000B003700BA
:101900000400FB004300DD00050040005001BE0064
:101910004000BE000040E10001C8E10002D0E1004B
:1019200003D8E1002B0039000442E800F44F5200D4
:10193000F3FF3A00270037000001200001002000DB
:101940006011B80014C0B3000040E10001C8E1001C
:1019500002D0E10003D8E1001E003900450020005C
:101960000000D0008180D2000281D2008381D200A9
:101970008502E900FAFF3A000442E800F04F520005
:10198000F1FF3A0013003700800020000100200022
:101990006011B80014C0B3000040E10001C8E100CC
:1019A00002D0E10003D8E1000A0039003C00200029
:1019B0000000D0008180D2000281D2008381D20059
:1019C0000C06E900FAFF3A000442E800F54F520025
:1019D000F1FF3A00E4D79F00EFD097000100FB0031
:1019E0003FB19700820F500002003D00E2D79F00F8
:1019F000040037003FB29700800F520001003D0005
:101A0000B0B79F00CFB297000500E000040032009D
:101A100063806600020032008502E900C5B79F00BE
:101A20000DE8A3000B0032004FB697003FB09700BF
:101A3000800F560003003C008000EB00C1B79F0000
:101A4000040037004FB197003FB2970004015100E6
:101A5000C2B79F00EFD297000500FB000006EB0025
:101A6000DCAF9F00CFB09700808F500002003400A1
:101A700000805000D0AF9F000D28A3003700320037
:101A8000E18066000D18A3000C003200D002200097
:101A90000100E00001003A000080E900FFB097007B
:101AA00028020700E10F40000E0032002FB197001E
:101AB0000201E800A2B79F000A0037000100E00021
:101AC00008003200FFB09700000220001D0207004E
:101AD000E10F4000030032002FB297000402E8003B
:101AE000A4B79F00DFAA97000500E0000F003200B6
:101AF0000006EB00FFB09700000320001102070072
:101B0000E10F4000030032002FB097000000E80012
:101B1000A0B79F000C06E800DFA89700810F5600D1
:101B2000F4FF3A000001EB00D2AF9F003FB29700F4
:101B3000C320DD00400C21008080400091B79F0051
:101B40004220DD006400500080B79F006320B90090
:101B5000F0AF9F006306500084003700DFAA9700B3
:101B60000500E00011003200688066000F003A00B6
:101B700000067800FFB0970000022000F101070086
:101B8000E10F4000030032002FB097000000E80092
:101B9000A0B79F000C06E800DFA89700810F560051
:101BA000F4FF3A000001EB00D2AF9F00E180660035
:101BB0000D18A3000C003200D00220000100E0004C
:101BC00001003A000080E900FFB09700DD01070046
:101BD000E10F4000D5FF32002FB297000402E80069
:101BE000A4B79F00D1FF37000100E000CFFF320013
:101BF000FFB0970000022000D2010700E10F400073
:101C0000CAFF3200AFB297008502E800A5B79F0077
:101C1000C6FF370000042000EFB09700808F50000F
:101C20003100320003003C000100E00008003200F7
:101C30003E003700000820006FB19700800F510070
:101C400011003200000C2000800F510037003A00D4
:101C50001FB097003002BE002003BE000800BE0087
:101C60000A01BE00FDFB0700A400200005002000C3
:101C70006033B80000FC070004C3B3000442400016
:101C8000E4D79F002900370035172100D5B79F0002
:101C90000D58A30002003A0040182100D0B79F0061
:101CA00014002000050020006033B8008FB09700BA
:101CB0008100E900050033000402D0008582D200D3
:101CC0000683D2008783D200F9FF37000800BE00E8
:101CD0000A01BE00E1FB07006F0060005FB19700E2
:101CE000624078001000370014002000050020003A
:101CF0006033B8000C0078000000E90005003300F4
:101D00000402D0008582D2000683D2008783D200ED
:101D1000F9FF37000800BE000A01BE00CFFB070034
:101D2000674060000043B000E0D79F00EFD097000D
:101D30000100FB00FFB0970082010700E10F4000A7
:101D4000030032002FB197000201E800A2B79F0004
:101D50001FB297006802520094B79F008FB297009D
:101D6000E482520085B79F0063065600D0FF2F0023
:101D70003FB197000090B9007FAA97000000420091
:101D800063005000800F5600A2FF3A000D38A300F8
:101D900010003200DFAA97000500E0000D003400BB
:101DA0000006EB00FFB0970000022000650107006D
:101DB000E10F4000030032002FB097000000E80060
:101DC000A0B79F000C06E800DFA89700810F56001F
:101DD000F4FF3A00BE407800E1D79F000104E00024
:101DE0005DFD3A002FB097004F0778004F06BE0008
:101DF0004F05BE004F04BE00EF01B1000000060019
:101E000000047800960107000800780023FA070014
:101E1000889FBE00000478008144780000FD2F00F8
:101E200000004400E90F500002003E00000178006D
:101E30000D00370008007800F9F907000000E00005
:101E40000300320008007800FBF907000004780066
:101E500008007800FFF907000000E00007003200EA
:101E600090FA2F00000144000980FB00800F510010
:101E700002003D000280FB0001003700F00F20004F
:101E80004F04BE0000000600881F7800708E80009E
:101E90008101070000047800F8F907000000E00065
:101EA000FAFF3A00E10F440003003200718E800017
:101EB00008007800AC0107004F047800000006001D
:101EC000EC874700889FBE008A9FBE008C9FBE00A3
:101ED0008E1F780081BF9F0002077800708E8800F7
:101EE0008046EB00040137008884FB00090078007D
:101EF000E2F90700800078000000E00002003200F4
:101F0000E1FF0700FC00370050C2B300804F5400CF
:101F1000F0003A000FBD970020C0B300C0EF9F0053
:101F2000D1EF9F0081EF9F000300370040C0B30056
:101F3000C0EF9F000FBD97000FB99700B240780027
:101F400082BF9F008184FB0090C6B30080CF500009
:101F50003500320017003E006640500080CF500030
:101F6000620032000C003E007740500080CF5000ED
:101F70002800320006003E000104E0009B00320011
:101F8000A0C2B30080CF50006E003A001D003700A1
:101F900080C5B3001600370040C6B30080CF5000A4
:101FA000210032006440400080CF500065003A00BC
:101FB0001200370030C7B30080CF50001E0032003F
:101FC00007003E006740500080CF500011003200F3
:101FD0006340400080CF50005A003A0014003700A0
:101FE00050C7B30080CF50000F0032006340400064
:101FF00080CF500053003A006500370020C0B30086
:10200000CBFF3700DFE897008140E800D1EF9F0069
:10201000C8FF37004FE9970080C0B300E24F51007E
:10202000C3FF3A00C1FF3700ACC0B300590037000E
:102030008CC0B3005700370093FF0700DFE897001C
:102040000104E00002003A004E017800D2B79F0080
:10205000708E80001001070000047800E10F40003E
:10206000A20032008FEC9700120037000A85E800CA
:102070008ABF9F00160037008FB897001100FB0041
:10208000800F5400F9FF32005FE997000204E0007E
:1020900003003A005FB0970008587800D0B79F005F
:1020A0008944E9000A003200708E8000FA000700BF
:1020B000000478000800E800E10F5000040036003A
:1020C000080078006DF907000000E000EAFF320028
:1020D000DFE897000104E00087003A008D46E80041
:1020E0005FB1970001497800830037005FE89700EF
:1020F0000004E00003003A008D46E800CE007800BE
:10210000D1B79F00708E8000E3000700E10F400010
:10211000760032005FE997000204E00003003A0015
:10212000DFB0970080587800D1B79F000FE9970083
:102130000241E90082EF9F004240A9006E00340096
:10214000F0FF37000180FB0008FD2F000800400071
:10215000E90F50005F003E000A0078001F010700F1
:1021600080EF9F0088007800030037000FB89700C9
:102170000000E80080BF9F000FB997001200FB002D
:1021800001004000E90F5000F8FF360069FF3700FA
:102190000CC1B3003CFF0700708E8000BE0007003A
:1021A000000578000040EB00E0EF9F00D002200027
:1021B000800F550005003A00708E8000B6000700C1
:1021C0000005780011C0B300E1EF9F008C4078005B
:1021D0000A0078000EFF0700E14F40000A003A00B5
:1021E000718E80000A007800DF0007000D04E00017
:1021F0004B003A00708E8000300090000048A30031
:1022000043003200480037008FED97006044B8006B
:102210000C81FB00030020000800BE00CEF907007F
:102220000004BE008C4078000A007800F8FE070029
:102230000080FB0001002000080440008984480061
:102240008B45E90007003200708E80009200070085
:10225000000578008C407800EDFE0700E14F40005B
:10226000EBFF3A008C4078000A007800E8FE070097
:10227000E14F400003003A00718E80000A007800B0
:10228000B90007006FE997000204E0000200320085
:1022900060041400E0841C005FE897000004E00084
:1022A00015003A008D46E800CFE89700E4CF5000D3
:1022B00003003A004E0078000888BE000E00370088
:1022C0000E81E90002077800120078000808780003
:1022D00009003700708E80006F000700808F540067
:1022E00005003200E10F40000B003A000D04E00051
:1022F0000D0032000A0037008FB897003144780093
:1023000081BF9F000804E000F7FE3A000400370098
:102310000000EB0005003700718E8000920007007E
:102320000D80FB00010037000080EB004F077800B4
:102330004F06BE004F05BE004F04BE00CF00B100E7
:1023400000000600889FBE000001780001047800AC
:10235000B10090000118A3003D0032000198A300D5
:1023600003003A00180090000000E00038003A0036
:102370000190A0003104980082047800F90FB200A7
:10238000180090000000E00002003A0028009000D1
:10239000000C7800EA8F540006003A0038009000E4
:1023A0000078A30003003A0088007800D0002000E5
:1023B000E4FF07009800900058009000808F5000C4
:1023C0000B0032000100E8001004980018007800AB
:1023D00009587800000C780011C0B300C01C21001F
:1023E00001487800EA8F54000600320019003700D7
:1023F00088007800094078009C000700800478007D
:1024000014003700380090000088A300110032004B
:1024100018019000A800900048009000A7F807005D
:1024200098009000810F50000400320038009000A6
:102430000003B300300498008084EB000000EB0040
:102440001004980028009000000C7800010037006C
:102450008084EB00090078004F04BE0000000600F5
:10246000881F7800808E80000000E00001003200AC
:10247000000001008819210008007800BE00070054
:102480006C044400C01B2100800F5400FAFF3A0086
:102490004F04780000000600881F780000047800D0
:1024A000B00090000148A30007003A000108A30013
:1024B000050032000198A3000800320010009000CF
:1024C0000000E00005003200380090000040A0004D
:1024D000300498008080EB00200037000190A100BC
:1024E00031049800180090000000E000060034005D
:1024F0000000E9001004980018007800B080FB008C
:10250000000C780006003700380090000068A30037
:10251000EDFF3A0008007800CF0007008000780047
:10252000380090000078A3000C003A00FA8F5000A9
:1025300008003A00280090000000E000E2FF3200AE
:10254000180090000000E80010049800180CE90042
:10255000DDFF3700ED8F5000E2FF32000100780010
:102560004F0478000000060080017800E10F400071
:1025700017003200310090000008A3001400320060
:102580000098A30012003A00210290000400E0002D
:102590000F0032001101900051009000800F510097
:1025A0000B00320011007800840F500002003A0046
:1025B0008008E800020037000200E8009000980060
:1025C0001100E90080087800034878000100370016
:1025D0008081EB0003007800000006000001780015
:1025E00000C2B300010037000201E8009240780009
:1025F00080CF5000FCFF3200E9CF5000FAFF3200DC
:10260000D0C2B30080CF500003003A000201E800BE
:1026100014C0B300050037000042EB00B0C2B300A5
:1026200080CF500001003A000201E8008000EB007A
:1026300005FD2F00040037006A08B9000080410042
:10264000850040000201E8009201FB000580410086
:10265000E90F5000F8FF36000404E00001003200EA
:102660008100EA0001007800000006000200FA0084
:10267000889FBE00A0FF9F0001047800B100900079
:10268000810478000904B200020032000000FB005F
:10269000360037000118A30005003A000103B3001B
:1026A00031049800190498000080EB002F003700D7
:1026B000580090000000E00006003A00480090003A
:1026C00012002000E6805700FCF70700190498006C
:1026D00024003700280090000000E00008003A00C5
:1026E000801C210020049800000C780020002000AD
:1026F00050049800100498000130A00031049800A4
:1027000018019000A800900048009000EBF7070027
:1027100028009000000C78000080EB001004980066
:1027200018007800AFF8970001587800000C780086
:102730002FF89700EA4F50000A003A003800900046
:102740000088A3000700320018019000A800900044
:1027500048009000D9F7070019049800A8009000DD
:10276000010C7800AFF897000100FB004F04BE0099
:102770000080FA0000000600889FBE008A1F7800D3
:1027800000047800300090006300600024003200F4
:10279000080078007E0007003805900080EF2F00C9
:1027A0000000650030049800280090000000E00060
:1027B00004003200E804650002003A00AD000700A2
:1027C0002904980048009000F3F70700E10F40004B
:1027D00013003200B80090000102B20010003A006D
:1027E0000AC8A30018003200A08E80000000E0009C
:1027F000150032000001780081047800012A2000D1
:1028000012289000880F5000070032004205B000E7
:102810004905B000818F54000B003200F8FF3700EB
:102820000080EB000900370002007800E3F70700A2
:10283000A08E8000090040008000EB001128980065
:1028400001007800010037000000EB004F05780020
:102850004F04BE00000006000200FA00889FBE0080
:102860008A1F7800000478000000EB001004980034
:10287000380090008080EB000008A3003F00320089
:10288000C01C21001004E000100032008919210052
:10289000EA1921001A0078006C0545002010B200EA
:1028A00021102000810F500002003A00090078003A
:1028B00037000700EC844400C01B2100808F5400C7
:1028C000F4FF3A00C01C21000048EB0048009000D3
:1028D000580190000200E0000D003A001204980038
:1028E00012002000E8805700BDF70700E10F5000FC
:1028F00003003A000FF897008080FB001F003700AC
:10290000380090000040A00030049800120037000A
:10291000A8009000B2F70700100498000000E00043
:1029200003003200E10F40000D003A0003003700C1
:10293000380090000040A0000200370038009000EE
:102940000003B30030049800A8009000010C780048
:102950000000EB00100498008080EB0007003700B7
:10296000A8009000010C78000000E9001004980015
:1029700001007800B080FB00000C780001007800B6
:102980004F0578004F04BE000080FA0000000600EA
:10299000881F780000047800300090000008A30031
:1029A00007003200800078000120B20004003A00E5
:1029B00011049800A8009000010C7800170037005F
:1029C0000018A300190032000098A300170032007D
:1029D000A80090000100E0001400320018019000EF
:1029E0000200E000110032004800900033F70700B9
:1029F00098009000810F50000300320038009000D2
:102A00000003B300300498000000EB0010049800AD
:102A100028009000000C7800380090000058A300B7
:102A2000020032000080EB00010037000000EB00E4
:102A30004F04780000000600918E80000100E00045
:102A40000300320011007800908E880003003700E8
:102A5000200020009BF7070080007800E18F4000F5
:102A600002003A00906E2600B08E880001007800C7
:102A700000000600918E800001087800908E88008A
:042A8000000006004C
:020000040000FA
:0200000401F009
:04000C00FBFF0000F6
:020000040000FA
:0200000401F009
:04001000FDFF0000F0
:020000040000FA
:0200000401F009
:040014007FFF00006A
:020000040000FA
:100008000C03000022D30000EAD2000006D300004F
:100018003ED300005AD300000C0300000C0300007C
:100028000C0300000C0300000C03000094FD00000A
:100038000C0300000C0300000C0300000C0300007C
:1000480092D300000C0300000C03000058F50000D8
:100058000C0300000C0300000C0300000C0300005C
:100068000C0300000C0300000C0300000C0300004C
:100078000C0300000C0300000C0300000C0300003C
:100088000C0300000C0300000C03000090F00000BB
:10009800B2F100000C0300000C0300000C03000088
:1000A8000C0300000C0300000C0300000C0300000C
:1000B8000C0300000C0300000C0300000C030000FC
:1000C8000C0300000C0300000C0300000C030000EC
:1000D8000C0300000C03000076D300000C030000A2
:1000E8000C0300000C0300000C0300000C030000CC
:1000F8000C0300000C0300000C0300000C030000BC
:100108000C0300000C0300000C0300000C030000AB
:100118000C0300000C0300000C0300000C0300009B
:100128000C0300000C0300000C0300000C0300008B
:100138000C0300000C0300000C0300000C0300007B
:100148000C0300000C0300000C0300000C0300006B
:100158000C0300000C0300000C0300000C0300005B
:100168000C0300000C0300000C0300000C0300004B
:100178000C0300000C0300000C0300000C0300003B
:100188000C0300000C0300000C0300000C0300002B
:100198000C0300000C0300000C0300000C0300001B
:1001A8000C0300000C0300000C0300000C0300000B
:1001B8000C0300000C0300000C0300000C030000FB
:1001C8000C0300000C0300000C0300000C030000EB
:1001D8000C0300000C0300000C0300000C030000DB
:1001E8000C0300000C0300000C0300000C030000CB
:0801F8000C0300000C030000E1
:020000040000FA
:100208000C03000022D30000EAD2000006D300004D
:100218003ED300005AD300000C0300000C0300007A
:100228000C0300000C0300000C03000094FD000008
:100238000C0300000C0300000C0300000C0300007A
:1002480092D300000C0300000C03000058F50000D6
:100258000C0300000C0300000C0300000C0300005A
:100268000C0300000C0300000C0300000C0300004A
:100278000C0300000C0300000C0300000C0300003A
:100288000C0300000C0300000C03000090F00000B9
:10029800B2F100000C0300000C0300000C03000086
:1002A8000C0300000C0300000C0300000C0300000A
:1002B8000C0300000C0300000C0300000C030000FA
:1002C8000C0300000C0300000C0300000C030000EA
:1002D8000C0300000C03000076D300000C030000A0
:1002E8000C0300000C0300000C0300000C030000CA
:1002F8000C0300000C0300000C0300000C030000BA
:100308000C0300000C0300000C0300000C030000A9
:100318000C0300000C0300000C0300000C03000099
:100328000C0300000C0300000C0300000C03000089
:100338000C0300000C0300000C0300000C03000079
:100348000C0300000C0300000C0300000C03000069
:100358000C0300000C0300000C0300000C03000059
:100368000C0300000C0300000C0300000C03000049
:100378000C0300000C0300000C0300000C03000039
:100388000C0300000C0300000C0300000C03000029
:100398000C0300000C0300000C0300000C03000019
:1003A8000C0300000C0300000C0300000C03000009
:1003B8000C0300000C0300000C0300000C030000F9
:1003C8000C0300000C0300000C0300000C030000E9
:1003D8000C0300000C0300000C0300000C030000D9
:1003E8000C0300000C0300000C0300000C030000C9
:0803F8000C0300000C030000DF
:020000040000FA
:102A84006865000061640000657200002E69000042
:102A94006E630000006600006F6F00007465000044
:102AA400722E0000696E00006300000021440000E3
:102AB40045460000000D00000A0000007478000084
:102AC40074000000687400006D0000006874000069
:102AD4006D6C00000063000067690000007800006E
:102AE4006D6C000000630000737300000067000059
:102AF40069660000007000006E670000006A000054
:102B040070670000006300006C6100000077000043
:102B140061760000000000000000000000000000DA
:102B24006095000064950000689500006D950000B4
:102B34007195000075950000799500007D95000061
:102B44008195000085950000899500008D95000011
:102B540074650000787400002F7000006C61000040
:102B6400696E00000074000065780000742F000096
:102B7400687400006D6C000000740000657800004B
:102B8400742F0000786D00006C0000007465000074
:102B9400787400002F630000737300000069000064
:102BA4006D610000676500002F6700006966000022
:102BB400006900006D610000676500002F7000006F
:102BC4006E670000006900006D6100006765000029
:102BD4002F6A00007065000067000000617000004B
:102BE400706C00006963000061740000696F00008C
:102BF4006E2F00006A610000766100002D760000EF
:102C04006D00000061750000646900006F2F000012
:102C1400782D000077610000766500000000000058
:102C2400AA950000B5950000B5950000B595000083
:102C3400BF950000C8950000D1950000DB95000009
:102C4400E5950000F0950000049600001196000040
:102C540048540000545000002F3100002E31000071
:102C64002032000030300000204F00004B0D0000E7
:102C74000A4300006F6E00006E650000637400007C
:102C8400696F00006E3A0000206300006C6F000062
:102C9400736500000D0A0000004800005454000051
:102CA400502F0000312E000031200000343000008D
:102CB40030200000426100006420000052650000E2
:102CC4007175000065730000740D00000A43000074
:102CD4006F6E00006E65000063740000696F000091
:102CE4006E3A0000206300006C6F00007365000002
:102CF4000D0A00000D0A00003430000030200000EE
:102D040042610000642000005265000071750000FB
:102D140065730000743A000020630000616E0000D7
:102D24002774000020680000616E0000646C0000DD
:102D340065200000436F00006E740000656E0000A3
:102D4400742D00004C6500006E670000746800007C
:102D54000D0A00000048000054540000502F0000E9
:102D6400312E0000312000003430000031200000FA
:102D7400556E000061750000746800006F720000F9
:102D8400697A0000656400000D0A000057570000CE
:102D9400572D00004175000074680000656E000046
:102DA4007469000063610000746500003A2000004B
:102DB4004261000073690000632000007265000036
:102DC400616C00006D3D000022500000726F000035
:102DD400746500006374000065640000220D000047
:102DE4000A4300006F6E00006E650000637400000B
:102DF400696F00006E3A0000206300006C6F0000F1
:102E0400736500000D0A00000D0A00003430000054
:102E140031200000556E00006175000074680000E8
:102E24006F720000697A0000656400003A200000B7
:102E34005061000073730000776F0000726400003B
:102E44002072000065710000756900007265000061
:102E5400640D00000A0000004854000054500000B3
:102E64002F3100002E3100002034000030340000E7
:102E7400204E00006F740000206600006F75000093
:102E84006E6400000D0A0000436F00006E6E0000C7
:102E940065630000746900006F6E00003A20000052
:102EA400636C00006F730000650D00000A430000AE
:102EB4006F6E0000746500006E7400002D540000F5
:102EC40079700000653A0000207400006578000005
:102ED400742F0000687400006D6C00000D0A00007F
:102EE4000D0A000034300000343A0000204600008F
:102EF400696C0000652000006E6F00007420000003
:102F0400666F0000756E0000643C00006272000091
:102F14003E55000073650000203C00006120000065
:102F240068720000656600003D2200002F750000F5
:102F3400706C00006F610000642200003E4D0000D0
:102F44005046000053200000557000006C6F0000D4
:102F5400616400003C2F0000613E0000207400000A
:102F64006F200000707200006F6700007261000043
:102F74006D20000077650000622000007061000091
:102F840067650000730D00000A000000485400004B
:102F9400545000002F3100002E3100002034000076
:102FA4003134000020520000657100007565000096
:102FB400737400002D550000524900002054000095
:102FC4006F6F0000204C00006F6E0000670D000062
:102FD4000A4300006F6E00006E6500006374000019
:102FE400696F00006E3A0000206300006C6F0000FF
:102FF400736500000D0A00000D0A00003431000062
:1030040034200000526500007175000065730000F3
:10301400742D00005552000049200000546F000038
:103024006F2000004C6F00006E6700003A20000023
:10303400427500006666000065720000206F0000A3
:1030440076650000726600006C6F00007720000057
:10305400646500007465000063740000656400002A
:103064000D0A00000048000054540000502F0000D6
:10307400312E0000312000003530000030200000E7
:10308400496E000074650000726E0000616C0000FF
:103094002053000065720000766500007220000075
:1030A40045720000726F0000720D00000A430000B8
:1030B4006F6E00006E65000063740000696F0000AD
:1030C4006E3A0000206300006C6F0000736500001E
:1030D4000D0A00000D0A0000353000003020000009
:1030E400496E000074650000726E0000616C00009F
:1030F4002053000065720000766500007220000015
:1031040045720000726F0000723A00002045000012
:10311400787000006563000074650000642000009E
:103124006461000074610000206E00006F74000090
:103134002070000072650000736500006E7400006A
:103144000D0A00000048000054540000502F0000F5
:10315400312E000031200000353000003120000005
:103164004E6F000074200000496D0000706C000078
:10317400656D0000656E000074650000640D00005C
:103184000A4300006F6E00006E6500006374000067
:10319400696F00006E3A0000206300006C6F00004D
:1031A400736500000D0A00000D0A000035300000B0
:1031B400312000004E6F000074200000496D0000B3
:1031C400706C0000656D0000656E000074650000A1
:1031D400643A0000204F00006E6C0000792000006B
:1031E4004745000054200000616E00006420000088
:1031F400504F00005354000020730000757000000D
:10320400706F000072740000656400000D0A000015
:103214000048000054540000502F0000312E0000DC
:103224003120000032300000302000004F4B0000FD
:103234000D0A0000436F00006E6E0000656300001D
:10324400746900006F6E00003A200000636C000097
:103254006F730000650D00000A4300006F6E0000EC
:10326400746500006E7400002D5400007970000035
:10327400653A00002074000065780000742F000097
:10328400687400006D6C00000D0A00000D0A000057
:103294003C680000746D00006C3E00003C6200005D
:1032A4006F6400007920000073740000796C0000E2
:1032B400653D0000226D0000617200006769000036
:1032C4006E3A0000313000003070000078220000B7
:1032D4003E3C0000666F0000726D0000206D00002F
:1032E40065740000686F0000643D0000706F0000AA
:1032F400737400002061000063740000696F0000B3
:103304006E3D0000222F0000757000006C6F0000FD
:103314006164000022200000656E000063740000F8
:1033240079700000653D0000226D0000756C00009E
:103334007469000070610000727400002F66000060
:103344006F7200006D2D0000646100007461000064
:10335400223E00003C6200003E4D0000504600004A
:1033640053200000496D00006167000065200000E3
:10337400557000006C6F0000616400003C2F000079
:10338400623E00003C7000003E3C0000696E00009C
:1033940070750000742000007479000070650000EE
:1033A4003D660000696C0000652000006E6100004D
:1033B4006D6500003D69000020730000697A00001B
:1033C400653D0000343000003E200000266E000001
:1033D40062730000703B0000203C0000696E000036
:1033E400707500007420000074790000706500009E
:1033F4003D730000756200006D69000074200000D8
:10340400766100006C750000653D000022550000E7
:10341400706C00006F610000642200003E3C0000FC
:103424002F6600006F7200006D3E00003C2F00000C
:10343400626F0000647900003E3C00002F680000C9
:10344400746D00006C3E00000048000054540000FD
:10345400502F0000312E00003120000032300000D7
:10346400302000004F4B00000D0A0000436F0000A5
:103474006E6E000065630000746900006F6E0000EA
:103484003A200000636C00006F730000650D0000BB
:103494000A4300006F6E0000746500006E74000043
:1034A4002D54000079700000653A0000207400007B
:1034B40065780000742F0000687400006D6C0000D3
:1034C4000D0A00000D0A00003C680000746D000045
:1034D4006C3E00003C6200006F6400007920000034
:1034E40073740000796C0000653D0000226D0000DB
:1034F40061720000676900006E3A0000313000001C
:1035040030700000782200003E3C0000623E000063
:103514004D50000046530000205500007064000028
:1035240061740000652000005375000063630000AF
:103534006573000073660000756C00003C2F00008A
:10354400623E00003C7000003E3C00006120000030
:1035540068720000656600003D2200002F22000012
:103564003E53000069740000652000006D61000096
:10357400696E00002070000061670000653C000077
:103584002F6100003E3C00002F6200006F640000C9
:10359400793E00003C2F0000687400006D6C000050
:1035A4003E00000048540000545000002F31000039
:1035B4002E3100002035000030300000204900008A
:1035C4006E740000657200006E6100006C200000E3
:1035D400536500007276000065720000204500000B
:1035E400727200006F7200000D0A0000436F000049
:1035F4006E6E000065630000746900006F6E000069
:103604003A200000636C00006F730000650D000039
:103614000A4300006F6E0000746500006E740000C1
:103624002D54000079700000653A000020740000F9
:1036340065780000742F0000687400006D6C000051
:103644000D0A00000D0A00003C680000746D0000C3
:103654006C3E00003C6200006F64000079200000B2
:1036640073740000796C0000653D0000226D000059
:1036740061720000676900006E3A0000313000009A
:1036840030700000782200003E3C0000623E0000E2
:103694004D50000046530000204900006D610000B9
:1036A40067650000204300006F720000727500001F
:1036B40070740000206F0000722000005772000038
:1036C4006F6E0000672000005665000072730000F2
:1036D400696F00006E3C00002F6200003E3C000059
:1036E400703E00003C61000020680000726500002C
:1036F400663D0000222F0000757000006C6F000012
:1037040061640000223E0000547200007920000031
:1037140061670000616900006E3F00003C2F0000FB
:10372400613E00003C2F0000626F000064790000DD
:103734003E3C00002F680000746D00006C3E0000E9
:103744000048000054540000502F0000312E0000A7
:10375400312000003330000032200000466F0000AA
:10376400756E0000640D00000A4300006F6E0000D7
:103774006E65000063740000696F00006E3A00001B
:10378400206300006C6F0000736500000D0A0000E8
:103794004C6F000063610000746900006F6E0000EC
:1037A4003A2000000048000054540000502F00004C
:1037B400312E00003120000034300000332000009E
:1037C400466F0000726200006964000064650000D6
:1037D4006E0D00000A4300006F6E00006E6500006D
:1037E40063740000696F00006E3A000020630000FB
:1037F4006C6F0000736500000D0A00000D0A0000E4
:103804003430000033200000466F00007262000074
:1038140069640000646500006E3A000020530000F3
:10382400534C0000205200006571000075690000CF
:1038340072650000642000002D20000075730000F4
:10384400652000004854000054500000530D00004F
:103854000A0000002A9600002A9600004F960000F5
:10386400AD9600002E970000C89700003598000020
:10387400A59800000B99000011960000279A0000FB
:10388400D49A0000A39B0000D59B0000436F000066
:103894006F6B0000696500003A000000417500008C
:1038A400746800006F720000697A0000617400009F
:1038B400696F00006E3A0000004300006F6E000064
:1038C400746500006E7400002D4C0000656E0000ED
:1038D40067740000683A000000000000489C000083
:1038E400509C00005F9C000047450000540000000D
:1038F400504F00005354000000750000706C00002D
:103904006F610000640000007377000069740000B8
:10391400636800002E680000746D0000000D000054
:103924000A0D00000A330000303400002052000069
:10393400656400006972000065630000743A000069
:1039440020000000436F00006E740000656E0000EC
:10395400742D000054790000706500003A200000C6
:10396400004300006F6E0000746500006E74000078
:103974002D4500006E6300006F640000696E000056
:10398400673A0000206700007A690000700D0000AB
:103994000A0000004361000063680000652D000018
:1039A400436F00006E740000726F00006C3A0000F8
:1039B400200000006E6F00002D63000061630000B2
:1039C40068650000006D0000617800002D61000052
:1039D400676500003D000000363000003000000044
:1039E40053650000742D0000436F00006F6B0000EE
:1039F400696500003A200000000D00000A0D000077
:103A04000A0000000D0A00000D0A00004D500000DD
:103A14004653000002010000000000000000000006
:103A24000000000000000000000000000000000092
:103A34000000000000000000000000000000000082
:103A44000000000000000000000000000000000072
:103A54000000000000000000000000000000000062
:103A64000000000000000000000000000000000052
:103A74000000000000000000000000000000000042
:103A84000000000000000000000000000000000032
:103A94000000000000000000000000000000000022
:103AA4000000000000000000000000000000000012
:103AB4000000000000000000000000000000000002
:103AC40000000000000000000000000000000000F2
:103AD40000000000000000000000000000000000E2
:103AE40000000000000000000000000000000000D2
:103AF40000000000000000000000000000000000C2
:103B040000000000000000000000000000000000B1
:103B140000000000000000000000000000000000A1
:103B24000000000000000000000000000000000091
:103B34000000000000000000000000000000000081
:103B44000000000000000000000000000000000071
:103B54000000000000000000000000000000000061
:103B64000000000000000000000000000000000051
:103B74000000000000000000000000000000000041
:103B84000000000000000000000000000000000031
:103B94000000000000000000000000000000000021
:103BA4000000000000000000000000004375000059
:103BB40072720000656E00007420000053740000EF
:103BC40065700000203D0000202500006C75000099
:103BD400005400006172000067650000742000005A
:103BE4005374000065700000203D00002025000093
:103BF4006C750000004300007572000072650000DF
:103C04006E740000205000006F72000074200000E9
:103C14003D20000025750000005400006172000082
:103C24006765000074200000506F0000727400008B
:103C3400203D0000202500007500000049730000AD
:103C4400204D00006F760000696E000067200000C0
:103C54003D2000002575000000490000732000008D
:103C6400486F00006D6900006E670000203D000091
:103C74002025000075000000497300002048000062
:103C84006F6D000065640000203D000020250000E9
:103C9400750000004D610000676E0000657400004F
:103CA400203100002053000074610000746500009E
:103CB400203D000020250000750000004D6100003B
:103CC400676E00006574000020320000205300007D
:103CD4007461000074650000203D00002025000090
:103CE400750000004D610000676E000065740000FF
:103CF400205000006F73000069740000696F0000B9
:103D04006E2000003D200000256C000075000000BE
:103D1400000000000000000000000000000000009F
:103D2400000000000000000000000000000000008F
:103D3400000000000000000000000000000000007F
:103D4400000000000000000000000000000000006F
:103D5400000000000000000000000000000000005F
:103D6400000000000000000000000000000000004F
:103D7400000000000000000000000000000000003F
:103D8400000000000000000000000000000000002F
:103D9400000000000000000000000000000000001F
:103DA400000000000000000000000000000000000F
:103DB40000000000000000000000000000000000FF
:103DC40000000000000000000000000000000000EF
:103DD40000000000000000000000000000000000DF
:103DE40000000000000000000000000000000000CF
:103DF40000000000000000000000000000000000BF
:103E040000000000000000000000000000000000AE
:103E1400000000000000000000000000000000009E
:103E2400000000000000000000000000000000008E
:103E3400000000000000000000000000000000007E
:103E4400000000000000000000000000000000006E
:103E5400000000000000000000000000000000005E
:103E6400000000000000000000000000000000004E
:103E7400000000000000000000000000000000003E
:103E8400000000000000000000000000000000002E
:103E9400000000000000000000000000000000001E
:103EA4004E690000636B00006E6100006D650000E8
:103EB400203D000020250000730000004C45000058
:103EC400442000004272000069670000687400002A
:103ED4006E65000073730000203D00002025000083
:103EE400750000004D61000078200000537400004C
:103EF40065700000732000003D200000256C000068
:103F040075000000446500007669000063650000E8
:103F14002054000079700000652000003D2000005E
:103F240025730000004800006F6D0000652000004C
:103F34004F6E000020530000746100007274000092
:103F4400203D000020250000750000004D610000A8
:103F540078200000537000006565000064200000B4
:103F64003D20000025750000000000000000000056
:103F7400000000000000000000000000000000003D
:103F8400000000000000000000000000000000002D
:103F9400000000000000000000000000000000001D
:103FA400000000000000000000000000000000000D
:103FB40000000000000000000000000000000000FD
:103FC40000000000000000000000000000000000ED
:103FD40000000000000000000000000000000000DD
:103FE40000000000000000000000000000000000CD
:103FF40000000000000000000000000000000000BD
:1040040000000000000000000000000000000000AC
:10401400000000000000000000000000000000009C
:10402400000000000000000000000000000000008C
:10403400000000000000000000000000000000007C
:10404400000000000000000000000000000000006C
:10405400000000000000000000000000000000005C
:10406400000000000000000000000000000000004C
:10407400000000000000000000000000000000003C
:10408400000000000000000000000000000000002C
:10409400000000000000000000000000000000001C
:1040A400000000000000000000000000000000000C
:1040B40000000000000000000000000000000000FC
:1040C40000000000000000000000000000000000EC
:1040D40000000000000000000000000000000000DC
:1040E40000000000000000000000000000000000CC
:1040F40000000000000000000000000000000000BC
:1041040000000000000000000000000000000000AB
:10411400000000000000000000000000000000009B
:104124000048000069670000682000005370000028
:1041340065650000642000003D2000002575000036
:104144000044000065660000617500006C740000A6
:1041540020480000696700006820000053700000D8
:1041640065650000642000003D2000002575000006
:10417400004C00006F7700002053000070650000C1
:1041840065640000203D000020250000750000004B
:104194004465000066610000756C00007420000036
:1041A4004C6F00007720000053700000656500002C
:1041B400642000003D20000025750000004D000033
:1041C4006F760000696E00006720000043750000F0
:1041D40072720000656E0000742000003D20000033
:1041E400257500000044000065660000617500004C
:1041F4006C740000204D00006F760000696E0000B2
:10420400672000004375000072720000656E0000B4
:10421400742000003D2000002575000000480000C7
:104224006F6C0000646900006E67000020430000AA
:1042340075720000726500006E740000203D00007D
:104244002025000075000000446500006661000040
:10425400756C000074200000486F00006C6400005E
:10426400696E000067200000437500007272000050
:10427400656E0000742000003D20000025750000DC
:10428400004D0000617800002043000075720000BA
:10429400726500006E740000203D000020250000BF
:1042A40075000000705F000061700000705F000026
:1042B400636F00006E660000696700000073000011
:1042C400726300002F480000756200002F48000050
:1042D400756200002E63000000250000733A0000A0
:1042E4002569000020250000732000002D2D00000A
:1042F400206100007373000065720000746900009F
:104304006F6E000020660000616900006C650000AB
:10431400640A00000000000000000000000000002B
:104324000000000000000000000000000000000089
:104334000000000000000000000000000000000079
:104344000000000000000000000000000000000069
:104354000000000000000000000000000000000059
:104364000000000000000000000000000000000049
:104374000000000000000000000000000000000039
:104384000000000000000000000000000000000029
:104394000000000000000000000000000000000019
:1043A4000000000000000000000000000000000009
:1043B40000000000000000000000000000000000F9
:1043C40000000000000000000000000000000000E9
:1043D40000000000000000000000000000000000D9
:1043E40000000000000000000000000000000000C9
:1043F40000000000000000000000000000000000B9
:1044040000000000000000000000000000000000A8
:104414000000000000000000000000000000000098
:104424000000000000000000000000000000000088
:104434000000000000000000000000000000000078
:104444000000000000000000000000000000000068
:104454000000000000000000000000000000000058
:104464000000000000000000000000000000000048
:104474000000000000000000000000000000000038
:104484000000000000000000000000000000000028
:104494000000000000000000000000000000000018
:1044A4000000000000460000697200006D77000003
:1044B4006172000065200000566500007273000000
:1044C400696F00006E2000003D200000257500008B
:1044D4002E250000752E0000257500000043000005
:1044E4006F6D00006D6100006E64000020560000D6
:1044F40065720000736900006F6E0000203D0000CB
:1045040020250000752E0000257500002E250000D2
:104514007500000032300000313700002F300000F9
:10452400382F00003130000000520000656C00009C
:1045340065610000736500002044000061740000A0
:10454400652000003D20000025730000005300009A
:1045540065720000696100006C2000004E75000067
:104564006D62000065720000203D000020250000FF
:1045740075000000576900007265000064200000A7
:1045840049500000203D000020250000642E00005A
:10459400256400002E250000642E00002564000020
:1045A4000000000000000000000000000000000007
:1045B40000000000000000000000000000000000F7
:1045C40000000000000000000000000000000000E7
:1045D40000000000000000000000000000000000D7
:1045E40000000000000000000000000000000000C7
:1045F40000000000000000000000000000000000B7
:1046040000000000000000000000000000000000A6
:104614000000000000000000000000000000000096
:104624000000000000000000000000000000000086
:104634000000000000000000000000000000000076
:104644000000000000000000000000000000000066
:104654000000000000000000000000000000000056
:104664000000000000000000000000000000000046
:104674000000000000000000000000000000000036
:104684000000000000000000000000000000000026
:104694000000000000000000000000000000000016
:1046A4000000000000000000000000000000000006
:1046B40000000000000000000000000000000000F6
:1046C40000000000000000000000000000000000E6
:1046D40000000000000000000000000000000000D6
:1046E40000000000000000000000000000000000C6
:1046F40000000000000000000000000000000000B6
:1047040000000000000000000000000000000000A5
:104714000000000000000000000000000000000095
:104724000000000000000000000000000000000085
:1047340000500000726900006D6100007279000091
:10474400204400004E530000203D000020250000BE
:10475400642E0000256400002E250000642E000055
:1047640025640000004E000065740000776F0000AF
:10477400726B000020430000616200006C65000061
:10478400204300006F6E00006E650000637400003B
:1047940065640000203D0000202500006400000046
:1047A40044480000435000002043000068610000BA
:1047B4006E67000065640000203D000020250000B5
:1047C400640000004D4100004320000046720000D8
:1047D4006565000020520000782000003D200000A4
:1047E40025640000004D0000414300002049000002
:1047F400732000005478000020520000656100001E
:1048040064790000203D00002025000064000000C1
:1048140052650000636F00006E6E00006563000067
:1048240074200000436F0000756E000074200000C7
:104834003D200000256400000000000054680000D2
:104844006520000072650000636500006976000061
:1048540065640000206300006F6D00006D6100005E
:104864006E6400002069000073200000666F000081
:10487400726D000061740000746500006420000023
:10488400696E0000636F00007272000065630000CF
:10489400746C00007900000054680000652000007A
:1048A40072650000636500006976000065640000BD
:1048B400206300006F6D00006D6100006E640000F5
:1048C4002077000061730000207400006F6F000007
:1048D400206C00006F6E0000670000005468000048
:1048E40065200000726500006365000069760000C1
:1048F40065640000206300006F6D00006D610000BE
:104904006E640000206300006F6E0000746100009C
:10491400696E000065640000206900006E76000086
:10492400616C000069640000207000006172000086
:10493400616D000065740000657200007300000082
:104944005468000065200000726500006365000083
:104954006976000065640000206900006465000059
:104964006E74000069660000696500007220000032
:1049740077610000732000006E6F00007420000057
:1049840072650000636F0000676E0000697A0000C2
:1049940065640000005400006865000020630000A6
:1049A4006F6D00006D6100006E64000020720000F5
:1049B40065630000656900007665000064200000FE
:1049C4007761000073200000666F00007220000011
:1049D400616E0000206900006E760000616C0000CA
:1049E40069640000207400006172000067650000C3
:1049F40074200000646500007669000063650000AF
:104A04000054000068650000206300006F6D000022
:104A14006D6100006E6400002069000073200000D6
:104A2400696E0000766100006C690000642000007B
:104A3400626500006361000075730000652000007A
:104A44007468000065200000646500007669000059
:104A5400636500002069000073200000686F000097
:104A64006D6900006E670000005400006865000076
:104A7400206300006F6D00006D6100006E64000033
:104A84002069000073200000696E00007661000058
:104A94006C6900006420000077680000696C000005
:104AA400652000006E6F000020740000656D00003A
:104AB400706500007261000074750000726500008A
:104AC40020700000726F0000626500002069000021
:104AD40073200000617400007461000063680000CA
:104AE400656400002E00000054680000617400003A
:104AF4002064000065760000696300006520000002
:104B04007479000070650000206400006F65000087
:104B1400732000006E6F00007420000065780000B0
:104B240069730000742E00000045000072720000DA
:104B34006F7200002074000065780000742000008B
:104B44006E6F000074200000646500006669000058
:104B54006E65000064000000556E00006162000094
:104B64006C650000207400006F200000636F00007B
:104B74006E6E00006563000074200000746F000016
:104B8400205700006946000069200000426F0000C1
:104B940061720000640000004E6500007720000090
:104BA4005769000046690000207300006574000026
:104BB400746900006E6700007320000061720000D9
:104BC40065200000696E0000636F000072720000CF
:104BD4006563000074000000546800006520000054
:104BE400636F00006D6D0000616E000064200000C2
:104BF40066610000696C00006564000020620000CA
:104C04006563000061750000736500002074000096
:104C14006865000020730000656C00006563000097
:104C2400746F0000722000006973000020640000AB
:104C340069730000636F00006E6E0000656300001E
:104C440074650000640000005468000065200000E2
:104C5400636F00006D6D0000616E00006420000051
:104C640066610000696C0000656400002062000059
:104C74006563000061750000736500002074000026
:104C84006865000020730000656C00006563000027
:104C9400746F00007220000069730000206E000031
:104CA4006F740000206800006F6D000065640000F0
:104CB400005400006869000073200000766500005D
:104CC40072730000696F00006E2000006F660000C0
:104CD400207400006865000020460000697200002E
:104CE4006D7700006172000065200000646F0000B1
:104CF40065730000206E00006F74000020730000D4
:104D040075700000706F0000727400002063000072
:104D1400686100006E670000696E00006720000093
:104D24007461000072670000657400007320000065
:104D340077680000696C0000652000006D6F00005A
:104D4400766900006E6700000000000070720000C9
:104D54006F7400006563000074000000736E00004F
:104D64006D70000000610000646D0000696E000059
:104D7400006D000069630000726F0000636800004A
:104D84006970000000730000656E00006443000059
:104D94006D64000000730000656C00006563000032
:104DA400746F0000722E0000687400006D00000033
:104DB400707200006F74000065630000742F0000BF
:104DC400636F00006E660000696700002E680000D3
:104DD400746D000000690000700000006777000037
:104DE4000073000075620000006400006E73000030
:104DF40031000000646E000073320000006D00009A
:104E040061630000006800006F730000740000001C
:104E14006468000063700000002F000070720000DE
:104E24006F74000065630000742F00007265000059
:104E3400626F00006F7400002E680000746D000043
:104E44003F0000002F700000726F000074650000C6
:104E5400637400002F6300006F6E00006669000039
:104E6400672E0000687400006D00000041750000AA
:104E74006720000031300000203200003031000093
:104E840037200000313200003A350000303A00008B
:104E94003434000000760000352E00003432000067
:104EA400006E0000616D0000650000006E6F000080
:104EB4007420000073650000740000003C62000070
:104EC4003E550000706C00006F610000642000001B
:104ED40061200000466900006C6500003C2F000062
:104EE400623E00000063000068650000636B000020
:104EF4006564000000660000616900006C00000049
:104F04005468000065200000447900006E610000D0
:104F14006D69000063200000444E0000532000002F
:104F2400436C0000696500006E7400002069000095
:104F3400732000006E6F000074200000656E000096
:104F4400616200006C650000642E0000006E0000C9
:104F54006F6E000065000000626C00006F6300006B
:104F64006B000000000000000000000000000000D2
:104F7400000000000000000000000000000000002D
:104F8400000000000000000000000000000000001D
:104F9400000000000000000000000000000000000D
:104FA40000000000000000000000000000000000FD
:104FB40000000000000000000000000000000000ED
:104FC40000000000000000000000000000000000DD
:104FD40000000000000000000000000000000000CD
:104FE40000000000000000000000000000000000BD
:104FF40000000000000000000000000000000000AD
:10500400000000000000000000000000000000009C
:10501400000000000000000000000000000000008C
:10502400000000000000000000000000000000007C
:10503400000000000000000000000000000000006C
:10504400000000000000000045740000682000001B
:10505400536F0000636B000065740000204400007F
:1050640069730000636F00006E6E000065630000EA
:1050740074200000436F0000756E0000743A000055
:10508400203D00002025000075000000457400004C
:1050940068200000536F0000636B0000657400001B
:1050A400204300006F6E00006E6500006374000012
:1050B400204300006F7500006E7400003A20000069
:1050C4003D200000257500000045000074680000C4
:1050D4002042000079740000657300002052000033
:1050E400783A0000203D0000202500006C75000087
:1050F4000000000047450000544400004E4E0000EC
:1051040000470000455400005354000041000000D3
:105114004745000054430000464700000044000097
:105124004F480000414C000054000000534500006B
:10513400544400004E4E0000004400004F4800005C
:105144004F4D00004500000052450000534500004B
:105154005452000000530000455400004445000030
:105164005600000053450000544D00004853000011
:1051740000530000455400004D4C00005300000053
:1051840053450000544D0000484300000053000004
:10519400455400004D4C000043000000474500000A
:1051A400544D00004F530000004700004F500000D2
:1051B4004F520000540000005254000030300000F0
:1051C4003035000000530000455400004C450000F9
:1051D400440000004E690000636B00006E61000033
:1051E4006D650000203D00002000000025680000DF
:1051F400750000002575000000000000300000006C
:1052040073720000632F0000436C000069650000A6
:105214006E740000436F00006E6E00006563000052
:10522400746900006F6E0000732F0000436C00006F
:10523400696500006E7400002E6300000025000004
:10524400733A000025690000202500007320000047
:105254002D2D0000206100007373000065720000B2
:10526400746900006F6E0000206600006169000030
:105274006C650000640A00000021000000000000CA
:10528400004500004E440000007000005F63000011
:105294006C690000656E0000742D00003E7700000C
:1052A400726900007465000000450000525200005D
:1052B4004F52000020490000442000003D2000001F
:1052C4002564000000450000525200004F520000C7
:1052D4002054000045580000542000003D200000E8
:1052E4002573000000210000000000000000000001
:1052F40000000000000000000000000000000000AA
:10530400503D000025750000000000000000000072
:105314000000000000000000000000000021000068
:105324000033000000450000523D0000330000003F
:10533400455200003D340000004C00003D250000B3
:1053440075000000455200003D2500007500000076
:105354004D3D000025750000005300004E3D000047
:1053640025750000005600003D250000752E000044
:1053740025750000257500000048000000000000AD
:105384004745000054430000464700000047000022
:10539400455400004442000047000000524500000C
:1053A400424F00004F5400000052000045530000DB
:1053B40045540000480000004745000054450000E3
:1053C40044490000005300004554000044530000C9
:1053D4004E000000257500000053000045540000F5
:1053E4000000000008000000C80000002C010000BC
:1053F40008000000C80000002C01000008000000A4
:10540400C80000002C0100000A0000000001000098
:10541400800000000A00000000010000800000007D
:105424000A00000000010000800000000D0A0000D6
:1054340044480000435000002F5000006F770000E4
:105444006572000020650000766500006E7400003F
:10545400206F000063630000757200007265000035
:105464006400000000040000A3000000000000002D
:105474005065000072730000657500007300000041
:105484004D500000465300000201000000000000DF
:020000040000FA
:105494000200FA00004F7800C4D0BF009E4F5000B5
:1054A4001B003200C4D0BF00E24F40000A003200AB
:1054B400C4D0BF000080FB007E00B90080007800EB
:1054C400C080200000804000419220000E000900AE
:1054D40031187800E001B1001E407800C4F0B70034
:1054E400E0CFB3009E4F1000090032001E80FB0085
:1054F4007E00B90080007800C08020000080400059
:10550400419220000E000900B0187800E001B100BB
:105514000080FA00000006000000FA00510C21008F
:1055240091407800C4D0BF0080CF500024003200E6
:10553400C5D0BF00E24F400016003200008C2000AE
:1055440000017800C5D0BF000080FB007E00B900D8
:10555400FC004000C08020000080400090427800A1
:10556400C5D0BF000080FB007E00B9008000780039
:10557400C0802000008040009000780080FD2F0053
:10558400008040008402200013C0B30085407800EE
:10559400E3100700C4D0BF00C5F0B7000394200097
:1055A400934178002149800080FD2F000081400054
:1055B400008C20008402200011C0B300D810070022
:1055C4000080FA00000006000C00FA0040F92000F8
:1055D400000F7800308680000000E00008003A00E8
:1055E40028A602000000000080007800F07F200060
:1055F40080806000004020000080400030868800E9
:10560400808E2000C20320008000EB00D807020037
:10561400000000000040EB00204F98000040EB0029
:10562400304F98004A0037003E48900098FF07002A
:105634003E4890000080FB006600B90080007800BE
:10564400409F2A000080400090409000214798002D
:105654003E4890000080FB006600B9008080E800AE
:10566400409F2A0000804000900078004107980085
:105674003E4890000080FB006600B900E400400052
:10568400409F2A0000804000900078003107980075
:105694002E4090000080FB000000E000010032007A
:1056A4002A0037001E00780020079800CE009000E2
:1056B4003E009000008040001E004000A102200037
:1056C400010F400000ED21009E0F1000FDFF3E0081
:1056D4002E40900040E9B7002E0090008002B000F8
:1056E40020498800214980004E009000008040003D
:1056F4000000E80030498800314980003E009000F5
:105704000080400040498800D0002000D049880033
:105714003C69A90080FF07003E4890000080FB0020
:105724006600B90080007800409F2A000080400095
:1057340010407800E7E8B700D30A07003E4890001D
:105744000040E800304F980001003700FFFF3700A9
:105754003E489000E54F5000B3FF36000080FA0049
:10576400000006001200FA001007980021079800B4
:105774006247980043079800244F98000040EB00CC
:10578400004F7800940037001E40780040FF070067
:10579400D0498000ED0F50008E003A005EFF0700F4
:1057A400718E2000914078002E48900080CF5000E8
:1057B40088003A0080212000204788006E40900035
:1057C4000004E00008003A004E0090008046880083
:1057D4003C69A80040002000D0498800CE00900019
:1057E400F14988007800370031868000F03F2000BE
:1057F400808F5000040036003186800080382100FC
:10580400808F50000200360000402000308688005F
:1058140030868000804688000000E80030868800DA
:105824004E00900070468800F6FC02000000000064
:1058340090498800A14988003C89A8006E409000E6
:105844000080FB00000F98008E089000E38F50004A
:10585400220032000E089000E30F500004003C00C8
:105864008E089000E18F5000570035000400370087
:105874000E089000E40F50002F0032005200370051
:105884001E009000AE009000B0468800C14688001B
:105894008040EB00614F98006E409000E24F500052
:1058A40002003A0010C0B300604F9800EE48900028
:1058B4000180FB00610060004201DD0011478000AF
:1058C400B0FF2F00008060000200700010478800C5
:1058D4000000EB00D04988003B0037000E80E80050
:1058E400900090000E80E800100078008080400056
:1058F4004E00900080804000804680000080680058
:10590400F04988001E009000AE009000B046880068
:10591400C14688000040EB00E6E8B700800920009B
:105924000100200000468800114688002000200065
:10593400D0498800240037001E009000AE0090007B
:1059440080007800214090000081FB0031409000ED
:105954000080FB004800DD000200700000017800B8
:105964001E009000AE0090009080FB00104090005C
:105974000080FB004800DD00010070008000410051
:105984004E009000808040008046800000806800C7
:10599400F04988001E009000AE009000800078005E
:1059A400608D20000900090031587800A000B10082
:1059B400A100B10050002000D049880011C0B300FC
:1059C40020C0B300EE0607001E80FB0060079800AD
:1059D400060037001E4FE80051C0B3009ECF1000F0
:1059E40069FF3600E00F2000600798006E00900009
:1059F4000080FA00000006000400FA00004F78005E
:105A040050C0B3009E4F1000030036001000200069
:105A1400100798000D0037001E4078009CFE070018
:105A2400E049800001002100010060000000E00066
:105A3400040032003D89A9001000200010079800DE
:105A4400020037000000EB00100798001E009000D1
:105A54000080FA00000006000400FA00004F7800FD
:105A640050C0B3009E4F1000030036008000EB00CE
:105A740011079800090037001E40780084FE0700D3
:105A8400D04980008000EB0011079800E70F500018
:105A940002003A0010002000100798001E00900039
:105AA4000080FA00000006000400FA00004F7800AD
:105AB40050C0B3009E4F10004B003E001E407800C3
:105AC40073FE07007049800080498800D049800037
:105AD400100798001E009000E50F50001F003200D0
:105AE4001E009000E50F50000A003E001E009000CA
:105AF400E10F5000150032001E009000E10F50002D
:105B0400160039001E009000E30F500032003E00E2
:105B1400120037001E009000EB0F50001E003200F0
:105B24001E009000EB0F500004003E001E00900089
:105B3400E70F500028003E000A0037001E009000C6
:105B4400EE0F50002100320023003700F8AD0200B0
:105B540000000000CC09070023003700CA09070031
:105B64002100370011C0B30010C1B3008406070040
:105B7400904680000000E00004003200514980009B
:105B840060468000808F5000F6FF3A0080002000BD
:105B9400D04988001400370011C0B30010C1B3000D
:105BA40077060700904680000000E0000400320001
:105BB4005149800060468000808F5000F6FF3A0013
:105BC400C0002000D049880007003700D000200022
:105BD400D0498800040037008040EB0040C1B30086
:105BE40067060700A80907000080FA000000060005
:105BF4000200FA00004F780050C0B3009E4F10001E
:105C040005003E001E40780021FE07003C69A90003
:105C14001E407800A4FF07000080FA000000060080
:105C24000400FA00004F780050C0B3009E4F1000EB
:105C3400030036008000EB00110798000B003700CA
:105C44001E40780012FE070033FE0700008020008B
:105C5400618D2000090009003158780070468000E9
:105C64005040880000802000100798001E0090001B
:105C74000080FA00000006000200FA00004F7800DD
:105C840050C0B3009E4F10000A003E001E40780032
:105C9400FFFD070020FE0700514980006046800098
:105CA400808F50000300320011C0B30000C1B30064
:105CB400330607000080FA00000006000600FA0020
:105CC400204798002E409000E54F50000300360016
:105CD4000000EB0020079800200037002E409000C1
:105CE400EBFD0700D0498000004F780070C0B3007E
:105CF4009E4F100006003200B0C0B3009E4F10004B
:105D0400030032000000EB00200798001300370066
:105D14005149800060498000808F50000A0039009A
:105D24003149800020498000008150006149800091
:105D34005049800000805000000041000000E9004C
:105D44002007980005003700604980005149800011
:105D5400010050000000E900200798002E00900088
:105D64000080FA00000006000600FA0020479800B0
:105D7400314798002E409000E54F50000300360054
:105D84000000EB0020079800400037002E409000F0
:105D9400BFFD07002E409000C8FF0700000F7800E9
:105DA4001E00E00003003A000000EB00200798000A
:105DB40036003700100020009E0F100002003A0049
:105DC4002E409000ACFF0700E04980000110200045
:105DD400010060000000E00009003A003149800041
:105DE40020498000008050000000D1009E0F500028
:105DF400030039002E4090009FFF07003D09A800D2
:105E0400630047000001780001942000914078006D
:105E1400504980001400200013C0B300C00E0700D6
:105E2400504980000000E800504988005149800032
:105E340030498000808F50000200390020498000E2
:105E440050498800100020009E0F100003003A0003
:105E54002E40900088FF07000A003700E0498000C8
:105E640001022000010060000000E00005003A008B
:105E74003CA9A8001EFD02000000000078004000BC
:105E8400B049880010002000200798002E009000E0
:105E94000080FA00000006000E00FA006047980037
:105EA40041079800520798000000EB00000F7800AB
:105EB4006E409000E54F5000030036000000EB00F8
:105EC400600798005E0037006E40900070FD070088
:105ED4006E40900079FF0700100798001E009000A4
:105EE4000000E00005003A006E40900062FF0700E9
:105EF4000000EB0060079800510037001E0090007E
:105F0400200798009E0090005E009000808F500053
:105F1400020036005E00900020079800E0498000EF
:105F240001102000010060000000E0000A003A00B7
:105F34003149800020498000008050008000D10059
:105F44001E009000808F5000030039006E409000C6
:105F540049FF07003D09A800514980002E00900028
:105F64008080400030498000808F50001400390048
:105F74003149800050498000008F50004E0090004D
:105F8400000178000194200091407800504980007D
:105F94001E02780013C0B300610E07009E00780053
:105FA4004E00900001004000400798002E00900031
:105FB4001E005000200798002049800050498800A6
:105FC4004E00900000017800019420009140780078
:105FD400504980002E02900013C0B300500E0700F9
:105FE400514980002E0090000080400050498800F4
:105FF4009E0090005E009000808F500003003E00E1
:106004006E4090001CFF07000A003700E049800042
:1060140001022000010060000000E00005003A00D9
:106024003CA9A8001EFD020000000000780040000A
:10603400B04988002E0090001E00400060079800C0
:106044006E0090000080FA00000006000400FA00D0
:10605400004F7800110798001E009000CA08020043
:1060640000000000000178009E0090001E407800AF
:1060740089FF0700800078001E0090000080400027
:106084000080FA00000006000800FA00404798006B
:106094004E409000E54F5000030036000000EB0036
:1060A400300798000C0037004E409000F8FC0700C1
:1060B400314980002049800000805000000FE90031
:1060C4004E409000FDFE0700100798001E0090004F
:1060D4001E001000300798003E0090000080FA0077
:1060E400000006000200FA00004F78001E4078000D
:1060F4000B0007000000E000070032001E4078009B
:10610400E3FC0700704980008049880011C0B30097
:1061140000C1B3001A0507000080FA000000060061
:106124000400FA00004F780050C0B3009E4F1000E6
:10613400030036000000EB0010079800140037003D
:106144001E407800D2FC070071498000804980001D
:10615400808F50000500390071498000804980001B
:1061640080805000110798000900370041498000E1
:1061740080498000008150007149800030498000CE
:1061840000805000000041000000E8001007980063
:106194001E0090000080FA00000006000800FA00CB
:1061A40020479800210798002E409000DCFF07004C
:1061B400000F78001E00E00003003A000000EB002E
:1061C40030079800270037002E409000B0FC0700ED
:1061D4002E0090000000E00008003200019420002E
:1061E40091407800824980002E0090001400200025
:1061F4008141780011C0B300C90D070080498000B7
:106204000000E800804988008149800040498000FE
:10621400808F500002003600304980008049880099
:10622400100020009E0F100002003A003D49A80013
:106234000A003700E04980000102200001006000EC
:106244000000E00005003A003CA9A8001EFD020081
:1062540000000000A007B000B04988001000200032
:10626400300798003E0090000080FA00000006000D
:106274000C00FA0040479800310798004207980044
:106284000000EB00000F78004E409000A4FF0700D0
:10629400100798001E0090000000E00003003A0080
:1062A4000000EB00500798004C0037004E4090006F
:1062B40077FC0700CE0090001E009000808F5000F5
:1062C400020036001E0090004007980081498000BB
:1062D4004E0090008080400040498000808F500034
:1062E4001800360041498000804980000080500039
:1062F400000FE8003E0090000000E0000C003200B7
:106304000194200091407800824980003E00900072
:106314001E0278008141780011C0B300800D07008F
:106324009E0078003E009000010040003007980075
:106334004E0090001E005000400798003049800035
:10634400804988003E0090000000E0000800320010
:106354000194200091407800824980003E00900022
:106364004E0290008141780011C0B3006C0D07000B
:10637400814980004E0090000080400080498800E0
:106384004E0090001E004000400798009E009000C0
:106394004E009000808050004E009000808F50008E
:1063A40002003E003D49A8000A003700E049800091
:1063B40001022000010060000000E00005003A0036
:1063C4003CA9A8001EFD020000000000A007B000C8
:1063D400B04988004E009000500798005E0090007D
:1063E4000080FA00000006000800FA004047980008
:1063F4004E409000E54F5000030036000000EB00D3
:10640400300798000B0037004E40900020FC070036
:106414004149800030498000008F50004E40900078
:106424003FFF0700100798001E0090001E00100098
:10643400300798003E0090000080FA00000006003B
:106444001000FA006047980041079800520798002E
:10645400630798006E409000E54F500003003E0033
:106464005E0090000000E00003003A000000EB0032
:1064740070079800450037006E40900004FC070048
:106484006E40900026FF070010079800EE00900071
:106494005E009000808040001E009000808F5000BD
:1064A400040036001E009000EE0090000100500031
:1064B40050079800814980006E00900000804000E1
:1064C40020079800414980002E009000808F5000E2
:1064D400070031003149800040498000808050002D
:1064E4002E009000008040000000E9002007980082
:1064F400414980002E00900000805000000FE80009
:106504005E0090009E0F50000A003E0040C9BF008C
:10651400CE009000810278005E02900080417800F5
:106524002E01900011C0B30005007800FC0C070098
:106534001400370001942000914078004E00900030
:106544001E027800814178002E01900011C0B30032
:10655400F30C07005E0090009E005000029420009F
:1065640012417800354980004E0090001E00400022
:1065740001027800824178000501780011C0B3005F
:10658400E70C07005E009000700798007E00900002
:106594000080FA00000006000600FA002047980078
:1065A40021079800AE019000120020008E007800B0
:1065B4002E409000A2FF07001E4078000080FB00E0
:1065C4000080FA00000006004000FA0020779800DE
:1065D400211F9800321F9800431F9800541F9800F1
:1065E400651F98002E709000E54F500003003E0098
:1065F4003E1890000000E00003003A000000EB00A9
:10660400701F9800320137002E709000A0FB070025
:106614002E709000C2FE0700800078004E18900093
:106624000080500070079800FE0090003E18900013
:10663400808F5000030031008080EB00711F9800B0
:10664400230137005E1890000000E00006003200CD
:10665400FE0090005E189000808F5000020036000B
:106664005E18900070079800814980004E189000D1
:106674000080400050079800414980005E0090006F
:10668400808F50000700310031498000404980006C
:10669400808050005E009000008040000000E9000F
:1066A40050079800DE009000010F980041498000D7
:1066B4005E009000008050000000E8006007980031
:1066C4004E18900050079800BE189000410798009B
:1066D4002E189000300798002E18900090407800F3
:1066E400314798002E1890000000E800201F980001
:1066F4000000EB00000F78006E1890000000E0002E
:106704000C003200BE40900000C6B30080CF5000A1
:1067140008003600BE409000A0C7B30080CF5000F0
:1067240004003E003E40900001CEB3000140400012
:106734003047980000C2B300204798002E409000D4
:106744008080FB006E009000808F500002003600B5
:106754006E009000204798002E4090008080FB003F
:106764007E009000808F5000020036007E00900072
:10677400204798002E4090008080FB000294200067
:1067840012417800720047000102780082417800CB
:106794000E09900011C0B300610C07002E40900058
:1067A4008080FB000E08900001004000000F98005C
:1067B4002E4090008080FB006E009000010050008D
:1067C400600798006E0090000000E00004003A00AA
:1067D40030498000000F98000080EB0060079800AB
:1067E4006E1890000000E0006F0032000040EB00E3
:1067F40040479800670037004E4090008080FB00BF
:1068040072004700008040009040780000C6B3004A
:1068140080CF5000160036004E4090008080FB0070
:10682400720047000080400090407800A0C7B30089
:1068340080CF50000E003E004E4090000081FB00CF
:106844004E4090008080FB007200470000804000B2
:10685400104078008040780000CEB30000C04000B3
:106864008040780072004700000041000148780031
:106874004E4090008080FB00720047000080400082
:10688400904078003E40900080CF500024003A00B1
:106894003E1890000000E900301F98003E18900058
:1068A4000000E00009003A00DE0090004E00900075
:1068B400808050004E4090000080FB00008040002B
:1068C4000000E800701F9800810037002E18900027
:1068D40090407800314798002E1890000000E8009E
:1068E400201F980010002000000F7800BE40900088
:1068F40000C6B30080CF500023003600BE40900095
:10690400A0C7B30080CF50001F003E003E4090005F
:1069140001CEB30001404000304798001A00370010
:106924004E009000301F98001E00E0001600320058
:10693400BE009000211F98002E189000904078000F
:10694400314798002E1890000000E800201F98009E
:10695400BE40900000C6B30080CF5000080036004F
:10696400BE409000A0C7B30080CF500004003E009A
:106974003E40900001CEB3000140400030479800F3
:106984000000EB00000F78004E4090000040E8004B
:1069940040479800CE4090002E40900080CF500099
:1069A40095FF3900380037000040EB00404798005D
:1069B400310037004E4090008080FB007200470099
:1069C40000804000904078003E40900080CF50000E
:1069D40018003A003E1890000000E900301F9800AB
:1069E4003E1890000000E00009003A00DE0090002C
:1069F4004E009000808050004E4090000080FB00CC
:106A0400008040000000E800701F9800300037004C
:106A14002E18900090407800314798002E1890006E
:106A24000000E800201F980010002000000F7800EC
:106A34000E0037004E009000301F98001E00E0004A
:106A44000A003200BE009000211F98002E1890000A
:106A540090407800314798002E1890000000E8001C
:106A6400201F98000000EB00000F78004E409000BB
:106A74000040E80040479800CE4090002E4090002F
:106A840080CF5000CBFF39002E4090008080FB0067
:106A94007E0090000100500070079800FE009000F6
:106AA4003E189000808F5000030031000080EB00FE
:106AB400701F9800060037002E4090008080FB0075
:106AC4005E009000010040005007980019FF370055
:106AD4007E1890000080FA00000006000800FA000A
:106AE400004F780011479800120798002307980078
:106AF400340798008E00E800BE0290002E02900039
:106B04009E019000120020001E407800AEFE070097
:106B14000080FA00000006001400FA00881F7800C4
:106B24000040EB00004F9800FD0137000E48900034
:106B340057FA07000040EB00204798000000EB00E4
:106B4400300798000000EB0020079800E14980001E
:106B540000202000008060000000E00005003A00F2
:106B6400E049800001402000010060000000E000D6
:106B74000B003200D2660200000000000000E000BA
:106B84000700320000C1B30020479800E0498000AC
:106B94004A00DE00614060000080FB00300798007E
:106BA400E049800001022000010060000000E000D4
:106BB40008003200B84980001EFD020000000000F9
:106BC400000054000000E00002003C0000C1B300DB
:106BD40020479800E0498000010420000100600083
:106BE4000000E00008003200C84980001EFD0200D9
:106BF40000000000000054000000E00002003C001F
:106C040000C1B30020479800D0498000EB0F50002A
:106C14000A003A00C84980001EFD0200000000007E
:106C2400000054000000E00004003C0010C1B30068
:106C340020479800C0002000D0498800D049800037
:106C4400E40F500056003A000000EB00000F7800FB
:106C5400500037001E0078007400B900F0004000B6
:106C6400808E200000804000100078000000E000CA
:106C74004B0032001E0078007400B900F0004000A0
:106C8400808E20000080400090007800F049800051
:106C9400808F50003E003A001FFA07001E00780063
:106CA4007400B90080007800808E200000804000CD
:106CB400618D200009000900B0587800A000B100DF
:106CC4001E0078007400B900EA004000808E2000A5
:106CD4000080400010007800704688001E00780094
:106CE4007400B900EC004000808E20000080400059
:106CF4001000BE0061004000E0804800404688006B
:106D040051468800C1468000B04680008080400023
:106D140070468000808040008046800000806800CB
:106D2400F049880020C1B30020479800600020008B
:106D3400D0498800220020001E0051007400B900D0
:106D4400000178001E0078007400B900800078000B
:106D5400C08F200000804000800278001E00780070
:106D64007400B90080007800808E2000008040000C
:106D74000202780013C0B3000501780011C0B3000B
:106D8400E70A07000000EB00004988000400370010
:106D94001E0FE800230020009E8F1100ADFF360077
:106DA4002E4090000004E0000A0032000040EB0096
:106DB400604F98003E0090000000E00002003A009E
:106DC40011C0B300614F9800EE4890002E4090002F
:106DD400EB010700E0498000700060000000E00063
:106DE4002C003A00D0498000E70F500049013A00D6
:106DF400F6FC0200000000000001BE009049800083
:106E0400A14980000000510081805900E00F50002A
:106E1400E08F58003F013500E049800067006000C2
:106E2400E60F50000E003A00E04980004300DE0007
:106E340061406000204798000E4890001AFB07004C
:106E44000E48900018FB07002E4090000004E0005C
:106E540030013A00E0002000D04988002D013700BD
:106E6400ADF9070021C0B30000C1B300C40107009D
:106E7400F6FC02000000000042782D00730120009F
:106E8400000041008180490090498800A1498800A0
:106E940020013700F6FC0200000000000001BE00E3
:106EA40090498000A1498000000051008180590070
:106EB400E00F5000E08F58001601350096F90700E6
:106EC400D04980006101B800020F9800130F9800A8
:106ED400C0002000010020000E0990009E099000CF
:106EE400800F5100818F5900D8003E000E08900099
:106EF4009E089000006001000C003700210037005C
:106F04004A00370052003700D000370075003700C0
:106F14008200370095003700A1003700AD0037002C
:106F2400B100370091003700BC003700DCAD02002F
:106F3400000000000000E000C40032001000200047
:106F4400D049880010478000640060000000E00021
:106F540006003200B0468000C146800011C0B30074
:106F64001EAE020000000000B8003700B0468000EA
:106F7400C146800011C0B3001EAE02000000000034
:106F8400B20037006A0047004EAE02000000000065
:106F94000000E000AD003200F8AD02000000000087
:106FA4000000E000150032005E009000EE0090004A
:106FB400B0468800C146880020002000D0498800DF
:106FC400C1468000B046800080804000704680004A
:106FD400808040008046800000806800F04988007E
:106FE4000040EB00E6E8B700800920000100200023
:106FF400004688001146880094003700F6FC020021
:10700400000000000001BE0040782D007101200046
:10701400020040008380480090498800A14988000C
:107024000000EB00D0498800880037001EFD0200F4
:1070340000000000B0498800608D2000E8D0020004
:107044000000000030002000D04988007F00370095
:10705400A18D2000608D2000B4D10200000000004A
:107064000000E00018003A001EFD020000000000CD
:1070740080007800B0498000008150000046800004
:1070840011468000800F510070003600E6C8BF0032
:10709400E54F500009003E00E6C8BF000040E8008C
:1070A400E6E8B7000046800011468000000040007A
:1070B4008180480000468800114688002000200096
:1070C400D04988006100370020C0B30020479800F1
:1070D4000000EB003007980050002000D0498800E1
:1070E4005A00370020C0B300204798001000200049
:1070F40030079800E6C8BF00E14F50005300360047
:1071040020C0B300E6E8B700404B2C00410020004B
:1071140000468800114688004C003700E6C8BF00CE
:10712400E14F500005003E0020C1B3002047980005
:10713400100020003007980044003700E049800028
:10714400680060000000E0000500320040C1B300A8
:107154002047980010002000200798003B003700CB
:1071640020C0B3002047980038003700E6C8BF00AD
:10717400E24F500005003E0000C1B30020479800D4
:1071840010002000300798003000370080002000F5
:10719400D049880010C1B300204798002B00370065
:1071A400E6C8BF00E24F500005003E0010C1B30026
:1071B4002047980010002000300798002300370073
:1071C40040C1B30020479800100020002007980019
:1071D4001E00370040C1B300204798001000200073
:1071E4002007980019003700E6C8BF00E24F50009E
:1071F40005003E0000C1B3002047980010002000A5
:10720400300798001100370040C1B30020479800B0
:1072140010002000200798000C003700E6C8BF00CB
:10722400E24F500005003E0010C1B3002047980013
:1072340010002000300798000400370040C1B3005C
:107244002047980010002000200798002E4090004E
:107254000004E0002B0032003E0090000000E0003B
:1072640025003200E6C8BF000040E800E6E8B700A9
:1072740000468000114680000000400081804800E4
:1072840000468800114688006146800060498000FD
:10729400008F50006146800060498000808F50005C
:1072A4000400310030498000214980000100500071
:1072B4001E0F400022468000334680001E007800E6
:1072C4000100200000005100818059002046880000
:1072D40031468800904680001E0040009046880099
:1072E40060498000604688008040EB002E4090009A
:1072F400A30007000300370011C0B3002E40900024
:107304009F0007002E0090000000E0000100320002
:10731400DD0307000E4890000040E800004F98008D
:107324000E489000E54F500000FE36000000EB00D0
:10733400000F78002D0037001E0078007400B9009B
:10734400F0004000808E2000008040001000780093
:107354000000E000280032001EFD020000000000D2
:10736400000178001E0078007400B900F2004000AB
:10737400808E2000008040001000780080005100C2
:1073840070722000808F500017003600210020000A
:107394001E8050007400B900000178001E007800BF
:1073A4007400B90080007800C08F20000080400085
:1073B400800278001E0078007400B9008000780014
:1073C400808E2000008040000202780013C0B300C9
:1073D4000501780011C0B300510907000000EB005B
:1073E400004988001E0FE9001E0FE800220020005B
:1073F4009E0F1100D0FF36004F0478000080FA0081
:10740400000006002E00FA0030179800411798007B
:1074140052179800BE1090001182FB00114090009A
:107424000080FB004800DD000400700000017800CB
:10743400214090000082FB00314090000080FB005E
:107444004800DD00040070008001780076004700E9
:107454000288BE004E1090001000BE007601470066
:107464002001980031019800F60047000040EB002D
:1074740080489800F600470060C0B3009048980028
:1074840076004700DE109000510098007600470017
:1074940050009000BEAB02000000000080007800A5
:1074A400760047005100980076004700C100200094
:1074B40036AC0200000000000080EA0010179800BB
:1074C4005E109000DA6A02000000000020179800A5
:1074D4009E1090002E109000808F50000500320006
:1074E400EA66020000000000100020006017980007
:1074F400200037000000EB0064F9020000000000E7
:107504000E80E80041012000926D0200000000009E
:107514000E80E800250307000E80E800600090005C
:107524004400DE006F4060004200DD00744F5000F4
:107534009E80FB005E10900001005000740050001B
:10754400501798000E80E800BE109000FC01070060
:107554000000E000030032000E80E800DE1090001E
:10756400E5030700EA6602000000000011002000A5
:10757400611798006E1090000080FA000000060069
:107584002A00FA00006F9800116F9800E2F70700D4
:107594000E6890000080FB00610060000004E000C1
:1075A400050032003D69A8000E689000E1CFB300E9
:1075B40001406000006F98003CA9A9003CC9A900E3
:1075C4003CE9A9003D29A9003D49A9003D09A900BC
:1075D400D2660200000000000000E000FCFF320060
:1075E4000E6890000080FB00660060000000E00070
:1075F400030032000000EB00000F78007D0037002C
:107604005149800060468000808F500003003A009A
:107614000000EB00000F780068003700514980003B
:1076240060468000808F5000190036005049800069
:1076340061468000010F5000904680009E0F50006C
:107644000200310090468000000F7800204780003F
:107654009E0F50000300310021478000010F780085
:107664003D49A80040C9BF00624680001E02780060
:10767400804178008040EB00909D2000A80807001E
:10768400604680001E004000604688004B003700C2
:107694003149800060468000808050007C004700B3
:1076A400510098007C004700D000900050498000B1
:1076B4008080400020498000008F50009046800068
:1076C4009E0F50000200310090468000000F7800A9
:1076D400204780009E0F50000300310021478000A6
:1076E400010F78003D49A8007C004700500090003D
:1076F4009E0F5000030036007C0047009E00780077
:10770400510098007C004700500090000194200034
:107714009140780062468000000278008141780040
:107724008040EB00909D20007D0807007C0047000E
:10773400500090009E0010007C004700510098000B
:107744007C004700500090000000E0000E00320072
:107754007C0047005001900003942000934178007E
:1077640025498000314980006046800080805000B7
:10777400909D2000008040000202780005017800FE
:107784008040EB0066080700604680001E00400051
:10779400604688006146800030498000808F500038
:1077A400060039006246800031498000204980008B
:1077B400008050000000510060468800E0498000CD
:1077C40001802000010060000000E0000900320098
:1077D400904680009E0F5000060032002047800033
:1077E4009E0F5000030032000E6890000004A000B9
:1077F400006F98001E00E00005003A000E6890003B
:107804000080FB00630060000000E0001D00320007
:10781400904680001E005000904688001E00E00044
:10782400030032000E6890000034A000006F98003E
:107834001E6890000080FB00610060000004E0000E
:10784400060032000040EB00E6E8B700D012230047
:10785400110020000046880011468800F6FC020052
:107864000000000002468000134680000000410032
:107874008180490090498800A14988003C89A8007A
:10788400370037001E6890000080FB000000D10024
:10789400610060000004E00014003200E049800050
:1078A400674060000040E800674060000080FB0023
:1078B40067016000E149800080FF2F0000806000C4
:1078C40002007000E04988002046800031468000B4
:1078D40061005000E080580020468800314688004E
:1078E40010002000000F78001D003700E0498000E0
:1078F400700060000000E000190032001E68900073
:107904000080FB00610060000000E0000C003A0011
:10791400E6C8BF000004E00009003200E6C8BF006A
:107924000040E900E6E8B700004680001146800008
:107934008100D1000080D3000046880011468800F1
:10794400F6FC02000000000002468000134680009E
:10795400000041008180490090498800A1498800C5
:107964008146800064004700010878007146800069
:1079740064004700110098002046800031468000D2
:1079840064014700200198003101980040468000BE
:10799400514680006401470040019800510198005D
:1079A40064014700E2009000F0FF230000806000C3
:1079B4006001980064014700E200900000FF2F007E
:1079C4000080600060019800640047008E689000A9
:1079D40051489800E40047000000EB00900898002C
:1079E40022468000334680001E00780001002000FB
:1079F4000200400083804800204688003146880009
:107A04000E6890000080FB000000D100610060005F
:107A14000004E0001E0032000E6890000080FB00AD
:107A24004400DE00610060000000E00004003A0051
:107A3400640147006000B8004001980051019800BB
:107A440010478000620060000000E000090032007E
:107A540064004700B00090002000900061005000D6
:107A6400E08058006401470020019800310198002B
:107A74000700370020468000314680006100400046
:107A8400E08048002046880031468800E228A800AB
:107A94000E6890000080FB00610060000004E000BC
:107AA40001003200E208A80071498000804980008A
:107AB400808F50000A00390041498000304980001D
:107AC400008150007149800080498000008050008E
:107AD40080005100640047007100980006003700E0
:107AE4008149800070498000008050008000E900D6
:107AF40064004700710098001E6702000000000047
:107B0400100798009E009000F0032000808F500022
:107B140003003E000000EB0010079800040037004B
:107B24001E00900001FC2F00010040001007980087
:107B340064004700F00090001E009000808F500009
:107B4400030036009E009000640047007100980016
:107B540064004700950107001E007800740F400080
:107B640064014700E2009000F0F02F000080600004
:107B74000105200001007000600198000E6890006B
:107B84000080FB000000D100610060000004E00000
:107B9400170032009E007800648F400020C0B300BC
:107BA400005F980040C0B300105F9800208021005F
:107BB400500F980064004700600090004400DE000D
:107BC4006F4060000040E8006F406000E40147003F
:107BD4000080FB006F0060004401DD00E3009000C2
:107BE400F0F02F000080600002007000E0019800B7
:107BF4005ACBBF008080FB005BCBBF000080FB0042
:107C04004800DD0001007000000178005CCBBF007B
:107C14008080FB005DCBBF000080FB004800DD00DE
:107C240001007000800178007C0047000288BE00DB
:107C3400B0468000C14680007C01470020019800C6
:107C440031019800FC0047000040EB008048980098
:107C5400FC00470060C0B300904898007C004700D7
:107C64009E007800510098007C004700500090006E
:107C7400BEAB020000000000800078007C004700DA
:107C8400510098007C004700C100200036AC02007F
:107C9400000000008080EA006400470001089800AA
:107CA400109B2000266A0200000000001E017800DC
:107CB40061C0B300608D2000C6F80200000000001F
:107CC4006400470041012000A46E0200000000008F
:107CD4000E6890000080FB000000D100610060008D
:107CE4000004E00004003200780047004100200056
:107CF400A46E020000000000509C2000546A0200A0
:107D0400000000001E007800DA6A02000000000093
:107D140010079800509D2000266A02000000000011
:107D24000E80E80021002000A46E02000000000084
:107D3400DC680200000000000080FA000000060079
:107D44000C00FA00881F780030079800410798005B
:107D54003E009000100090000000E00003003A0094
:107D64000000EB00500798000C013700E0CFB3008F
:107D740040479800CE009000214090000081FB0015
:107D8400314090000080FB004800DD0002007000DC
:107D9400000178004E0090009080FB00104090009D
:107DA4000080FB004800DD000100700080004100FD
:107DB4003E00900010007800808040003E0090005B
:107DC4001000900000806800100798000040EB004D
:107DD40050479800380037005E409000ACF507002B
:107DE400D0498000ED0F500030003200D0498000AF
:107DF400E40F500008003A00F0498000BE009000F3
:107E040091009000810F500028003A00DE4090005D
:107E14004147980025003700F14980001E0090007A
:107E2400808F500021003A00BBF507003E0090000F
:107E34009000900080468000808F50001B003A0024
:107E44003E0090009000780070468000808F5000C3
:107E540016003A00CE0090001182FB001140900001
:107E64000080FB004800DD00040070000001780081
:107E7400214090000082FB00314090000080FB0014
:107E84004800DD000400700080017800B0468000E6
:107E9400C1468000800F5100818F590003003A00D1
:107EA4001000200050079800BC0037005E4090008E
:107EB4000040E800504798005E409000E54F5000B5
:107EC400C5FF36004E409000E24F400018003200DB
:107ED4004E4090006EF507008FF507004E4090006D
:107EE400E24F4000120032009E009000F1498800E9
:107EF4004E009000618D200009000900B058780000
:107F0400A000B1003E009000100078007046880088
:107F14003E009000100090008046880020498000B8
:107F24006046880010002000500798009B0037002E
:107F34003E009000E00090000020200000806000DF
:107F44000000E00003003A008000EB0051079800B5
:107F540092003700004980000000E0000300320076
:107F64000000EB00500798008C0037000000EB0085
:107F7400000F7800400037001E0078007400B9003C
:107F8400F0004000808E2000008040001000780047
:107F94000000E0003B0032001E0078007400B900CD
:107FA400F0004000808E20000080400090007800A7
:107FB4003E00900010009000808F50002D003A0089
:107FC4001E0078007400B900EA004000808E200092
:107FD40000804000900078003E009000100078007F
:107FE400808F500023003A001E0078007400B9000E
:107FF40080007800808E2000008040001003BE00C6
:10800400CE0090001182FB00114090000080FB0024
:108014004800DD0004007000000178002140900059
:108024000082FB00314090000080FB004800DD002E
:108034000400700080017800820F5300838F5B007E
:108044000C003A001E0478001EFD0200000000002F
:10805400000178007440B900F2004000808E2000D6
:1080640000804000020878008000EB00510798006F
:108074004A0037001E0FE800200020009E0F100069
:10808400BDFF36000040EB00504798003E0037002B
:108094005E409000FEF40700E04980006800600044
:1080A4000000E000350032001BF507008046800028
:1080B400BE00900091009000810F50002F003A0004
:1080C4001E0078007400B90080007800808E2000C3
:1080D400808040004E00900009000900B0587800EC
:1080E400A100B100A000B1009E0078003E00900005
:1080F400100178007408B900EA004000808E200066
:1081040000804000020878009E0078003E00900045
:1081140020019000B00190007408B900EC00400008
:10812400808E2000008040000288BE009E007800FF
:108134003E009000100190007408B900F000400067
:10814400808E200000804000020878001E04780021
:108154001EFD020000000000000178007440B90018
:10816400F2004000808E2000008040000208780069
:108174008000EB0051079800080037005E40900033
:108184000040E800504798005E409000E54F5000E2
:10819400BFFF36000000EB00500798005E0090001F
:1081A4004F0478000080FA00000006000200FA0084
:1081B400000F78001E00780010007800BEAB0200AB
:1081C40000000000800078001E007800010878009C
:1081D4001E00780010009000BEAB020000000000FA
:1081E400800078001E007800110098001E007800BE
:1081F400B000900020009000D8AB02000000000006
:108204001E01780020019800310198001E007800BA
:10821400D000900040009000D8AB020000000000A5
:108224001E01780040019800510198001E0078005A
:1082340070009000BEAB02000000000080007800D7
:108244001E007800710098001E007800000890005D
:10825400BEAB020000000000800078001E00780021
:10826400010898001E00780010089000BEAB0200C0
:1082740000000000800078001E00780011089800BB
:108284000080FA00000006000200FA00881F78004F
:10829400A1F4070080468000F0498800204980004E
:1082A4005049880020498000604988003049800096
:1082B400704988003049800080498800E049800086
:1082C400680060000000E00003003200400020006D
:1082D400000F780002003700D0002000000F780063
:1082E4001E007800D04988003C09A9003C29A90057
:1082F4003C49A9003C89A9003CA9A9003CC9A900A2
:108304003CE9A9003D09A9003D29A9003D49A9006E
:108314003D69A9003D89A800E208A900E228A90056
:10832400E268A900E288A90020498000604688002C
:10833400488C2000BAA5020000000000000C780060
:10834400488C2000BAA50200000000001004980028
:108354000080EB0000478800100020009046880051
:108364004F0478000080FA00000006000600FA00BE
:10837400881F7800C000200064F90200000000009B
:10838400606D020000000000104798001E4090003D
:108394008080FB00000F2000008060004280DE002F
:1083A40074405000104798001E4090000004E00004
:1083B40003003A0080212000200798004A0037007B
:1083C400710020000000EB00926D0200000000002C
:1083D4003D003700606D020000000000004F78008F
:1083E4001E04E0003E00320010C0B3009E4F100097
:1083F4003500320020C0B3009E4F100022003A0026
:108404001E409000E24F5000350036000000EB00A3
:1084140010079800606D020000000000004F780013
:1084240040C0B3009E4F100009003A000E80E800DF
:108434000004E800606D020000000000004C7800B9
:108444000E84E800606D020000000000004C78001B
:108454009E00900070212000808F50002000360084
:108464009E009000405B2000808F50000300360087
:10847400405B2000200798001B0037001E0090007E
:1084840020079800180037001E409000E14F50006C
:1084940013003600606D020000000000004F7800F9
:1084A4001E4090009E4F50000D0039009E80FB003E
:1084B4000000EB00926D0200000000001E409000DE
:1084C4001E405000104798001E4090000040E900F4
:1084D400104798001E409000E14F4000BDFF3A0055
:1084E40080212000200798002E0090004F0478007F
:1084F4000080FA00000006002800FA00700F9800BF
:10850400011798007E089000D0489000614F9800B1
:108514007E08900040019000D0019000520798001E
:10852400630798007E08900020019000B00190003D
:1085340032079800430798003C09A9003C29A90088
:108544003C49A900E0498000700060000000E000A0
:1085540008003A00F6FC02000000000042782D00FA
:108564007301200000004100818049009049880087
:10857400A1498800D3498000331798003E10900029
:10858400E40F500004003200BE109000E58F50004C
:108594002E0032007D0037006E4890000080FB0002
:1085A4004200DE00610060000004E00002003200CE
:1085B40035FF0700170437006E4890000080FB0069
:1085C4004400DE00610060000004E00009003200A5
:1085D4005E019000EE019000224688003346880038
:1085E4008040EB0040C0B300E5FB070026FF070016
:1085F400080437006E4890000080FB000000D100A2
:10860400610060000004E0000E0032003E009000B3
:10861400CE00900061004000E080480040468800A1
:108624005146880051FF07002047880011C0B3005D
:1086340020C1B300D2FB070060002000D0498800AD
:10864400F403370010FF0700F20337006E48900070
:108654000080FB004200DE00610060000004E000D6
:10866400EC033A006E4890000080FB004400DE00FA
:10867400610060000004E000170032002246800020
:10868400334680005E009000EE009000800F5100A1
:10869400818F59001000320020468000314680004E
:1086A40030079800410798005E019000EE019000A9
:1086B400224688003346880011C0B30040C0B3008E
:1086C400AFFB07003E009000CE00900020468800DB
:1086D40031468800CF0337006E4890000080FB00CD
:1086E4000000D100610060000004E000C903320012
:1086F4003E009000CE00900061004000E080480001
:1087040040468800514688007E0890007000900022
:108714009046880015FF0700204788006E489000A7
:108724000080FB004400DE00610060000004E00003
:108734001000320011C0B30000C1B30090FB070069
:1087440070002000D0498800F6FC02000000000000
:108754000001BE0040782D0071012000020040009D
:108764008380480090498800A14988003C89A90079
:10877400A803370011C0B30020C1B30080FB070079
:1087840060002000D0498800A20337008E109000BA
:10879400210798006E4890000080FB006100600093
:1087A4000004E000030032002E0090000000E80006
:1087B400200798006E4890000080FB000000D10064
:1087C400610060000004E000030032002E0090000D
:1087D4000000E8002007980071498000804980006B
:1087E400808F5000090039004149800030498000E1
:1087F4000081500071498000804980000080500051
:1088040000005100000F98000500370081498000E6
:1088140070498000008050000000E900000F9800BB
:1088240042468000534680003E009000CE009000F7
:108834000200500083805800200F9800310F9800E8
:108844002E099000120F98000000EB00100798000A
:108854002E0090000000E000350032000E08900069
:108864000000E000480032002E089000BE0890008E
:10887400E00F5000E08F58000A0035000E08900009
:108884006101B8002E089000BE089000800F5100CE
:10889400818F590003003600100020001007980053
:1088A400140037002E0090006101B8002E089000DB
:1088B400BE0890000200400083804800E00F500092
:1088C400E08F58000B0034008E0890002E009000BA
:1088D400008050006101B9002E089000BE0890008D
:1088E400800F5100818F59000200350010002000D4
:1088F400100798000E0890006101B8002E0890003F
:10890400BE089000800F5100818F59001E00340072
:108914001E089000AE009000010040000000E0003E
:1089240019003400100020001007980016003700CA
:108934002E089000BE089000E00F5000E08F580011
:1089440003003A0010002000100798000E003700C2
:108954002E089000BE089000E00F5000E08F5800F1
:10896400090035000E0890006101B8002E0890003F
:10897400BE089000800F5100818F5900020036001C
:1089840010002000100798001E0090000000E00076
:108994000A003A006E4890000080FB004200DE00AE
:1089A400610060000000E0001A033A0011C0B30047
:1089B40000C1B300F2FA0700160337006E489000B6
:1089C4000080FB00660060000000E000020032004E
:1089D4002DFE07000F0337006E4890000080FB0057
:1089E4004400DE00610060000000E0000903320082
:1089F400D3498000231798002E109000EB0F5000ED
:108A040007003E00AE109000E78F500021003100B7
:108A14002E119000E60F5100050032006701370067
:108A2400AE119000EC8F5100590132006301370000
:108A340022468000334680005E009000EE009000E5
:108A4400800F5100818F59001000320020468000B1
:108A54003146800030079800410798005E0190007D
:108A6400EE019000224688003346880011C0B3000E
:108A740040C0B300C2FA07003E009000CE00900050
:108A84002046880031468800E2023700700020004A
:108A9400D049880051498000604680000080500021
:108AA400400F98004E0890000000E00006003D00D2
:108AB4003149800020498000808050004E08900099
:108AC40001004000400F9800224680003346800099
:108AD4004E089000010020000200400083804800FE
:108AE400500F9800610F98005E019000EE01900015
:108AF4005E089000EE08900000005100818059004B
:108B0400500F9800610F98005E089000EE089000E6
:108B1400E00F5000E08F580015003400104780002B
:108B2400610060000000E000070032005E09900070
:108B3400EE0990001000200001002000800F510079
:108B4400818F5900040032008040EB0000C1B30063
:108B54008BFA0700AF0237005E009000EE00900031
:108B640061005000E08058005007980061079800A9
:108B740022468000334680006146800060498000C0
:108B840000805000CF80DE00000051008180590039
:108B9400500F9800610F9800614680006049800082
:108BA400808F50000A003100314980002049800044
:108BB400008050006101B8005E089000EE0890004B
:108BC4000200500083805800500F9800610F9800F5
:108BD4005E019000EE0190005E089000EE089000A7
:108BE4000000510081805900500F9800610F9800D7
:108BF4005E089000EE089000E00F5000E08F5800EF
:108C04005200340031498000204980000080500027
:108C14006101B8005E089000EE089000800F5100DA
:108C2400818F590049003900E268A900E288A9004F
:108C34003D09A90061498000410F98006149800005
:108C44005E08900000804000604988006146800012
:108C54004E089000808F500011003900614680005A
:108C640060498000808F500023003100224680003C
:108C740033468000614980006046800000805000D7
:108C84000100200002004000838048002046880044
:108C9400314688006049800060468800160037002D
:108CA40062468000314980002049800000805000E5
:108CB40000004100400F9800614980004E08900078
:108CC400808F50000C00360022468000334680001E
:108CD400614980004E08900000805000010020008F
:108CE4000200400083804800204688003146880006
:108CF40060498000604688006149800030498000F6
:108D0400808F50000600390062498000314980009C
:108D14002049800000805000000051006049880014
:108D24006146800030498000808F50003000390057
:108D34006246800031498000204980000080500054
:108D44000000510060468800290037006149800016
:108D540060468000808F500025003200104780005C
:108D6400680060000000E00020003200104780002E
:108D7400700060000000E0001B003200224680000A
:108D840033468000614680006049800000805000C6
:108D9400CF80DE0000005100818059002046880009
:108DA400314688006146800060498000808F500011
:108DB4000A00310022468000334680003149800099
:108DC4002049800000805000CF80DE000000510068
:108DD400818059002046880031468800604980001F
:108DE400604688003D49A800E288A800E268A8001F
:108DF4006149800050498000808F50001C003A0077
:108E0400E049800001802000010060000000E000D3
:108E14000A003A00F6FC02000000000042782D002F
:108E240073012000000041008180490090498800BE
:108E3400A14988003C89A9000D0037002246800022
:108E4400334680005E009000EE009000800F5100D9
:108E5400818F590006003A001047800061006000CD
:108E64000000E000020032003C89A9003D69A9002D
:108E74007E089000700190002046800031468000FA
:108E8400800078005E00900000805000000F5100C8
:108E9400904680000000E00003003A001E00E0005D
:108EA400010032003D29A8001E0178009246880086
:108EB400D0498000E80F500018003A002246800094
:108EC400334680005E009000EE009000800F510059
:108ED400818F590039003A0010478000610060001A
:108EE4000000E00035003200F6FC02000000000043
:108EF4000001BE0020BC2E00B10020000200400092
:108F04008380480090498800A14988003C89A800D2
:108F140090002000D049880028003700D049800004
:108F2400E90F50000E003A006E4890000080FB00EC
:108F3400610060000000E00020003A005E00900044
:108F4400EE00900020468800314688008040EB0007
:108F540040C1B3008AF90700CBFC0700AD0137001C
:108F6400D0498000EA0F500014003A0022468000E5
:108F7400334680005E009000EE009000800F5100A8
:108F8400818F5900A3013A00BFFC0700A1013700FB
:108F9400204680003146800061014000E0814800A5
:108FA4005E009000EE009000800F5100818F590008
:108FB40098013A00B4FC0700960137006E4890000F
:108FC4000080FB004500DE00610060000004E0005A
:108FD40090013A00D0498000EB0F50008D0132001F
:108FE400D0498000EA0F50008A013200D049800045
:108FF400EC0F5000870132000E1090000000E000DA
:10900400180132001E0890000000E0007B003C00C4
:109014007E089000600090004400DE006F40600015
:109024000080FB004200DD00800078001E089000F4
:109034000080500064F90200000000008E109000CF
:109044001E08900000804000001798008E109000C9
:109054000E089000808F5000020036008E089000A9
:109064000117980042468000534680000E1090007D
:109074000100200002004000838048004046880030
:1090840051468800714980000E1090008080400095
:1090940040498000808F50001E0036004149800006
:1090A40070498000008050000000E800400F9800E4
:1090B4000194200091407800704980004E0A90008D
:1090C4008041EB000081EB00150207008E10900038
:1090D4004E089000008050000194200091407800D8
:1090E40035498000000278008041EB000081EB00EC
:1090F400050078000A020700324980008E109000B3
:109104004E08900000805000000041007049880023
:109114000B003700019420009140780070498000D2
:109124000E1290008041EB000081EB00FC0107006F
:10913400714980000E109000008040007049880042
:1091440000478000E10F4000C60032000047800065
:10915400800078000E1090000080500000478800C6
:10916400A14680000047800000804000400F980026
:109174004E0890000000E00003003D000080EB007A
:1091840000478800B7003700004780000000E00077
:10919400B4003C0042468000534680004E089000D4
:1091A40001002000020040008380480040468800FF
:1091B40051468800714980004E08900000804000AC
:1091C400704988007149800040498000808F5000B8
:1091D4000700360072498000314980004049800010
:1091E40000805000000041000000E9007049880040
:1091F4000080EB00004788009A0037001E089000AA
:109204000000E000970034008E1090001E089000CB
:10921400808040000E089000808F500004003600CB
:109224000E0890009E08900001005000001798005E
:109234007E089000600090004400DE006F406000F3
:109244000080FB004200DD0064F902000000000021
:10925400714980001E089000808040000E1090002C
:109264008080400040498000808F500030003600EC
:109274004149800070498000808050001E089000A1
:10928400008050000000E800400F98004E08900055
:109294000000E00016003500059420009542780097
:1092A400714980001E089000008040004E0A900022
:1092B4008041EB000081EB008540780098010700B5
:1092C4008E1090004E089000008050000194200001
:1092D4009140780035498000000278008041EB001D
:1092E4000081EB00050078008D0107001A003700AB
:1092F4000594200095427800714980001E08900072
:1093040000814000314980004049800000805000C5
:10931400000041000000E9000E1290008041EB00C3
:109324000081EB00854078007D0107000A003700CA
:109334000594200095427800714980001E08900031
:10934400008040000E1290008041EB000081EB0091
:10935400854078007201070000478000E10F40005B
:1093640005003A001E089000004788000E11900086
:10937400A24688003B003700004780008000780048
:109384001E089000808F50001C0036009E0890003C
:109394000E1090000081400000478000800078009B
:1093A400A046800000804000800F510006003E006F
:1093B4009E0890000E1090008080400000478000BE
:1093C400808F5000030031008E119000A346880066
:1093D400070037000047800080007800A046800026
:1093E400808040001E08900000805000A046880045
:1093F4001E089000004788001A0037009E0890005D
:109404000E1090000081400000478000800078002A
:10941400A046800000804000800F510011003600FB
:109424000047800080007800A046800080804000D3
:109434001E089000808F50000A003900A246800068
:109444009E0890000E10900080804000004780002D
:1094540080805000A0468000008050000000410041
:10946400A04688002E0090000000E0001A003200A0
:10947400D0498000E70F500002003200704980009C
:1094840080498800E0498000010820000100600054
:109494000000E0000500320011C0B30000C1B300B9
:1094A40037F807001CF007000B0037003CE9A80060
:1094B400E049800001042000010060000000E00099
:1094C40005003A003CC9A8001EFD0200000000008F
:1094D400D003B000C04988006E4890000080FB00B3
:1094E400610060000004E0004A0032004046800051
:1094F4005146800061024000E08248002E00900046
:109504006101B8003E009000CE00900002004000CF
:1095140083804800800F5200818F5A003D003A003A
:10952400404680005146800061004000E0804800D1
:109534004046880051468800D049800010179800A2
:109544009E109000E78F5000140032001E1190000E
:10955400E70F510004003E009E119000E68F510079
:1095640008003200280037001E109000E80F500059
:10957400110032009E109000E98F50001D0032004F
:1095840021003700C0002000D049880011C0B3007A
:1095940010C1B300FAF707001E003700B000200026
:1095A400D04988001EFD020000000000A007B000A2
:1095B400C0498800140037002246800033468000EA
:1095C4005E009000EE009000800F5100818F5900E2
:1095D40005003A008040EB0000C1B300E8F7070043
:1095E40029FB07000B003700A0002000D0498800A9
:1095F400050037008040EB0000C1B300E0F707002E
:1096040021FB07000300370011C0B30000C1B30001
:10961400DBF707000080FA00000006001000FA00E3
:10962400604798004107980052079800434F9800FC
:109634006E409000E54F5000030036000000EB0040
:1096440070079800B30037006E40900090EF070059
:109654004E0090000000E00002003A0010002000DC
:109664004007980041498000204980000080500054
:109674000000E90020079800CE0090005E009000F2
:10968400808040002E009000808F50000300360040
:109694000000EB00700798009E0037009EEF070063
:1096A4004E4890000080FB00630060000000E00072
:1096B40003003A004E4890003040B300404F9800F9
:1096C4005E009000000F7800CE0090005E009000D5
:1096D400808040002E009000010050002007980078
:1096E4004E4890000080FB000000D1006100600043
:1096F4000004E0000B0032004E4890000080FB00A4
:10970400610060000004E000040032002E009000BC
:109714000000D1001E0F4000020037002E00900010
:109724001E0F4000204980001E0040000000E80099
:1097340020079800704980001007980000478000B7
:10974400E10F4000120032000047800080007800E2
:10975400A0468000808040001E0090000100400070
:1097640010079800414980001E009000808F50002F
:10977400070031003149800040498000808050005A
:109784001E009000008040000000E90010079800CF
:10979400814980001E009000808F5000120031002B
:1097A400814980002E009000808F500028003100F5
:1097B4004E4890000080FB004200DE006100600023
:1097C4000004E000030032000000EB007007980082
:1097D400500037002E009000804988002E00900031
:1097E400704988001A003700814980001E009000EB
:1097F400808F500012003600314980002E00900006
:10980400808F5000120031004E4890000080FB0011
:109814004200DE00610060000004E000030032004A
:109824000000EB00700798003A0037002E0090000B
:10983400804988002E009000704988000400370099
:109844002E009000804988002E0090007049880006
:10985400814980001E009000808F50001D0036005A
:109864004E4890000080FB004200DE006100600072
:109874000004E00017003200314980001E0090000F
:10988400010050000194200091407800324980008A
:109894000594200095427800000278008141780008
:1098A400854078002E0090001D000700714980005B
:1098B40080498000808F500006003100724980008A
:1098C400314980002E0090000080500000005100BB
:1098D400704988002E00900030498800204980009B
:1098E4006046880020498000604988002049800043
:1098F40050498800D0498000E70F500003003A0027
:1099040011C0B30000C1B3001DF707001000200010
:10991400700798007E0090000080FA0000000600A6
:109924001000FA00000F78002147980022079800E1
:1099340063479800440798006E4090000080FB0045
:10994400700798007E0090000000E0001F003200C5
:109954007E009000E10F5000010032003900370012
:109964002E4090000080FB00600798006E0090007D
:109974000000E0000A0032006E009000E10F500089
:10998400010032002F003700AE0090001E00780066
:109994004E019000F6080200000000002900370084
:1099A4000080EB009E0F1000030032001E007800C0
:1099B400266A0200000000002E009000CE009000F5
:1099C400A46E0200000000001E0037002E4090002C
:1099D4000080FB00500798005E0090000000E0004B
:1099E4000F0032005E009000E10F500001003200D1
:1099F400140037002E009000E10F400003003200F5
:109A04002E009000546A0200000000001E0078003E
:109A1400CE009000926D02000000000009003700A3
:109A24004E019000AE0090001E0078008E6B020084
:109A340000000000486D0200000000000000E0008B
:109A4400FCFF32000080FA00000006000800FA0063
:109A5400008FBE001E00BE0020079800310798004A
:109A640070002000010020002E019000BE01900033
:109A7400800F5100818F59002900320070002000AE
:109A8400010020002E019000BE019000800F5100C3
:109A9400818F59000D003E002E009000BE00900002
:109AA400E00F5000E08F5800170032002000200023
:109AB400010020002E019000BE019000800F510093
:109AC400818F5900130032001E00370080002000EF
:109AD400010020002E019000BE019000800F510073
:109AE400818F5900110032009000200001002000F5
:109AF4002E019000BE019000800F5100818F59000B
:109B04000D0032000F00370020542900A60B070077
:109B140018003700D0542900A30B070015003700A4
:109B2400EA9B02000000000012003700409C020083
:109B3400000000000F0037006E9C020000000000CF
:109B44000C0037008355290056CBBF000080FB0072
:109B5400E1B420004200DD000080E8000100400084
:109B64001040780042002000830078004E2F02004D
:109B7400000000000080FA00000006000000FA0067
:109B840056CBBF000080FB00E1B420004200DD00A2
:109B94000080E8000100400010407800E1C7B300F5
:109BA400B62E0200000000000080FA00000006004B
:109BB4000200FA00881F78000040EB0056EBB70063
:109BC4002D00370056CBBF000080FB00E1B420001D
:109BD4004200DD00810040000000EB0080087800B6
:109BE40056CBBF000084FB0084C0B30003052000F3
:109BF4000041EB006000B800B42B0200000000003C
:109C040000417800E1B420004240DD000080E8001B
:109C1400010040000248780000C0EB00CCEAB70025
:109C240000C0EB00CDEAB70056CBBF008080FB003C
:109C3400600920000088B9008000780000ED210050
:109C440000804000266A020000000000000F780037
:109C540080AB200061092000A46E02000000000017
:109C64001E007800266A02000000000056CBBF00E8
:109C74000040E80056EBB70056CBBF00E14F500060
:109C8400D0FF36000040EB0056EBB7004F047800DD
:109C94000080FA00000006000200FA000040EB0019
:109CA400004F78004C0037001E80FB00E1B4200018
:109CB4004200DD000080E800010040001040780010
:109CC400E24F4000430032001E80FB00E1B420005C
:109CD4004200DD000080E8000100400010407800F0
:109CE400FE2C0200000000000000E000250032000D
:109CF4001E4078003D00070056CBBF000080FB00EB
:109D0400E1B420004200DD00810040000000EB00CF
:109D140080087800CCCABF00E14F40000500320043
:109D2400CCCABF00F87F02000000000000C0EB00B6
:109D3400CCEAB700CDCABF00E14F400005003200B5
:109D4400CDCABF00F87F02000000000000C0EB0095
:109D5400CDEAB70056CBBF000080FB00E1B4200081
:109D64004200DD000080E80001004000104078005F
:109D740043C0B3000001EB0011002000104B0200AF
:109D8400000000001E80FB00E1B420004200DD0062
:109D940001004000100078000000E0000A003A00D2
:109DA4001E80FB00E1B420004200DD000080E800DA
:109DB40001004000104078009230020000000000D2
:109DC4000000E000030032001E4078000700070096
:109DD400330007001E4FE80010C0B3009E4F100070
:109DE400B1FF36000080FA00000006000400FA000B
:109DF4002047980061B52000914078002E409000E3
:109E0400814F50002400320056CBBF008080FB00FD
:109E1400600920000088B9008000780000ED21006E
:109E240000804000266A020000000000000F780055
:109E340080AB200061092000A46E02000000000035
:109E44001E007800266A0200000000002E409000E8
:109E54008080FB00600920000088B9008000780041
:109E640000ED210000804000546A02000000000060
:109E7400000F780080AB200061092000926D020081
:109E8400000000001E007800546A02000000000078
:109E94002E40900056EBB7000080FA000000060048
:109EA4002A00FA00881F780010002000100798008C
:109EB40056CBBF000080FB00E1B420004200DD006F
:109EC40001004000100078006101B80002179800FA
:109ED40013179800B0002000010020000E1190001C
:109EE4009E119000800F5100818F59003F063E0063
:109EF4000E1090009E109000006001000B003700CF
:109F04004200370005023700D50237000C03370042
:109F140016033700B0033700D4033700C2043700F8
:109F2400D2053700F20537001006370056CBBF00C4
:109F34000080FB00E1B420004200DD000080E80066
:109F44000100400010407800923002000000000040
:109F5400400798004E0090000000E0002306320005
:109F640040AD20004056880056CBBF000080FB0067
:109F7400E1B420004200DD00810040001000200018
:109F84008008780000C0EB00CFEAB7000040EB0087
:109F9400CEEAB700F6FC0200000000000001BE009B
:109FA400209D2400B1062000020040008380480068
:109FB40000568800115688000080EB008080EB007A
:109FC40020568800315688006000B800C0558800CB
:109FD400D15588000040EB004CEBB70056CBBF00D6
:109FE4000080FB00E1B420004200DD000080E800B6
:109FF400010040001040780053C0B3000001EB00A2
:10A0040011002000104B02000000000056CBBF00DE
:10A014000080FB00E1B420004200DD000080E80085
:10A0240001004000104078000002EB008001EB00CA
:10A034000001EB00A1C0B300703502000000000075
:10A04400E10F400033003A0056CBBF000080FB0014
:10A05400E1B420004200DD000080E800010040007F
:10A0640010407800F6310200000000000000E0001B
:10A074000B003A00500020008056880056CBBF00E9
:10A084000080FB00E1B420004200DD0081004000BC
:10A0940070002000800878000000EB001007980092
:10A0A400F6FC0200000000000001BE000056800023
:10A0B400115680000000510081805900E00F5000CB
:10A0C400E08F5800C905340056CBBF000080FB0068
:10A0D400E1B420004200DD000080E80001004000FF
:10A0E40010407800562D02000000000056CBBF003F
:10A0F4000080FB00E1B420004200DD00810040004C
:10A10400B0002000800878000000EB0010079800E1
:10A11400B6053700F6FC0200000000000001BE0096
:10A12400209D2400B10620000200400083804800E6
:10A13400005688001156880056CBBF000080FB00F3
:10A14400E1B420004200DD000080E800010040008E
:10A15400104078000002EB008001EB000001EB00EE
:10A1640001C2B300703502000000000040079800EF
:10A174004E009000E50F5000020036005000200011
:10A18400400798004E0090000001E80056CBBF0045
:10A194000080FB00E1B420004200DD000080E80004
:10A1A400010040001040780041AD20003A31020027
:10A1B400000000003200200061C7290040AD2000EB
:10A1C40094070200000000000000E00003003A00D1
:10A1D4000000EB0080568800160037004200200083
:10A1E400A1C7290040AD2000940702000000000030
:10A1F4000000E00003003A001000200080568800B0
:10A204000C003700700020008056880056CBBF0039
:10A214000080FB00E1B420004200DD00810040002A
:10A2240070002000800878000000EB001007980000
:10A234006E05370056CBBF000080FB00E1B4200060
:10A244004200DD000080E80001004000104078007A
:10A254000002EB008001EB000001EB0001C2B3003F
:10A2640070350200000000004007980056CBBF0084
:10A274000080FB00E1B420004200DD000080E80023
:10A2840001004000104078000002EB00CE01900075
:10A294000001EB00F1C3B3007035020000000000C0
:10A2A40030079800CE009000311798003E019000CE
:10A2B40022179800AE1190003E109000808F51003C
:10A2C40002003600BE109000211798002E11900055
:10A2D40042079800CE009000B0062000808F500006
:10A2E4000C003600500020008056880056CBBF007A
:10A2F4000080FB00E1B420004200DD00810040004A
:10A3040070002000800878000000EB00100798001F
:10A314003605370056CBBF000080FB00E1B42000B7
:10A324004200DD000080E800010040001040780099
:10A334004E01900041AD20003A31020000000000BF
:10A34400300798003E009000FC00400080AB2000E5
:10A35400808040000040EB008048780040AD200041
:10A36400F006070040AD2000CA080200000000000B
:10A374003007980050AD200072002000F1C729007A
:10A3840094070200000000000000E00016003A00FC
:10A3940050AD2000AE93020000000000CFEAB700E9
:10A3A400805680000000E00003003A008000200096
:10A3B40080568800020037009000200080568800F4
:10A3C40056CBBF000080FB00E1B420004200DD005A
:10A3D4008100400020002000800878000000EB008D
:10A3E40010079800010537003E0090000000E900C6
:10A3F400FC00400080AB20000080400090407800CA
:10A40400F0C2B30080CF50000400320050AD2000F1
:10A41400267E020000000000CCEAB700CCCABF00D0
:10A42400E14F400020003A003E0090000000E900A7
:10A43400FC00400080AB2000008040009040780089
:10A44400F0C2B30080CF5000090032003E009000FB
:10A45400FC00400080AB200080804000F0C2B300CC
:10A46400804878003E0090000000E8003007980023
:10A47400BE00900040AD20000080400063C8290069
:10A484000A00090033587800B000B1003E00900083
:10A494006A0040003007980050AD2000267E02007C
:10A4A40000000000CCEAB7003E00900041AD20005F
:10A4B4008100E900010F4000060037001E0078000B
:10A4C40090407800E0C2B30080CF50000400320016
:10A4D4001E0FE90040AD20009E0F1000F7FF3A0068
:10A4E4001E0FE8000000EB00905688000E003700B5
:10A4F40090568000800040002059290000804000D0
:10A5040010007800800078001E00780026AB02005E
:10A51400000000000004E0000600320090568000B5
:10A524000000E8009056880090568000EA0F500022
:10A53400EFFF360050AD2000AE9302000000000093
:10A54400CFEAB700CCCABF00E14F40000E00320092
:10A55400CCCABF0062860200000000000000D100E7
:10A56400610060000004E00007003200CCCABF00B4
:10A574006E880200000000000000E800747F020002
:10A5840000000000CDEAB70056CBBF000080FB00FE
:10A59400E1B420004200DD000080E800010040003A
:10A5A400104078000002EB008001EB000001EB009A
:10A5B40001C2B3007035020000000000400798009B
:10A5C4004E0090000000E0003200320010C0B300E2
:10A5D400CEEAB70056CBBF000080FB00E1B42000F8
:10A5E4004200DD000080E8000100400010407800D7
:10A5F400EA004700D0300200000000004E00900046
:10A604000000E90040079800CE00900050072000A9
:10A61400808F50000C0036005000200080568800C7
:10A6240056CBBF000080FB00E1B420004200DD00F7
:10A634008100400070002000800878000000EB00DA
:10A6440010079800690437004856800056CBBF00B5
:10A654000080FB00E1B420004200DD000080E8003F
:10A6640001004000104078004E01900041AD2000F0
:10A674003A31020000000000000044004056880007
:10A684004156800060C2B300804878000100E800B1
:10A694004056880056CBBF000080FB00E1B4200088
:10A6A4004200DD000080E800010040001040780016
:10A6B4000002EB008001EB000001EB00A1C0B3003D
:10A6C4007035020000000000400798004E00900022
:10A6D4000001E80056CBBF000080FB00E1B420007D
:10A6E4004200DD000080E8000100400010407800D6
:10A6F4008000EB003A3102000000000056CBBF009E
:10A704000080FB00E1B420004200DD008100400035
:10A7140020002000800878000000370056CBBF00DE
:10A724000080FB00E1B420004200DD000080E8006E
:10A7340001004000104078000002EB008001EB00B3
:10A744000001EB00A1C0B30070350200000000005E
:10A75400400798004E009000E10F400033003A009B
:10A7640056CBBF000080FB00E1B420004200DD00B6
:10A774000080E8000100400010407800F63102003B
:10A78400000000000000E0000B003A005000200030
:10A794008056880056CBBF000080FB00E1B4200047
:10A7A4004200DD0081004000700020008008780035
:10A7B4000000EB0010079800F6FC02000000000007
:10A7C4000001BE00005680001156800000005100B8
:10A7D40081805900E00F5000E08F580003043400DA
:10A7E40056CBBF000080FB00E1B420004200DD0036
:10A7F4000080E8000100400010407800562D02005F
:10A804000000000056CBBF000080FB00E1B4200034
:10A814004200DD0081004000B00020008008780084
:10A824000000EB0010079800F0033700F6FC02006C
:10A83400000000000001BE00209D2400B10620009D
:10A8440002004000838048000056880011568800AA
:10A854004E009000E10F500015003A0056CBBF00A7
:10A864000080FB00E1B420004200DD000080E8002D
:10A874000100400010407800220020008000EB001E
:10A884003A3102000000000056CBBF000080FB00FC
:10A89400E1B420004200DD008100400030002000CF
:10A8A400800878000000EB0010079800CF03370001
:10A8B40056CBBF000080FB00E1B420004200DD0065
:10A8C4000080E80001004000104078000002EB0026
:10A8D400CE0190000001EB00A1C3B300703502006B
:10A8E400000000000080E800300798000000EB0042
:10A8F400100798003E009000F00F50000D00360045
:10A904004E0090000001E80056CBBF000080FB0021
:10A91400E1B420004200DD000080E80001004000B6
:10A92400104078008000EB003A3102000000000083
:10A934007AFF370056CBBF000080FB00E1B4200053
:10A944004200DD000080E800010040001040780073
:10A95400EB0047003E0190003A3102000000000085
:10A964003E0090000001E900EB0047000040EB00CE
:10A9740000F17800CE0090003E009000008050006E
:10A98400400798000040EB00404798001300370050
:10A994004E4090000080FB008000400000C729006A
:10A9A40000804000900078006B004700C807020058
:10A9B400000000000000E00005003A004E40900056
:10A9C4002404070010002000100798000600370038
:10A9D4004E4090000040E800404798004E409000F0
:10A9E400E24F5000EAFF36001E0090000000E00035
:10A9F4000E00320056CBBF000080FB00E1B4200003
:10AA04004200DD000080E8000100400010407800B2
:10AA14000002EB008001EB000001EB00A1C0B300D9
:10AA24007035020000000000400798004E009000BE
:10AA34000001E80056CBBF000080FB00E1B4200019
:10AA44004200DD000080E800010040001040780072
:10AA54008000EB003A310200000000002FFF3700B5
:10AA6400CFCABF000004E0000C0035003000200015
:10AA74008056880056CBBF000080FB00E1B4200064
:10AA84004200DD0081004000700020008008780052
:10AA94000000EB0010079800540337004156800073
:10AAA4000040EB008048780040AD20001D05070001
:10AAB4004056880080568000E80F50000A003A0093
:10AAC40056CBBF000080FB00E1B420004200DD0053
:10AAD4008100400070002000800878000000EB0036
:10AAE400100798004103370056CBBF000080FB00DD
:10AAF400E1B420004200DD0081004000400020005D
:10AB040080087800CECABF000004E00007003A00C5
:10AB140056CBBF000080FB00E1B420004200DD0002
:10AB24008100400050002000800878000000EB0005
:10AB3400100798000040EB00CEEAB7002B03370063
:10AB44001294020000000000E20F500027033200BC
:10AB540056CBBF000080FB00E1B420004200DD00C2
:10AB640081004000500020008008780056CBBF00D0
:10AB74000080FB00E1B420004200DD000080E8001A
:10AB840001004000104078009230020000000000F4
:10AB94006101B8002056800031568000800F5100BA
:10ABA400818F59001D003A00F6FC020000000000ED
:10ABB4000001BE00005680001156800000005100C4
:10ABC40081805900E00F5000E08F580013003400DA
:10ABD40056CBBF000080FB00E1B420004200DD0042
:10ABE4000080E8000100400010407800562D02006B
:10ABF4000000000056CBBF000080FB00E1B4200041
:10AC04004200DD0081004000B00020008008780090
:10AC14000000EB0010079800F40237008056800013
:10AC2400E10F50000600320080568000E80F50000B
:10AC34006200360080568000EB0F50005F003E003B
:10AC440080568000E80F50001200360080568000C5
:10AC5400EB0F50000F003E003F060700204F980006
:10AC64002E4890000004E0000D003A0056CBBF00CF
:10AC74000080FB00E1B420004200DD0081004000C0
:10AC840070002000800878000000EB001007980096
:10AC9400D60237008094020000000000204F980084
:10ACA4002E489000E24F50000E003A0056CBBF00F1
:10ACB4000080FB00E1B420004200DD000080E800D9
:10ACC40001004000104078009230020000000000B3
:10ACD4000000E90001002000205688003156880059
:10ACE400C20237002E489000E14F500033003A0072
:10ACF40056CBBF000080FB00E1B420004200DD0021
:10AD04000080E8000100400010407800923002000A
:10AD14000000000001002000205688003156880001
:10AD2400F6FC0200000000000001BE00209D24008B
:10AD3400B1062000020040008380480000568800CD
:10AD440011568800C2558000D355800020568000DB
:10AD540031568000800F5100818F59000B0036005E
:10AD640056CBBF000080FB00E1B420004200DD00B0
:10AD74000080E8000100400010407800F631020035
:10AD8400000000000000E00098023A00600020008B
:10AD94008056880056CBBF000080FB00E1B4200041
:10ADA4004200DD008100400070002000800878002F
:10ADB4000000EB00100798008C02370056CBBF0050
:10ADC4000080FB00E1B420004200DD00810040006F
:10ADD4006000200080087800CCCABF00E14F40002A
:10ADE4000C003A00400020008056880056CBBF007B
:10ADF4000080FB00E1B420004200DD00810040003F
:10AE040070002000800878000000EB001007980014
:10AE1400760237006000B800C0558800D15588001C
:10AE2400CDCABF00E14F400005003A000080EB00AE
:10AE34008080EB00E0558800F1558800040037005D
:10AE4400CDCABF00C1AB2000308202000000000068
:10AE540056CBBF000080FB00E1B420004200DD00BF
:10AE640081004000700020008008780056CBBF00AD
:10AE74000080FB00E1B420004200DD000080E80017
:10AE8400010040001040780023C0B3000001EB0033
:10AE940011002000104B02000000000080568000CA
:10AEA40080004000C0C229000080400010007800EB
:10AEB4000001780056CBBF000080FB00E1B4200005
:10AEC4004200DD000080E8000100400010407800EE
:10AED40082007800283002000000000080568000C4
:10AEE400EC0F500029003A0056CBBF000080FB0055
:10AEF400E1B420004200DD000080E80001004000D1
:10AF04001040780041AD200028300200000000000D
:10AF140012C9290056CBBF000080FB00E1B4200019
:10AF24004200DD000080E80001004000104078008D
:10AF340082007800283002000000000056CBBF00D9
:10AF44000080FB00E1B420004200DD000080E80046
:10AF5400010040001040780041AD2000283002007C
:10AF64000000000056CBBF000080FB00E1B42000CD
:10AF74004200DD000080E80001004000104078003D
:10AF8400D1552900283002000000000080568000BE
:10AF94000000E0000B00320080568000E10F5000FA
:10AFA4000800320056CBBF000080FB00E1B4200053
:10AFB4004200DD0081004000B000200080087800DD
:10AFC4000A02370090568000EB0F50002500320033
:10AFD40042CA290056CBBF000080FB00E1B4200028
:10AFE4004200DD000080E8000100400010407800CD
:10AFF4008200780028300200000000009056800093
:10B00400800040002061290000804000100078008A
:10B014000001780056CBBF000080FB00E1B42000A3
:10B024004200DD000080E80001004000104078008C
:10B0340082007800283002000000000056CBBF00D8
:10B044000080FB00E1B420004200DD000080E80045
:10B054000100400010407800D1552900283002003A
:10B0640000000000CCCABF0062860200000000009D
:10B07400610060000004E0000B00320032CB2900C4
:10B0840056CBBF000080FB00E1B420004200DD008D
:10B094000080E80001004000104078008200780041
:10B0A4002830020000000000C2CC290056CBBF00AB
:10B0B4000080FB00E1B420004200DD000080E800D5
:10B0C400010040001040780082007800283002001F
:10B0D4000000000080568000E10F5000070032009D
:10B0E400E2558000F35580000080EB008080EB0087
:10B0F400800F5100818F59000C003200C2CD29000D
:10B1040056CBBF000080FB00E1B420004200DD000C
:10B114000080E800010040001040780082007800C0
:10B1240028300200000000001600370052CE29002B
:10B1340056CBBF000080FB00E1B420004200DD00DC
:10B144000080E80001004000104078008200780090
:10B154002830020000000000E2CE290056CBBF00D8
:10B164000080FB00E1B420004200DD000080E80024
:10B17400010040001040780082007800283002006E
:10B184000000000056CBBF000080FB00E1B42000AB
:10B194004200DD000080E80001004000104078001B
:10B1A400D15529002830020000000000CECABF009B
:10B1B4000004E0000800320056CBBF000080FB0012
:10B1C400E1B420004200DD00810040008000200046
:10B1D400800878001100370056CBBF000080FB00C8
:10B1E400E1B420004200DD000080E80001004000DE
:10B1F40010407800D15529002830020000000000DA
:10B2040056CBBF000080FB00E1B420004200DD000B
:10B214008100400090002000800878000000EB00CE
:10B22400100798007101370040AD20005056880087
:10B23400FA00370022CF290056CBBF000080FB0064
:10B24400E1B420004200DD000080E800010040007D
:10B2540010407800820078002830020000000000CE
:10B2640059003700AE48900000C2B30080CF5000B0
:10B274000B003A0056CBBF000080FB00E1B4200075
:10B284004200DD000080E80001004000104078002A
:10B29400B1C2B300B62E0200000000004A0037001D
:10B2A400AE489000F0C2B30080CF500014003600C6
:10B2B400AE48900090C3B30080CF50000400360025
:10B2C400AE48900000C4B30080CF50000C0036009C
:10B2D400AE489000A0C5B30080CF500004003600F3
:10B2E400AE48900000C6B30080CF50000400360082
:10B2F400AE489000A0C7B30080CF500027003600AE
:10B3040056CBBF000080FB00E1B420004200DD000A
:10B314000080E800010040001040780051C2B300F2
:10B32400B62E0200000000002E489000D8AA0200A9
:10B33400000000000041780056CBBF000080FB00F5
:10B34400E1B420004200DD000080E800010040007C
:10B354001040780082407800B62E02000000000001
:10B364002E48900000AB020000000000004178006D
:10B3740056CBBF000080FB00E1B420004200DD009A
:10B384000080E8000100400010407800824078000E
:10B39400B62E0200000000000B0037002E4990007A
:10B3A40056CBBF000080FB00E1B420004200DD006A
:10B3B4000080E800010040001040780082407800DE
:10B3C400B62E02000000000050568000700F980056
:10B3D400FE08900011407800204F98002E489000FD
:10B3E400006F98000E6990000204E0000200320031
:10B3F40013C0B300036F98008E6890007E0990001C
:10B404000200E800505688000104E00095FF3A006D
:10B4140056CBBF000080FB00E1B420004200DD00F9
:10B424000080E8000100400010407800D1C3B30060
:10B43400B62E02000000000059003700AE4890000C
:10B4440000C2B30080CF50000B003A0056CBBF00BF
:10B454000080FB00E1B420004200DD000080E80031
:10B464000100400010407800B1C2B300B62E0200C3
:10B47400000000004A003700AE489000F0C2B3005C
:10B4840080CF500014003600AE48900090C3B30043
:10B4940080CF500004003600AE48900000C4B300D2
:10B4A40080CF50000C003600AE489000A0C5B30019
:10B4B40080CF500004003600AE48900000C6B300B0
:10B4C40080CF500004003600AE489000A0C7B300FF
:10B4D40080CF50002700360056CBBF000080FB0011
:10B4E400E1B420004200DD000080E80001004000DB
:10B4F4001040780051C2B300B62E020000000000D4
:10B504002E489000D8AA02000000000000417800F4
:10B5140056CBBF000080FB00E1B420004200DD00F8
:10B524000080E8000100400010407800824078006C
:10B53400B62E0200000000002E48900000AB02006E
:10B54400000000000041780056CBBF000080FB00E3
:10B55400E1B420004200DD000080E800010040006A
:10B564001040780082407800B62E020000000000EF
:10B574000B0037002E49900056CBBF000080FB0023
:10B58400E1B420004200DD000080E800010040003A
:10B594001040780082407800B62E020000000000BF
:10B5A40053568000630F9800EE0890001140780015
:10B5B400204F98002E489000106F98001E6990004C
:10B5C4000204E0000200320013C0B300136F9800BD
:10B5D4009E6890006E0990000200E80050568800B2
:10B5E4000104E00095FF3A0056CBBF000080FB0049
:10B5F400E1B420004200DD000080E80001004000CA
:10B6040010407800D15529002830020000000000C5
:10B61400CECABF000040E900CEEAB700CECABF00E0
:10B624000004E00003FF3A0056CBBF000080FB009B
:10B63400E1B420004200DD000080E8000100400089
:10B6440010407800D1552900283002000000000085
:10B6540056CBBF000080FB00E1B420004200DD00B7
:10B664008100400090002000800878000000EB007A
:10B6740010079800630007000000E0000E0032008D
:10B68400CCCABF00F87F02000000000000C0EB003D
:10B69400CCEAB70056CBBF000080FB00E1B4200029
:10B6A4004200DD0081004000B000200080087800E6
:10B6B400100020001007980056CBBF000080FB004C
:10B6C400E1B420004200DD000080E80001004000F9
:10B6D40010407800602E0200000000000000E0002E
:10B6E40042003A0010002000100798003F00370085
:10B6F400100020001007980056CBBF000080FB000C
:10B70400E1B420004200DD000080E80001004000B8
:10B7140010407800602E020000000000EF0F50007F
:10B72400320036000056800011568000C7F807002A
:10B734002056800031568000E00F5000E08F580002
:10B744002A003A000000EB001007980056CBBF0017
:10B754000080FB00E1B420004200DD0081004000D5
:10B76400900020008008780020003700CCCABF0079
:10B77400E14F400005003200CCCABF00F87F020050
:10B784000000000000C0EB00CCEAB700CDCABF0047
:10B79400E14F400005003200CDCABF00F87F02002F
:10B7A4000000000000C0EB00CDEAB70056CBBF009C
:10B7B4000080FB00E1B420004200DD000080E800CE
:10B7C4000100400010407800562D020000000000E7
:10B7D40056CBBF000080FB00E1B420004200DD0036
:10B7E400810040000000EB00800878001E009000FB
:10B7F4000000E000ACF932004F0478000080FA0049
:10B80400000006005200FA0056CBBF000080FB0087
:10B81400E1B420004200DD000080E80001004000A7
:10B8240010407800602E020000000000000F780035
:10B83400E2558000F3558000C0558000D15580004A
:10B8440000015100818159001E0078006102B80096
:10B8540074279800052F98005227980063279800B2
:10B864005E209000EE2090007E2190008E299000B2
:10B87400820F5000838F5800040036007E2290000F
:10B884008E2A90005427980065279800DE229000A5
:10B8940015079800C2558000D35580001E00900003
:10B8A400010020000200400083804800C055880049
:10B8B400D1558800210037001E00900040279800D1
:10B8C40000042000CE209000808F5000020036003B
:10B8D4000204200042279800CCCABF00E5004700BC
:10B8E4004E2190002081020000000000000F78002B
:10B8F4001E00E00003003A001300200033279800E4
:10B904005100370056CBBF000080FB00E1B420009B
:10B914004200DD000080E800010040001040780093
:10B92400E50047001E0178004E2F020000000000D1
:10B934001E0090001E005000100798001E0090008A
:10B944000000E000DCFF3A00C2558000D3558000BF
:10B95400E0558000F1558000800F5100818F59001F
:10B9640037003A0056CBBF000080FB00E1B4200052
:10B974004200DD0081004000A00020008008780023
:10B984006000B8002056880031568800CCCABF0039
:10B994008000EB001A80020000000000CCCABF0047
:10B9A400E40047001A800200000000000000E000EC
:10B9B4000A003200C0558000D1558000610040006B
:10B9C400E0804800C0558800D1558800CE409000E2
:10B9D400E0C7B30080CF5000F0FF3A00C0558000AC
:10B9E400D155800061004000E0804800C0558800C7
:10B9F400D1558800CDCABF0001AC200030820200BE
:10BA040000000000CDCABF00C1AB2000308202009C
:10BA1400000000000000E00009003A000080EB0094
:10BA24008080EB00E0558800F1558800CDCABF0046
:10BA3400F87F02000000000000C0EB00CDEAB70070
:10BA44000002EB00342798003E2090000080FA00AA
:10BA5400000006000200FA00004F78001E04E00017
:10BA640002003A00750007000900370010C0B30057
:10BA74009E4F100002003A00070007000400370040
:10BA840020C0B3009E4F100001003A00F4000700EC
:10BA94000080FA00000006002E00FA00CFCABF00A2
:10BAA4000004E0006300350056CBBF000080FB00BB
:10BAB400E1B420004200DD000080E8000100400005
:10BAC40010407800620020008000EB003A31020050
:10BAD4000000000056CBBF000080FB00E1B4200052
:10BAE4004200DD000080E8000100400010407800C2
:10BAF4008002EB000002EB008001EB00220020003A
:10BB0400D1552900E6320200000000001007980019
:10BB14001E00900063004000100798009E009000F3
:10BB2400C00F200000806000100798001E009000E5
:10BB34006017980040022000EE109000808F5000A3
:10BB4400020036004002200060179800EE109000BA
:10BB540011079800640F47001600370056CBBF004A
:10BB64000080FB00E1B420004200DD000080E8001A
:10BB74000100400010407800420020009E00780040
:10BB84003A31020000000000330020001E0178005A
:10BB9400410020001E007800A6A80200000000005A
:10BBA4001E00900064005000100798001E007800EA
:10BBB400630F40001E0090000000E000E7FF3A0021
:10BBC4001E0078008040EB00014878000000EB0084
:10BBD40010079800640F4700090037001E00780022
:10BBE40090407800A0C3B30080CF5000080032001A
:10BBF4001E0090000000E800100798001E0FE800E7
:10BC04009E00900070022000808F5000F3FF3600E9
:10BC14009E0078000040EB00804878001E0FE8008A
:10BC2400640047009E007800E493020000000000D6
:10BC3400CFEAB7000080FA00000006000A00FA000C
:10BC440056CBBF000080FB00E1B420004200DD00C1
:10BC54000080E80001004000104078008002EB0002
:10BC64000002EB008001EB0022002000D1552900E6
:10BC7400E632020000000000000F780040AD200012
:10BC84006107200080804000405680000080500002
:10BC94009E0F50006E003E00500020008056880029
:10BCA40056CBBF000080FB00E1B420004200DD0061
:10BCB4008100400070002000800878006600370092
:10BCC40056CBBF000080FB00E1B420004200DD0041
:10BCD4000080E80001004000104078000002EB0002
:10BCE4008001EB000001EB00B1C3B300703502002A
:10BCF40000000000100798004056800030079800AC
:10BD04009E009000410798001E00780020079800CC
:10BD1400AE0090004E009000808F5000020036006C
:10BD2400CE009000210798004356800056CBBF00F8
:10BD34000080FB00E1B420004200DD000080E80048
:10BD440001004000104078002E019000830078002C
:10BD54003A31020000000000BE0090000080400064
:10BD6400405688004156800060C2B3008048780085
:10BD74000100E800405688001E0090009E0F50000D
:10BD84002400310056CBBF000080FB00E1B420004A
:10BD94004200DD000080E80001004000104078000F
:10BDA4008000EB00D0300200000000000A003700E1
:10BDB40056CBBF000080FB00E1B420004200DD0050
:10BDC4000080E80001004000104078008000EB0093
:10BDD400D03002000000000056CBBF000080FB0002
:10BDE400E1B420004200DD000080E80001004000D2
:10BDF400104078000002EB008001EB000001EB0032
:10BE040001C2B30070350200000000000000E00031
:10BE1400E7FF320056CBBF000080FB00E1B42000F6
:10BE24004200DD000080E80001004000104078007E
:10BE34008002EB000002EB008001EB0022002000F6
:10BE4400D1552900E632020000000000000F7800FE
:10BE54001E00E0009AFF3A000080FA00000006008D
:10BE64000C00FA0056CBBF000080FB00E1B42000B8
:10BE74004200DD000080E80001004000104078002E
:10BE84008002EB000002EB008001EB0022002000A6
:10BE9400D1552900E632020000000000000F7800AE
:10BEA400900020009E0F10000600360020002000A5
:10BEB400805688006000B800C0558800D1558800BD
:10BEC4001600370056CBBF000080FB00E1B4200011
:10BED4004200DD000080E8000100400010407800CE
:10BEE4008E80E8001E0178003A3102000000000054
:10BEF400000F78009E0078000E80E80080804000EB
:10BF04000040EB00804878000E80E800040902003D
:10BF140000000000C0558800D15588000080FA0058
:10BF2400000006000C00FA00500798005E00900024
:10BF3400CA08020000000000100798005E0090008C
:10BF4400200798002E009000300798004D0037001D
:10BF54003E009000104F78003E0090000000E80082
:10BF6400300798001E0090000000E90010079800B8
:10BF7400D0C3B3009E4F10000300320060C2B30070
:10BF84009E4F100007003A00AE0090000040EB0006
:10BF9400804878002E0090000000E80020079800F8
:10BFA40038003700B0C2B3009E4F100007003A00BB
:10BFB400AE00900000C2B300804878002E009000CC
:10BFC4000000E800200798002E00370050C2B3009C
:10BFD4009E4F100026003A001E009000E10F500012
:10BFE40003003E000000EB00100798002500370016
:10BFF400680047008000E8003E0090001040780090
:10C00400804878003E0090000000E8003007980067
:10C01400E80047003E009000104078008048780017
:10C024003E0090000000E800300798001E009000D9
:10C034000000E900100798001E0090000000E900CD
:10C0440010079800680047001000780062AA0200F8
:10C0540000000000804078002E0090000148780025
:10C064002E0090000000E80020079800050037002B
:10C074002E0090001E4878002E0090000000E8007A
:10C08400200798001E0090000000E000B0FF3A0076
:10C09400AE0090000040EB00804878002E00900035
:10C0A4000000E80020079800AE0090000040EB007C
:10C0B400804878002E0090000080FA0000000600FE
:10C0C4000600FA00000F78001107980017003700E7
:10C0D4009E0078001E009000C807020000000000C7
:10C0E4000000E00007003A001E009000CA080200A9
:10C0F400000000001E0040000000E8002007980037
:10C10400100037001E007800CA080200000000007A
:10C114001E004000000FE8001E007800CA0802005C
:10C12400000000001E004000000FE8001E00780020
:10C13400104078000004E000E5FF3A000000EB0046
:10C14400200798002E0090000080FA0000000600EE
:10C154000600FA0010079800210798002E019000AD
:10C164009E009000D0C3B3003A000700000F78008F
:10C174001E0090000000E000060032001E00900047
:10C18400104078000004E000020032001E0090001D
:10C1940064FF07001E0078000080FA00000006001B
:10C1A4000600FA00889FBE00100798002107980037
:10C1B4002E0190009E00900060C2B300250007008D
:10C1C400000F7800200020009E0F100014003A0099
:10C1D400C8558000D955800056CBBF000080FB00B5
:10C1E400E1B420004200DD000080E80001004000CE
:10C1F400104078009230020000000000010020008E
:10C20400800F5400818F5C0005003A002E019000DD
:10C214009E0090000040EB000E000700000F780025
:10C224001E0090000000E000060032001E00900096
:10C23400104078000004E000020032001E0090006C
:10C2440038FF07001E0078004F04BE000080FA008B
:10C25400000006000C00FA00889FBE0040479800CA
:10C2640031079800420798004E4090000004E00017
:10C274000F00320056CBBF000080FB00E1B4200069
:10C284004200DD000080E80001004000104078001A
:10C294000002EB008001EB000001EB00CE409000B7
:10C2A4007035020000000000000F78000A0037001B
:10C2B40056CBBF000080FB00E1B420004200DD004B
:10C2C4000080E80001004000104078009230020035
:10C2D40000000000000F78000080EB009E0F1000AB
:10C2E40003003A0020002000500798009600370011
:10C2F4004E009000E10F500018003E003E009000F8
:10C304000000E00015003200C8558000D9558000B7
:10C3140056CBBF000080FB00E1B420004200DD00EA
:10C324000080E80001004000104078001E01780001
:10C334008000EB003A310200000000000100200000
:10C344000000540081805C00C0558800D1558800ED
:10C354001000200010079800650037003E00900090
:10C364000000E00015003A00C8558000D95580004F
:10C3740056CBBF000080FB00E1B420004200DD008A
:10C384000080E80001004000104078001E017800A1
:10C394008000EB003A3102000000000001002000A0
:10C3A4000000540081805C00C0558800D15588008D
:10C3B4000000EB00100798004D0037004E0090007D
:10C3C4000080E9009E0F500030003100C855800005
:10C3D400D95580004E0090000081E90056CBBF0083
:10C3E4000080FB00E1B420004200DD000080E80092
:10C3F4000100400010407800BE0090003A31020075
:10C4040000000000010020000000540081805C0056
:10C41400C0558800D1558800C8558000D955800082
:10C424004E0090001E0010000081E80056CBBF00B3
:10C434000080FB00E1B420004200DD000080E80041
:10C4440001004000104078008000EB003A31020007
:10C4540000000000010020000000540081805C0006
:10C46400C0558800D1558800CE0090003E00900051
:10C47400008040008080E9000040EB0080487800A4
:10C48400100020001007980019003700C8558000DC
:10C49400D955800056CBBF000080FB00E1B42000DA
:10C4A4004200DD000080E8000100400010407800F8
:10C4B4001E017800BE0090003A3102000000000026
:10C4C400010020000000540081805C00C0558800F9
:10C4D400D15588009E0078003E0090008080400086
:10C4E4000040EB00804878000000EB001007980043
:10C4F4004E4090000004E00011003200C855800056
:10C50400D955800056CBBF000080FB00E1B4200069
:10C514004200DD000080E800010040001040780087
:10C524008000EB00D0300200000000000100200079
:10C534000000540081805C00C0558800D1558800FB
:10C544001E009000500798005E0090004F04BE004B
:10C554000080FA00000006001A00FA00889FBE005E
:10C5640080568000400F98004E089000EA0F50005B
:10C57400BA0032004E089000EB0F500086003200E3
:10C584004E089000E90F500001003200000137000E
:10C59400F6CF290056CBBF000080FB00E1B4200099
:10C5A4004200DD000080E8000100400010407800F7
:10C5B4008002EB000002EB008001EB00420020004F
:10C5C40086007800E63202000000000010079800A0
:10C5D4001E009000E10F40005100320056CBBF0016
:10C5E4000080FB00E1B420004200DD000080E80090
:10C5F40001004000104078001E0190008000EB0014
:10C604003A3102000000000010079800C255800073
:10C61400D35580001E00900001002000000051004E
:10C6240081805900C0558800D155880056CBBF0081
:10C634000080FB00E1B420004200DD000080E8003F
:10C644000100400010407800923002000000000019
:10C65400E90F500006003E001E0090000000E800B4
:10C664001007980010002000300F9800CA0037000F
:10C6740056CBBF000080FB00E1B420004200DD0087
:10C684000080E8000100400010407800E40047000A
:10C69400A20020003A3102000000000010079800B8
:10C6A400C2558000D35580001E0090000100200078
:10C6B4000000510081805900C0558800D155880080
:10C6C40064004700A200200041D029009407020022
:10C6D400000000000000E0000C003A00A000200070
:10C6E400805688002C84020000000000CCEAB700C9
:10C6F40064004700E4004000CCCABF006200200090
:10C70400C68402000000000002003700B0002000D0
:10C714008056880020002000300F98009E003700CB
:10C7240056CBBF000080FB00E1B420004200DD00D6
:10C734000080E800010040001040780092300200C0
:10C74400000000006401500056CBBF000080FB00D5
:10C75400E1B420004200DD000080E8000100400058
:10C76400104078008000EB003A3102000000000025
:10C7740010079800C2558000D35580001E00900019
:10C78400010020000000510081805900C05588003C
:10C79400D15588007E003700C8558000D9558000E7
:10C7A40056CBBF000080FB00E1B420004200DD0056
:10C7B4000080E80001004000104078009230020040
:10C7C40000000000010020000000540081805C0093
:10C7D400C0558800D155880056CBBF000080FB00AF
:10C7E400E1B420004200DD000080E80001004000C8
:10C7F400104078007430020000000000C255800030
:10C80400D35580003006200001002000800F510025
:10C81400818F590007003600C2558000D35580002F
:10C824000000200001002800800F5100818F590072
:10C834005700360056CBBF000080FB00E1B4200057
:10C844004200DD0081004000700020008008780074
:10C854000000EB00300F98004F00370056CBBF00AC
:10C864000080FB00E1B420004200DD000080E8000D
:10C8740001004000104078009230020000000000E7
:10C88400100798001E0090006101B800C055800098
:10C89400D1558000800F5100818F59002700360048
:10C8A400C0558000D1558000100798002300370040
:10C8B4001E009000200F98002E089000F00F5000EA
:10C8C4000200360000012000200F980056CBBF0064
:10C8D4000080FB00E1B420004200DD000080E8009D
:10C8E4000100400010407800E40047002E09900049
:10C8F4003A31020000000000000F7800C2558000A9
:10C90400D35580001E007800010020000000510073
:10C9140081805900C0558800D15588001E009000C0
:10C924001E00500010079800CCCABF00E400470066
:10C934001E017800C6840200000000001E00900062
:10C944000000E000DAFF3A00C0558000D1558000B5
:10C95400E00F5000E08F58000D003A001000200056
:10C964006A8502000000000056CBBF000080FB0077
:10C97400E1B420004200DD0081004000700020008E
:10C98400800878000000EB00300F980002003700A8
:10C9940010002000300F98003E0890004F04BE00A5
:10C9A4000080FA00000006004A00FA00881F7800A0
:10C9B400302798002056800031568000E00F500048
:10C9C400E08F58000D003A003E209000267E0200C1
:10C9D40000000000004F780000C0EB009E4F1000E4
:10C9E4005200320048AC20001E4078006E880200DD
:10C9F40000000000000C78000F00370040AC20005D
:10CA040010007800747F020000000000004F7800DE
:10CA140080C0EB009ECF10004400320040AC2000E8
:10CA2400100090006101B800210020001E40780031
:10CA3400508202000000000056CBBF000080FB00C3
:10CA4400E1B420004200DD000080E8000100400065
:10CA540010407800602E02000000000020079800BB
:10CA6400270037002E009000402798000004200083
:10CA7400CE209000808F5000020036000004200079
:10CA840040279800E60047004E2190001E407800A1
:10CA94002081020000000000100798001E00900092
:10CAA4000000E00007003A001E407800F87F020012
:10CAB400000000006000B80020568800315688004D
:10CAC4001A00370056CBBF000080FB00E1B4200001
:10CAD4004200DD000080E8000100400010407800C2
:10CAE400E60047001E0190004E2F020000000000E7
:10CAF400AE0090001E0090000080500020079800B7
:10CB04002E0090000000E000D6FF3A0048AC200060
:10CB14001E4078004E8802000000000010049800B7
:10CB24001E407800F87F0200000000004F047800E7
:10CB34000080FA00000006000400FA00CD22A800DC
:10CB4400C922A9000000EB0000128800F0002000B8
:10CB5400101288000000EB00201288004302A80095
:10CB640042A2A80041E2A80000003700E104070047
:10CB74000E80E800D1C1B300F90407002E409000F4
:10CB8400004F78001E80FB004300DE00610060005F
:10CB94000004E000F5FF3A001E80FB000080EA007C
:10CBA400610060000004E000F0FF3A001000200083
:10CBB400308488000000EB00108488008040EB0083
:10CBC40080C0B300670507008040EB0090C0B3004D
:10CBD4006405070011CAB300C0C0B30061050700B3
:10CBE40091C0B300D0C0B3005E05070011CAB30002
:10CBF400A0C0B3005B05070091C0B300B0C0B30090
:10CC04005805070021CAB30040C0B300550507000A
:10CC140091C0B30050C0B3005205070021CAB3004D
:10CC240020C0B3004F05070091C0B30030C0B3006B
:10CC34004C0507000040EB002604070000202000FC
:10CC4400D6050700D1C0B3000040EB00450507003E
:10CC540021C3B30020C0B3004205070021C1B300C3
:10CC640040C0B3003F05070001C4B30030C0B300A7
:10CC74003C050700F1C3B30090C0B30039050700B9
:10CC840021C1B30060C0B30036050700C1C0B300C2
:10CC940070C0B30033050700E1CEB300A0C0B300F9
:10CCA4003005070051C0B300B0C0B3002D05070024
:10CCB40040302000B905070071B820009140780089
:10CCC40040C0B3002705070081B8200091407800D8
:10CCD40050C0B3002305070091B8200091407800AC
:10CCE40020C0B3001F050700A1B8200091407800C0
:10CCF40030C0B3001B050700B1B820009140780094
:10CD04000040EB0017050700C1B8200091407800EF
:10CD140010C0B300130507008040EB0050C1B300FE
:10CD2400100507006300470021C1B3008C0407000D
:10CD34003E40900088F0B7000110200000C1B3000D
:10CD4400790507002147230040C1B3007605070099
:10CD54008000EB000040EB00730507000000EB00CF
:10CD64008E05070041C0B300F0C1B30049050700B8
:10CD74000080FA00000006000200FA0011C0B300AF
:10CD84000E007800CD0407001E0078004200DE008B
:10CD9400614060000080FB000080FA000000060093
:10CDA4000200FA00F1C1B3000E0078006C04070021
:10CDB4001E4078000080FB004300DE000004A20057
:10CDC4000080FB00610060000080FA0000000600A3
:10CDD4000200FA00308480000000E00014003A00F1
:10CDE4001000200030848800108480000000E900D6
:10CDF400000F78009E007800109A2000808F500069
:10CE040002003600109A2000000F780001C4B3001D
:10CE1400E0C1B3001F0507009E407800C0C0B30006
:10CE2400D00407009E409000D0C0B300CD0407009A
:10CE34000080FA00000006000C00FA0090112000A7
:10CE4400560507006400470091C1B300440407007D
:10CE54004E409000004F7800E00020004F0507008E
:10CE640065004700E1C0B3003D0407005E40900048
:10CE74002047980066004700F1C0B300380407005B
:10CE84006E40900030479800901120004305070041
:10CE94006700470091C1B300310407007E40900051
:10CEA400804078001E40780080CF5000E5FF3A00B3
:10CEB400C00020003905070068004700C1C0B30066
:10CEC400270407000E489000004F780069004700CF
:10CED400D1C0B300220407001E48900010479800F8
:10CEE4009E0090001E007800808F500007003600DE
:10CEF4009E0090001E00780080805000109A200050
:10CF040001005000500798000C0037009E0090006C
:10CF14001E007800808F500003003A00109A200011
:10CF240050079800050037001E0078009E0090000E
:10CF3400010050000000E900500798005E009000D6
:10CF44000080FA00000006001E00FA00300F98006E
:10CF5400410F980090112000100507007A00470047
:10CF640091C1B300FE0307002E589000004F7800D3
:10CF74000000EB00090507001E04E00003003A006E
:10CF84000000EB00600F98005D00370030848000E3
:10CF94000000E00004003A008DFF07000000EB00F1
:10CFA400600F9800560037001084800020848800A9
:10CFB40041082100914078000040EB00690407001B
:10CFC400510821009140780010C0B30065040700A7
:10CFD4000E80E80041012000D10207000E80E80025
:10CFE40010089000BEAB0200000000008000780032
:10CFF4000E80E800110898000E80E8009000780088
:10D00400109A2000808F50001B003E000E80E80024
:10D0140010407800614060000004E00016003A000F
:10D024000E80E800A000900000002800008060004E
:10D034000000E00010003A000E80E800200090009C
:10D04400700060000000E0000B003A000E80E80071
:10D0540090009000E05E2000808F500006003E00AB
:10D064000E80E800A000900000082000008060000E
:10D074000000E00001003A000000FE000E80E8001D
:10D084001000780010848800BE0890000E80E8002C
:10D094006C00400005000900B05878006100B10040
:10D0A4006000B100CE08900000C0EB00804878001A
:10D0B4000E80E80030509000E84F50000C003A0019
:10D0C4000E80E800205090000004E00004003200CC
:10D0D4000E80E80020509000E64F500004003A0013
:10D0E4000E80E800A05090004E089000014878009F
:10D0F4000000EB003084880010002000600F9800CE
:10D104006E0890000080FA00000006000800FA0093
:10D11400000F7800214798002207980031CAB30015
:10D1240020C0B3000F04070091C0B30030C0B300A7
:10D134000C040700AE009000009B2000008040001B
:10D1440020079800640047009040780060C0B30056
:10D1540004040700640047009040900070C0B300CE
:10D16400000407001E00780061002000F50207009B
:10D1740070B8200061002000F202070080C0B300F4
:10D18400D40207002E4090000004E00003003A009F
:10D194000040EB00604798000200370060C0B30015
:10D1A400604798006E409000CA0207000080FA00B1
:10D1B400000006001800FA0001C8B300F0C1B30073
:10D1C4003404070001C8B300F0C1B3000C04070025
:10D1D400A1C0B300C0C1B3000904070081C0B300FB
:10D1E400F0C1B3002B04070088D0BF00E54F500006
:10D1F4000300320088D0BF00E64F500079003A00A7
:10D204000000EB001007980070004700C1C1B30094
:10D21400530307000E5090000080FB006A0060007A
:10D224000000E00007003A001E0090000000E80043
:10D23400100798009E009000703E2000808F5000E0
:10D24400F1FF360071004700C1C1B3004403070079
:10D254001E509000624060000004E00004003A00A8
:10D264009E009000703E2000808F50005D003600CC
:10D2740081C0B300F0C1B300E103070072004700AE
:10D284008040EB00360307002E5090004047980082
:10D294007300470011C0B300310307003E509000F3
:10D2A400504798007400470061C0B3002C03070086
:10D2B4004E509000604798007500470071C0B3005D
:10D2C400270307005E509000704798003E009000CE
:10D2D4000000E80030079800EE4090000040EB00AA
:10D2E400A0030700FE40900010C0B3009D03070098
:10D2F4006800470081002000090207000040EB009D
:10D30400004F78002E00370076004700C1C1B300FB
:10D31400130307006E509000624060000004E000B8
:10D324002A003200680047009000900000002200AC
:10D33400008060000000E0002400320001C8B30057
:10D34400F0C1B300D303070001C8B300F0C1B300B8
:10D35400AB030700A1C0B300C0C1B300A80307001A
:10D3640081C0B300F0C1B300CA03070077004700CF
:10D37400C1C1B300FA0207007E5090000080FB0098
:10D384006A0060000000E000F8FF320081C0B300D2
:10D39400F0C1B3009A030700EE4090000040EB0098
:10D3A40070030700FE40900010C0B3006D03070037
:10D3B4006800470081002000D90107001E4FE800E3
:10D3C400F0C0B3009E4F1000CFFF3600CE40900057
:10D3D4000040EB0063030700DE40900010C0B30080
:10D3E400600307000080FA00000006000400FA0051
:10D3F40010079800218480001E00900000804000E7
:10D4040074004000000F78009E007800109A2000FD
:10D41400808F5000040036001E007800E1652F0064
:10D4240001004000000F78009E4078000040EB00AF
:10D434004C0307009E40900010C0B300490307004E
:10D444000080FA00000006000600FA0010079800A9
:10D454006400470021C0B300C10207004E409000A1
:10D46400004F78006500470031C0B300BC020700DC
:10D474005E409000104798000E80E80090407800CD
:10D4840020C0B300370307000E80E80090409000EE
:10D4940030C0B300330307001E0078000080FA0098
:10D4A400000006000600FA00100798006400470018
:10D4B4008040EB00AA0207004E409000004F780025
:10D4C4006500470011C0B300A50207005E4090004C
:10D4D400104798000E80E800904078000040EB0070
:10D4E400200307000E80E8009040900010C0B300B5
:10D4F4001C0307001E0078000080FA0000000600EC
:10D504000A00FA002007980031079800218480005F
:10D514002E0090000080400074004000000F78004E
:10D524009E007800109A2000808F5000040036007E
:10D534001E007800E1652F0001004000000F780014
:10D54400680047008040EB00850207000E48900009
:10D55400204798006900470011C0B300800207000B
:10D564001E489000304798009E4078000040EB0031
:10D57400FC0207009E40900010C0B300F9020700AF
:10D584003E0090000A000700000F7800AE409000B3
:10D594000040EB00F3020700BE40900010C0B3004F
:10D5A400F00207001E0078000080FA000000060068
:10D5B4002400FA00700F98006000B800200798005B
:10D5C40031079800000220000E0040008040EB006C
:10D5D400630207000E6090002047980010022000AC
:10D5E4000E00400011C0B3005D0207001E609000F1
:10D5F400304798002F0037007E08900010179800DD
:10D604001E109000F40F500002003600400120006C
:10D61400101798001E10900040079800CE0090004C
:10D624006A0047003E010700CE0090007E0890008B
:10D6340001005000700F9800680047001000780047
:10D64400610060000000E00008003200EA004700CA
:10D654004E009000808040000040EB00804878003D
:10D664004E0090000000E800400798006A0F470051
:10D674000D0037002E019000BE0190001E007800BE
:10D684001000780001002000020040008380480060
:10D6940020079800310798001E8FE8004E00900084
:10D6A4000080E900400798004E0090000000E00070
:10D6B400F0FF3A007E0890000000E000CEFF3A0040
:10D6C400AE4090000040EB00A6020700BE40900070
:10D6D40010C0B300A30207002E0090006101B8003F
:10D6E4003E009000010020000200400083804800BA
:10D6F4002007980031079800AE0090003E0090008B
:10D7040000804000200798002E0090000080EA006E
:10D714000080FA00000006001800FA00881F780054
:10D724004007980051079800620798000000EB003A
:10D73400200798000000EB00300798000000EB0081
:10D74400100798000000EB00000F78004E009000D6
:10D75400E10F40000F003A0010002000100798006D
:10D764006E00470021C0B300FD0107006E48900021
:10D774000080FB0040079800680047000004E800B0
:10D784006F00470031C0B300F50107007E489000E8
:10D79400004C78005E009000E10F40000F003A005A
:10D7A40010002000000F7800700047008040EB005C
:10D7B400EB0107000E5090000080FB00500798001A
:10D7C4006A0047000004E8007100470011C0B3007C
:10D7D400E30107001E509000004C78006E0090009A
:10D7E400E10F500046003E001E00E0000A003A002F
:10D7F400720047008040EB00D90107002E509000D2
:10D80400404798007300470011C0B300D4010700DB
:10D814003E509000504798001E0090000000E00029
:10D824000A003A007400470021C0B300CC0107008D
:10D834004E509000604798007500470031C0B30017
:10D84400C70107005E509000704798006A004700C7
:10D85400904078000040EB00420207006A00470055
:10D864000000E8009040780010C0B3003D020700BB
:10D87400680047009040780020C0B30039020700D8
:10D88400680047000000E8009040780030C0B30012
:10D894003402070002003700880007000D0107006A
:10D8A4006E0090000000E900600798006E00900090
:10D8B400E10F4000F8FF3A001E00E00006003A00C5
:10D8C400CE4090000040EB0026020700DE409000AE
:10D8D40010C0B300230207001E0090000000E00007
:10D8E40067003A00EE40900020C0B3001D0207001C
:10D8F400FE40900030C0B3001A02070060003700F9
:10D904001E0090000000E0000A003200CE009000EB
:10D914006E0090000080400030079800EE409000B8
:10D9240020C0B3000F020700FE40900030C0B300D7
:10D934000C020700DE0090006E00900000804000A2
:10D944000000E9006007980076004700F1C1B300C9
:10D95400830107006E5090000042B2000004E00012
:10D96400F9FF3A006A0047009040780000C1B30014
:10D97400FC0107006A0047000000E80090407800BE
:10D9840010C1B300F7010700680047009040780019
:10D9940040C1B300F3010700680047000000E8003D
:10D9A4009040780050C1B300EE010700DE00900003
:10D9B400109A2000808F500008003E00EE00900076
:10D9C400109A2000808F5000040036006E009000F2
:10D9D400E1652F0001004000600798006C004700DB
:10D9E4009040780020C1B300DE0107006C004700BE
:10D9F4000000E8009040780030C1B300D90107006E
:10DA040001C1B300F0C1B300FD01070001C2B300BE
:10DA1400F0C1B3001F0207001E00E000180032002E
:10DA24006E0090000000E80060079800DE0090009F
:10DA3400109A2000808F500008003E00EE009000F5
:10DA4400109A2000808F5000040036006E00900071
:10DA5400E1652F0001004000600798006C0047005A
:10DA6400904078000040EB00BE0107006C004700C6
:10DA74000000E8009040780010C0B300B90107002E
:10DA84004F0478000080FA00000006000200FA004B
:10DA9400F1C1B3000E007800310107001E40780088
:10DAA4000080FB004500DE000004A2000080FB00B3
:10DAB400610060000080FA00000006000200FA0025
:10DAC400CD22A90041E2A9004342A80041E2A800F6
:10DAD40000A02300401288000000370040C2BF00AD
:10DAE400624060000004E000FCFF3A0040C2BF0056
:10DAF400614060000004E000F8FF320041E2A90048
:10DB04004342A90041E2A80040128000004F78007F
:10DB1400CD22A8001E80FB000080FA000000060051
:10DB24000A00FA003007980041079800CD22A900A6
:10DB3400A0032000401288000000EB00000F7800D2
:10DB44003E0090000000E000040032003E0090001F
:10DB54000000E900300798000000370040C2BF0011
:10DB6400624060000004E000FCFF3A0040C2BF00D5
:10DB7400614060000004E000F8FF320040128000C1
:10DB8400204798004E009000E10F50004A003600F4
:10DB940041E2A9004342A80041E2A8000000EB00D2
:10DBA400401288001E8FE8000000370040C2BF000A
:10DBB400624060000004E000FCFF3A0040C2BF0085
:10DBC400614060000004E000F8FF32004012800071
:10DBD400200798003E0090000000E0000C00320096
:10DBE4003E0090000000E80030079800DE409000FE
:10DBF4003E009000014878003E0090000000E800DC
:10DC040030079800CE4090003E0090000148780014
:10DC14004E0090001E005000E10F5000010036003D
:10DC2400DEFF370041E2A9004342A90041E2A80017
:10DC3400210037000000EB00401288001E0FE800AE
:10DC44003E0090000000E000110032003E00900011
:10DC54000000E800300798000000370040C2BF0011
:10DC6400624060000004E000FCFF3A0040C2BF00D4
:10DC7400614060000004E000F8FF320040128000C0
:10DC8400804078003E009000014878000A00370088
:10DC940040C2BF00624060000004E000FCFF3A00A4
:10DCA40040C2BF00614060000004E000F8FF3200A1
:10DCB40040128000204798004E0090009E0F1000F4
:10DCC400DCFF3900CD22A8001E0078000080FA0095
:10DCD400000006000400FA0020479800CD22A900A5
:10DCE40041E2A9004342A80041E2A8002E4090006E
:10DCF4008080FB0000A02700008070004012880094
:10DD04000000370040C2BF00624060000004E00031
:10DD1400FCFF3A0040C2BF00614060000004E00024
:10DD2400F8FF320041E2A9004342A90041E2A80001
:10DD340040128000004F7800CD22A8000080FA0035
:10DD4400000006000800FA00200798003107980038
:10DD5400CD22A900A007200040128800000037004F
:10DD640040C2BF00624060000004E000FCFF3A00D3
:10DD740040C2BF00614060000004E000F8FF3200D0
:10DD840040128000004F78003E009000E10F5000E8
:10DD9400520036002E009000104078003047980062
:10DDA4002E0090000000E800200798002E0090004C
:10DDB40010407800204798002E0090000000E800F2
:10DDC4002007980041E2A9004342A80041E2A800CC
:10DDD4001E009000401288003E0090000080E90080
:10DDE400300798003E009000E10F50001800360004
:10DDF4002E00900010407800304798002E009000CC
:10DE04000000E800200798002E00900010407800E1
:10DE1400204798002E0090000000E800200798009A
:10DE24000000370040C2BF00624060000004E00010
:10DE3400FCFF3A0040C2BF00614060000004E00003
:10DE4400F8FF320040128000004F7800E0FF3700F6
:10DE540040C2BF00624060000004E000FCFF3A00E2
:10DE640040C2BF00614060000004E000F8FF3200DF
:10DE740040128000004F780041E2A9004342A9000B
:10DE840041E2A800150037002E00900010407800F1
:10DE94000080FB00401288002E0090000000E80083
:10DEA400200798003E0090000000E9003007980029
:10DEB4000000370040C2BF00624060000004E00080
:10DEC400FCFF3A0040C2BF00614060000004E00073
:10DED400F8FF320040128000004F78003E009000AE
:10DEE4000000E000E8FF3A00CD22A8000080FA001C
:10DEF400000006000200FA0001C2B300E0C1B30052
:10DF0400BF00070010002000F2040200010000001E
:10DF1400CD22A900F00F2000401288000000370035
:10DF240040C2BF00624060000004E000FCFF3A0011
:10DF340040C2BF00614060000004E000F8FF32000E
:10DF440040128000004F7800CD22A800100020006D
:10DF5400F2040200010000000080FA000000060044
:10DF64000600FA002007980021479800CD22A90056
:10DF74002E4090000080FB00401288000000370013
:10DF840040C2BF00624060000004E000FCFF3A00B1
:10DF940040C2BF00614060000004E000F8FF3200AE
:10DFA40040128000004F78000000EB00401288000F
:10DFB4000000370040C2BF00624060000004E0007F
:10DFC400FCFF3A0040C2BF00614060000004E00072
:10DFD400F8FF320040128000004F7800CD22A800E4
:10DFE4002E0090001E4878002E0090000080FA0059
:10DFF400000006000600FA00200798002147980058
:10E00400CD22A9002E4090000080FB004012880021
:10E014000000370040C2BF00624060000004E0001E
:10E02400FCFF3A0040C2BF00614060000004E00011
:10E03400F8FF320040128000004F78000000EB002F
:10E04400401288000000370040C2BF0062406000F8
:10E054000004E000FCFF3A0040C2BF0061406000E1
:10E064000004E000F8FF320040128000004F780006
:10E074000000EB00401288000000370040C2BF00DF
:10E08400624060000004E000FCFF3A0040C2BF00B0
:10E09400614060000004E000F8FF3200401280009C
:10E0A400004F7800CD22A8002E0090001E48780072
:10E0B4002E0090000080FA00000006000800FA001C
:10E0C400300798002147980040212000B300070042
:10E0D400AE40900040C1B3002200070011C0B3005D
:10E0E40020C1B3001F000700A0302000AB000700D0
:10E0F40063004700A1C0B300BEFF07003E4090008C
:10E10400614060000004E000F9FF3A004021200073
:10E11400A20007008040EB0020C1B30011000700FB
:10E124006400470081C1B300B2FF07004E40900075
:10E13400004F78006500470091C1B300ADFF0700B0
:10E144005E409000104798000000EB009300070029
:10E154003E0090001E0878003E0090000080FA0007
:10E16400000006000400FA00204798003147980098
:10E17400CD22A900AE40900000C4B30000C07000DE
:10E184000080FB00401288000000370040C2BF003E
:10E19400624060000004E000FCFF3A0040C2BF009F
:10E1A400614060000004E000F8FF3200401280008B
:10E1B400004F78003E4090000080FB004012880031
:10E1C4000000370040C2BF00624060000004E0006D
:10E1D400FCFF3A0040C2BF00614060000004E00060
:10E1E400F8FF320040128000004F78000000000069
:10E1F40000000000CD22A8000080FA000000060004
:10E204000400FA002047980031479800CD22A90065
:10E21400AE40900000CAB30000C070000080FB0054
:10E22400401288000000370040C2BF006240600016
:10E234000004E000FCFF3A0040C2BF0061406000FF
:10E244000004E000F8FF320040128000004F780024
:10E254003E4090000080FB00401288000000370020
:10E2640040C2BF00624060000004E000FCFF3A00CE
:10E2740040C2BF00614060000004E000F8FF3200CB
:10E2840040128000004F7800CD22A8000080FA00E0
:10E29400000006000400FA00204798003147980067
:10E2A400CD22A900AE40900000C8B30000C07000A9
:10E2B4000080FB00401288000000370040C2BF000D
:10E2C400624060000004E000FCFF3A0040C2BF006E
:10E2D400614060000004E000F8FF3200401280005A
:10E2E400004F78003E4090000080FB004012880000
:10E2F4000000370040C2BF00624060000004E0003C
:10E30400FCFF3A0040C2BF00614060000004E0002E
:10E31400F8FF320040128000004F7800CD22A800A0
:10E324000080FA00000006000600FA00004F7800A2
:10E334001107980040212000180007009E40780033
:10E3440040C1B30087FF07000E80E80090407800CA
:10E3540060C1B30083FF07000E80E8009040900086
:10E3640070C1B3007FFF0700A03020000B0007003E
:10E3740064004700A1C0B3001EFF07004E40900098
:10E38400614060000004E000F9FF3A000000EB0087
:10E39400020007000080FA00000006000200FA00F4
:10E3A400000F780031C0B300F0C1B30094FF070040
:10E3B4000E00780090409000F0C1B300B5FF070054
:10E3C4000080FA00000006000200FA0041C0B30019
:10E3D400F0C1B3008AFF0700D1C1B3000E0078007A
:10E3E400DFFE07001E407800644060000004E00087
:10E3F400F9FF3A000E00E800F1C1B300D8FE0700AF
:10E404001E409000684060000004E000F9FF3A00FC
:10E4140001C2B300E0C1B3009EFF07000080FA0010
:10E42400000006000200FA0001C2B300E0C1B3001C
:10E4340073FF0700D1C1B3000E007800C8FE0700C7
:10E444001E407800614060000004E000F9FF3200E3
:10E4540041C0B300F0C1B3008EFF07000080FA0092
:10E46400000006000200FA00004F7800503120003E
:10E47400CAFF07009E40780050C1B30039FF07006F
:10E484000000EB00C5FF07000080FA000000060052
:10E494000400FA0050312000C0FF07000E80E8009D
:10E4A40051C1B300AEFE07002E409000004F78002B
:10E4B4000000EB00B9FF07001E80FB000080FA009B
:10E4C400000006000400FA000000EB0010079800AA
:10E4D4000E0037001E0090007200B9008000780022
:10E4E400C0F52000008F40009E0078000000EB0083
:10E4F400900098009E00780000C0EB0080509800C7
:10E504001E0090000000E800100798001E00900014
:10E51400E20F5000EFFF36000080FA000000060012
:10E524000E00FA002007980031079800420798006F
:10E53400C0F52000100798002E009000E20F500054
:10E5440003003200E00F200050079800430037001A
:10E554004E0090000000E00010003A00BE00900061
:10E564006107980040062000EE009000808F500064
:10E5740008003200E0062000EE009000808F50007A
:10E584000100320005003700100120004007980008
:10E594000200370060002000400798000040EB00B4
:10E5A400004F7800280037001E00900010009000F3
:10E5B4000000E00020003A001E009000BE00900021
:10E5C40001087800BE009000E0062000808F500013
:10E5D40009003A004E009000F10F500006003A0086
:10E5E4009E00900010002000900098001E80FB0008
:10E5F4005007980019003700BE0090004006200024
:10E60400808F500009003A004E009000E60F500041
:10E6140006003A009E009000100020009000980030
:10E624009E80FB00510798000C003700E00F20008B
:10E6340050079800090037001E4FE8001E009000A4
:10E64400720040001007980021C0B3009ECF100054
:10E65400D5FF3600E00F2000500798005E009000C0
:10E664000080FA00000006000E00FA0060479800DF
:10E6740041079800520798006E409000E24F500006
:10E68400030036000080EB00600798004700370065
:10E694006E4090000080FB007200B900800078009A
:10E6A400C0F5200000804000200798002E00900054
:10E6B40010009000E10F5000030032008080EB0056
:10E6C40061079800390037005E009000EF0F50009A
:10E6D40003003E000080EB00600798003300370021
:10E6E400CE009000110798009E00900021409000F9
:10E6F4000081FB00314090000080FB004800DD00F9
:10E7040002007000000F78001E00E0000A003A00CA
:10E71400F0858000000F78000000E800F085880094
:10E72400F185800080382100808F5000020036007F
:10E7340000402000F08588002E00900090007800B2
:10E74400E0062000808F500010003A000002EB0029
:10E754009E0178000041EB006000B8007EB5020025
:10E7640000000000804078002E00900001509800C6
:10E774002E00900000509000E14F400003003A004A
:10E784000080EB0060079800080037002E0090001E
:10E794009E00780021009800AE0090002000200028
:10E7A400900098000000EB00600798006E00900055
:10E7B4000080FA00000006000E00FA00004F9800E6
:10E7C400510798000E489000E24F500003003600B5
:10E7D4000080EB0060079800800037000E4890002E
:10E7E4000080FB007200B90080007800C0F52000B2
:10E7F40000804000300798003E00900090007800B0
:10E8040040062000808F5000030032008080EB001F
:10E8140061079800710037003E00900010009000DE
:10E82400E30F500003003A003E009000E000900027
:10E83400510798003E00900010009000E20F500035
:10E844005E0032003E00900010009000E30F500084
:10E854005A0032000080EB00600798005F00370028
:10E864000040EB00004F78000000EB001007980018
:10E874004A0037001E0090007200B9008080E80052
:10E88400C0F5200000804000100078000000E00087
:10E894003F003A003E00900020009000A4C0B30066
:10E8A400800178000041EB006000B800B42B020046
:10E8B40000000000404798004E409000E24F4000A6
:10E8C40003003A008080EB006107980043003700A2
:10E8D4004E409000FE2C02000000000010C0B30067
:10E8E400004F7800BE009000300020009000980097
:10E8F4003E009000DE009000610098001E00900031
:10E904007200B900F0004000C0F520000080400013
:10E91400CE409000014878001E0090007200B900BB
:10E924008080E800C0F52000808040004000200086
:10E93400800878001E0090007200B900EE004000CC
:10E94400C0F520008080400010002000800878007E
:10E954009E0090003E009000200190007208B900D3
:10E96400E4004000C0F52000008040000208780068
:10E974001E0090007200B90080007800C0F52000ED
:10E9840080804000400620008008780006003700A0
:10E994001E0090000000E800100798001E00900080
:10E9A400E20F5000B3FF36001E04E00003003A00FB
:10E9B4000080EB0060079800080037005E009000BC
:10E9C4000000E900500798005E009000E10F40004D
:10E9D400A3FF3A008000EB00610798006E009000EE
:10E9E4000080FA00000006001200FA00204F980090
:10E9F40061079800720798002E489000E24F50007B
:10EA040003003600E00F2000000F98009900370043
:10EA14002E4890000080FB007200B900800078004E
:10EA2400C0F5200000804000400798004E00900090
:10EA340010009000E30F500003003200E00F2000AC
:10EA4400000F98008B0037004E0090009000780073
:10EA540040062000808F500003003200E00F2000A9
:10EA6400000F9800830037000000EB0010079800A7
:10EA74007B0037001E0090007200B9008080E8001F
:10EA8400C0F520000080400010007800E40F500022
:10EA940070003A001E0090007200B900E4004000CB
:10EAA400C0F5200000804000900078004E009000E7
:10EAB40020009000808F500066003A001E009000F5
:10EAC4007200B900F0004000C0F520000080400052
:10EAD400104F78001E407800FE2C02000000000059
:10EAE4001E4078002E2D0200000000000000E0000F
:10EAF400580032001E407800122E02000000000070
:10EB0400300798006E0090000000E00036003200EC
:10EB14007E0090000000E000330032007E00900090
:10EB240010007800EF0F500003003E00E00F2000BB
:10EB3400000F98004F0037006E00900020079800E7
:10EB44003E0090001001BE00AE009000F00F2000C7
:10EB54000002610041409000604060000440700089
:10EB6400C04098004812DE005140900060406000B0
:10EB740004407000D0409800F00F20000082610033
:10EB8400614090006040600004407000E0409800E4
:10EB94004819DE007140900060406000024070003F
:10EBA400F04098003E009000D0019000AE0090002C
:10EBB400F00F20000081610021409000604060005F
:10EBC40002407000A04098004819DE0031409000D7
:10EBD4006040600002407000B0409800FE00900069
:10EBE40000012000800878009E0090003E00900004
:10EBF400500190007208B900E6004000C0F5200002
:10EC040000804000020878009E0090003E009000C2
:10EC14001001BE007208B900E8004000C0F52000F1
:10EC2400008040000288BE001E0090007200B900FF
:10EC34008080E800C0F52000808040006000200053
:10EC4400800878001E0090000080FB00000F9800F0
:10EC5400080037001E0090000000E800100798002C
:10EC64001E009000E20F500082FF3600E00F2000EB
:10EC7400000F98000E0890000080FA0000000600C3
:10EC84001600FA00404F980071079800020F980090
:10EC94004E489000E24F5000030036000080EB0025
:10ECA400200F9800BD0037004E4890000080FB0004
:10ECB4007200B90080007800C0F520000080400098
:10ECC400500798005E009000100090000000E000E3
:10ECD40003003A008080EB00210F9800AF0037005A
:10ECE4000E089000EF0F500003003E000081EB007F
:10ECF400220F9800A9003700FE01900043079800F6
:10ED0400CE009000214090000081FB003140900033
:10ED14000080FB004800DD0002007000100798002E
:10ED2400CE009000414090000082FB0051409000D2
:10ED34000080FB004800DD00040070000001780042
:10ED4400614090000082FB00714090000080FB0055
:10ED54004800DD000400700080017800220798005C
:10ED6400330798002E009000BE009000E00F500082
:10ED7400E08F5800030032001E0090000000E00005
:10ED840003003A000080EB00200F98008300370056
:10ED94005E0090009000780040062000808F5000B4
:10EDA4004C003A005E00900010009000100F980094
:10EDB4009E089000E58F50000F0032001E0990005D
:10EDC400E50F510005003E009E0990000300E90094
:10EDD400E10F50003C003E001D0037001E0890006B
:10EDE400E60F500001003200370037008000EB00CE
:10EDF400210F9800690037004E4890002503070052
:10EE04000000E000030032000081EB00220F9800B4
:10EE1400620037005E009000005090002E2D02002A
:10EE2400000000000000E00003003A00E3FF2F00B0
:10EE3400230F980059003700DE0090006000200086
:10EE4400900098000000EB00200F9800530037005A
:10EE5400B4C0B3009E01900032C0B3002E009000F5
:10EE6400BE009000B42B0200000000008040780037
:10EE74005E009000015098005E00900000509000E9
:10EE8400E24F400003003A008080EB00210F98001D
:10EE9400420037005E00900000509000FE2C0200FB
:10EEA40000000000DE0090000000EB00F00098007D
:10EEB400DE0090005000200090009800E2FF2F0038
:10EEC400220F9800350037008081EB00230F980053
:10EED400320037005E00900010009000E10F5000F7
:10EEE4001D003A00F0858000000F78000000E80063
:10EEF400F0858800F185800080382100808F5000E3
:10EF04000200360000402000F08588001E029000B8
:10EF14009E0178000041EB006000B8007EB502005D
:10EF240000000000804078005E00900001509800CE
:10EF34005E00900000509000E14F400003003A0052
:10EF44000080EB00200F980014003700DE009000D2
:10EF540020002000900098005E00900010009000B7
:10EF6400E20F5000030032008080EB00210F980074
:10EF74000A0037005E0090001E01900032009800E5
:10EF84005E0090002E019000BE01900042009800A7
:10EF9400530098008001EB00230F98002E08900086
:10EFA4000080FA00000006000800FA00004F780014
:10EFB4001107980022079800330798008002EB009D
:10EFC4000002EB00BE0190002E0190009E00900014
:10EFD4001E407800020007000080FA0000000600CE
:10EFE4002E00FA0000679800111798002217980065
:10EFF4003317980044179800551798000080EB00C9
:10F00400100798000E609000E24F50000300360095
:10F014000080EB0060179800D90037000E60900064
:10F024000080FB007200B90080007800C0F5200069
:10F0340000804000200798002E00900010009000EF
:10F044000000E00003003A008080EB0061179800A4
:10F05400CB0037002E00900090007800E0062000DE
:10F06400808F50009E003A002E009000D000900047
:10F0740040009000660147000089BE002E00900009
:10F08400B0009000010F78004E1090000000E000E6
:10F09400390032005E109000F00F5000030032007F
:10F0A4000080EB0060179800B5003700CE10900088
:10F0B400214090000081FB00314090000080FB0063
:10F0C4004800DD0002007000000F7800CE109000B0
:10F0D400414090000082FB00514090000080FB0002
:10F0E4004800DD00040070000001780061409000D9
:10F0F4000082FB00714090000080FB004800DD00AE
:10F104000400700080017800660047000288BE0099
:10F114002E00900010009000E10F500016003A00FD
:10F1240070004700000178006000B8000089BE004C
:10F13400640141006000B8000089BE006401410020
:10F144006000B8000089BE00640141006000B8009E
:10F154000089BE00F0004700020120000E6090000C
:10F1640041FD0700E10F400003003A008080EB00FE
:10F17400611798008200370066014700120078008A
:10F1840092009000E00F5000E08F580004003A0015
:10F19400660147000080EB008080EB000089BE0020
:10F1A4002E009000005090000080FB007800B90011
:10F1B40080007800C0EA2000008040001002BE00F9
:10F1C400660147001200780092009000800F520000
:10F1D400818F5A002A00320066004700E400400094
:10F1E40066004700B4D10200000000000000E00007
:10F1F4000D0032002E009000005090000080FB00B3
:10F204007800B90080007800C0EA200080804000C7
:10F214006600470009000900B0587800A100B10059
:10F22400A000B10016003700F6FC02000000000048
:10F234000001BE00C07A8000D17A80000001510034
:10F2440081815900A025260021002000800F510053
:10F25400818F59000700360066004700E8D002009D
:10F2640000000000F6FC020000000000C07A8800E4
:10F27400D17A88000080EB006017980040003700C6
:10F284002E0090000050900004B90200000000001D
:10F294000000E000380032002E0090000050900082
:10F2A4000080FB007800B900EA004000C0EA2000BA
:10F2B400008040001E087800AE1090001E109000E0
:10F2C4006EB902000000000010079800BCB90200EB
:10F2D400000000009E00900061179800280037008D
:10F2E4002E0090009000780040062000808F50008F
:10F2F40021003A002E00900010009000E60F50000C
:10F30400030032000080EB00601798001C003700F7
:10F314000E609000DF0107000000E00003003200EF
:10F324008080EB0061179800150037002E109000C4
:10F334000000E00003003A000000EB0060179800B2
:10F344000F0037002E1190009E1090002E009000A8
:10F35400005090004E2F020000000000100798009B
:10F364001E0090000000E000030032009E009000A8
:10F3740061179800020037000080EB0060179800C6
:10F384006E1090000080FA00000006000C00FA00E5
:10F3940020479800210798003207980043079800F7
:10F3A4002E409000E24F5000030036000080EB0036
:10F3B400500798003B0037002E4090000080FB006F
:10F3C4007200B90080007800C0F52000008F400072
:10F3D4001E0078009000780040062000808F5000C6
:10F3E40016003A001E00780010009000E60F50004E
:10F3F400030032000080EB0050079800290037001A
:10F404002E409000A30107000000E000030032003A
:10F414000080EB0050079800220037003E01900066
:10F42400AE0090001E007800005090003A310200B7
:10F4340000000000500798001A0037001E007800F2
:10F4440090007800E0062000808F500013003A00FE
:10F454001E00780010009000E20F500003003200FC
:10F464000080EB00500798000E0037001E00780063
:10F474000050900018BA0200000000000000E000F4
:10F4840006003200BE0090002E0090007EBA0200FA
:10F494000000000050079800020037000000EB0055
:10F4A400500798005E0090000080FA0000000600FB
:10F4B4001400FA006047980041079800520798002A
:10F4C4006307980074079800050F98006E40900039
:10F4D4000080FB007200B90080007800C0F52000B5
:10F4E40000804000200798007E00900010079800DC
:10F4F4002E00900090007800E0062000808F5000DD
:10F5040056003A002E00900010009000E20F5000C8
:10F51400030032000000EB00100F98008E0037004B
:10F524002E0090000050900018BA02000000000065
:10F534000000E000460032007E0090000000E00081
:10F544003D0032000E0890000000E0003A00320056
:10F554000E08900010007800EF0F500036003600BF
:10F564002E009000005090000080FB007800B9004D
:10F5740080007800C0EA2000008040001001BE0036
:10F584009E009000F00F20000002610041409000B6
:10F594006040600004407000C04098004812DE00E3
:10F5A400514090006040600004407000D0409800DA
:10F5B400F00F200000826100614090006040600014
:10F5C40004407000E04098004819DE00714090004B
:10F5D4006040600002407000F04098002E009000EF
:10F5E400005090000080FB007800B900EA00400061
:10F5F400C0EA200000804000900178009E00900046
:10F60400F00F200000816100214090006040600004
:10F6140002407000A04098004819DE00314090007C
:10F624006040600002407000B04098008E08900076
:10F634000001200080087800DE0090004E00900059
:10F644007EBA020000000000100F9800420037004C
:10F654000000EB00100F98003F0037007E00900080
:10F664000000E000360032000E0890000000E000C8
:10F67400330032000E08900010007800EF0F5000A5
:10F684002F0036002E00900000509000122E020031
:10F6940000000000000F78001E0078001001BE007A
:10F6A4009E009000F00F2000000261004140900095
:10F6B4006040600004407000C04098004812DE00C2
:10F6C400514090006040600004407000D0409800B9
:10F6D400F00F2000008261006140900060406000F3
:10F6E40004407000E04098004819DE00714090002A
:10F6F4006040600002407000F04098001E007800F6
:10F70400D00190009E009000F00F20000081610065
:10F71400214090006040600002407000A0409800CA
:10F724004819DE00314090006040600002407000E3
:10F73400B04098008E0890000001200080087800F6
:10F744008001EB005E019000CE0090006E409000BE
:10F754000EFF0700100F98001E0890000080FA00AA
:10F76400000006000C00FA003007980041079800DA
:10F7740000012000200798000000EB00100798000B
:10F784000D0037001E009000FC004000A0B52000D2
:10F7940000804000104F780000C2B3009E4F10005C
:10F7A400090032001E04E000070032001E00900031
:10F7B4000000E800100798009E0090002E009000C2
:10F7C400808F5000EFFF39001E0090002007980042
:10F7D4002E0090008000E8004E009000808F5000C2
:10F7E400030034000080EB00500798000C00370041
:10F7F4003E00900061B720002E019000F608020040
:10F8040000000000AE0090003E00900080804000A8
:10F814000040EB00804878000000EB00500798009F
:10F824005E0090000080FA00000006000800FA0064
:10F83400404798004E409000E24F500003003600CD
:10F844000080EB00300798008F0037004E40900096
:10F854000080FB007200B90080007800C0F5200031
:10F86400008F40001E007800100090000000E000AF
:10F8740003003A000000EB003007980082003700D4
:10F884001E0078009000780040062000808F500011
:10F8940070003A001E00780010009000E30F500042
:10F8A4002F003A000040EB00204798002800370062
:10F8B4002E4090000080FB007200B9008080E800B8
:10F8C400C0F520000080400010007800E40F5000D4
:10F8D4001C003A002E4090000080FB007200B9002A
:10F8E400E4004000C0F52000008040009000780053
:10F8F4001E00780020009000808F500011003A0014
:10F904002E4090000080FB007200B900F00040001F
:10F91400C0F520000080400010407800FA2D02005D
:10F92400000000002E4090000080FB007200B9002F
:10F934008080E800C0F52000808040000000EB00DB
:10F94400800878002E4090000040E800204798008E
:10F954002E409000E24F5000D5FF3600450037009E
:10F964001E00780010009000E30F500041003600A4
:10F974001E007800700090000000E0002C003200AF
:10F984000040EB0020479800210037002E409000F3
:10F994000080FB007200B9008080E800C0F5200000
:10F9A4000080400010007800E30F500015003A007A
:10F9B4002E4090000080FB007200B900E40040007B
:10F9C400C0F5200000804000900078001E00780000
:10F9D40020009000808F50000A003A001E0078003A
:10F9E40000509000562D0200000000009E00780098
:10F9F40040002000900098000000EB0030079800C1
:10FA0400210037002E4090000040E8002047980075
:10FA14002E409000E24F5000DCFF36001E007800BC
:10FA240000509000FA2D0200000000001100370081
:10FA34001E00780010009000E70F50000D00320007
:10FA44001E00780000509000FA2D02000000000013
:10FA5400080037001E00780010009000E20F5000EC
:10FA640004003A001E00780000509000A4B8020080
:10FA7400000000009E0078000000EB009000980059
:10FA84000000EB00300798003E0090000080FA0070
:10FA9400000006000A00FA00604798006E409000DB
:10FAA4000080FB007200B90080007800C0F52000DF
:10FAB40000804000200798002E0090001000900065
:10FAC400E70F500003003A001000200040079800A0
:10FAD4003F0037002E00900000509000FE2C0200E2
:10FAE40000000000000F78002E00900070009000CD
:10FAF4000000E000280032000040EB00204798009E
:10FB0400220037002E4090000080FB007200B900F4
:10FB14008080E800C0F520000080400010007800DC
:10FB2400E30F500016003A002E4090000080FB00C6
:10FB34007200B900E4004000C0F5200000804000DD
:10FB4400900078002E00900020009000808F5000DC
:10FB54000B003A001E00E00003003A000000EB0036
:10FB6400400798001A003700AE00900040002000C3
:10FB740090009800100020004007980014003700FF
:10FB84002E4090000040E800204798002E4090004E
:10FB9400E24F5000DBFF36001E00E0000A00320096
:10FBA4002E00900000509000FA2D0200000000008A
:10FBB400AE0090007000200090009800100020001B
:10FBC40040079800020037000000EB00400798004F
:10FBD4004E0090000080FA00000006000200FA00C7
:10FBE40010C0B300004F7800090037001E80FB00EE
:10FBF4006A00B9008000780060E3200000814000C2
:10FC04000080EB008080EB000089BE001E4FE800FE
:10FC140070C0B3009E4F1000F4FF360014E20200DF
:10FC2400000000000080EB008080EB00107588006D
:10FC340021758800320507000000EB00307488004D
:10FC44000080FA00000006001E00FA00500F980021
:10FC54000040EB00005F98005E08900010407800C0
:10FC64000004E0000300320030748000E10F500013
:10FC740003003A00F00F2000600F98009600370050
:10FC84000000EB0020079800DE089000010F7800C8
:10FC94000A0037001E007800104078008080FB00C6
:10FCA4002E00900001004000200798002E009000D4
:10FCB40000004000200798001E0FE8001E00780096
:10FCC400104078000004E000F2FF3A0010C0B300D6
:10FCD400604798000F0037006E4090000080FB00E2
:10FCE4006A00B9008000780060E3200000804000D2
:10FCF4001001BE000080EB008080EB00800F5100FB
:10FD0400818F5900060032006E4090000040E800E8
:10FD1400604798006E409000E74F5000EEFF3600B9
:10FD24006E409000E74F500003003A00F00F2000AF
:10FD3400600F9800680037000000EB00100798007F
:10FD44005F0037001E009000670060000000E000C4
:10FD54000E003A001E0090000000400068004000C1
:10FD640001002000B0718800C171880000012000EA
:10FD740001002000D0718800E1718800E80047008C
:10FD8400020120000040EB002C0107001E0090003F
:10FD940067006000E800470000004000E080780051
:10FDA4002E009000808F500042003A001E00900008
:10FDB400560307004074800051748000B0718800BD
:10FDC400C1718800F00F200001002000D07188006C
:10FDD400E1718800DE089000010F78000900370007
:10FDE400F80047000040EB00910007001E00780077
:10FDF400904078000E58900080CF500005003A00E3
:10FE04001E0FE8001E007800104078000004E00097
:10FE1400F3FF3A00F80047000040EB0084000700BD
:10FE24000E5890000004E00022003A001E00780002
:10FE3400104078000004E0001E003A006E4090007C
:10FE44000080FB0062748000737480006A00B90053
:10FE54008000780060E32000008040000288BE003B
:10FE64006E4090000080FB008274800093748000D8
:10FE74006A00B900E400400060E320000080400014
:10FE84000288BE006E4090000080FB006A00B9004A
:10FE9400E800400060E32000008040009E009000E5
:10FEA400010878006E4090000080FB00600F98000D
:10FEB400090037001E0090000000E80010079800B9
:10FEC400017580001E009000810F50009DFF3900D5
:10FED400F00F2000600F98006E0890000080FA0078
:10FEE400000006000600FA00100798003074800035
:10FEF400E10F500004003200017580001E009000E4
:10FF0400810F500003003600F00F200020079800F6
:10FF14003300370010C0B300004F78000C003700E6
:10FF24001E80FB006A00B9008000780060E32000B6
:10FF3400008040001001BE000080EB008080EB00D8
:10FF4400800F5100818F5900040032001E4FE800D9
:10FF540071C0B3009ECF1000F1FF360070C0B30033
:10FF64009E4F100003003A00F10F20002107980073
:10FF74001B0037001E009000E40207001E80FB00F7
:10FF84006A00B900E800400060E3200000804000FF
:10FF94009E009000010878001E80FB0062748000BF
:10FFA400737480006A00B9008000780060E3200068
:10FFB400008040000288BE001E80FB008274800026
:10FFC400937480006A00B900E400400060E32000FC
:10FFD400008040000288BE001E80FB0020079800BD
:10FFE4002E0090000080FA00000006000200FA00D3
:10FFF400004F78001E04E0000B00320070C0B30014
:020000040001F9
:100004009E4F100008003E001E80FB006A00B900ED
:100014008000780060E32000008140000080EB0055
:100024008080EB000089BE000080FA00000006001A
:100034000600FA00004F78001107980070C0B30062
:100044009E4F1000030036000000EB0020079800CC
:10005400770037001E80FB006A00B900800078003A
:1000640060E32000008040001001BE000080EB002F
:100074008080EB00800F5100818F5900090032000D
:100084001E80FB006A00B900E400400060E3200029
:10009400008040001000BE00E00F5000E08F5800C8
:1000A40003003A000000EB002007980060003700CE
:1000B4001E0090000000E0001D003A001E82FB00BC
:1000C4006A20B9008000780060E3200000804000CE
:1000D4001000BE0061014000E08148006A20B900C0
:1000E4008000780060E32000008040000288BE00A9
:1000F4001E82FB006A20B900E400400060E3200097
:10010400008040001000BE0061015000E0815800F2
:100114006A20B900E400400060E320000080400051
:100124000288BE001000200020079800400037001D
:100134001E80FB006A00B9008000780060E32000A4
:10014400008040001001BE00107580002175800001
:1001540061004000E0804800800F5100818F590009
:100164000A0032001E80FB006A00B900800078009B
:1001740060E32000008040001000BE009008B00042
:100184000180B00032E202000000000046E20200FA
:1001940000000000804078001E00900001487800B4
:1001A4001E80FB006A00B9008000780060E3200034
:1001B400008040001000BE00107588002175880082
:1001C4001E82FB006A20B9008000780060E32000F2
:1001D400008040001000BE0061014000E081480042
:1001E4006A20B9008000780060E3200000804000AD
:1001F4000288BE001E82FB006A20B900E4004000B1
:1002040060E32000008040001000BE006101500047
:10021400E08158006A20B900E400400060E3200057
:10022400008040000288BE001000200020079800D3
:100234002E0090000080FA00000006000800FA007A
:10024400004F7800110798002207980070C0B3008F
:100254009E4F1000030036000000EB0030079800AA
:100264007B0037002E0090006101B8001E80FB0067
:100274006A00B900E400400060E320000080400010
:100284001000BE00800F5100818F59000700360016
:100294001E80FB006A00B900E400400060E3200017
:1002A400008040001000BE00200798001E80FB0064
:1002B4006A00B9008000780060E3200000804000FC
:1002C4001001BE000080EB008080EB00800F510025
:1002D400818F5900030032002E0090000000E000DE
:1002E40003003A000000EB00300798005800370084
:1002F4001E0090000000E00023003A001E82FB0074
:100304001E80FB006A00B9008000780060E32000D2
:10031400008040001001BE002E009000010020006B
:1003240002014000838148006A20B90080007800FF
:1003340060E32000008040000288BE001E82FB00B3
:100344001E80FB006A00B900E400400060E3200066
:10035400008040001001BE002E009000010020002B
:1003640000015100818159006A20B900E400400075
:1003740060E32000008040000288BE002E00900050
:1003840030079800320037001E80FB006A00B90075
:100394008000780060E32000008040001000BE0070
:1003A4009008B0000180B000AE0190001E019000E2
:1003B4008CE20200000000001E82FB001E80FB0095
:1003C4006A00B9008000780060E3200000804000EB
:1003D4001001BE002E009000010020000201400028
:1003E400838148006A20B9008000780060E320001F
:1003F400008040000288BE001E82FB001E80FB00BD
:100404006A00B900E400400060E32000008040007E
:100414001001BE002E0090000100200000015100D8
:10042400818159006A20B900E400400060E32000A3
:10043400008040000288BE000080EB008080EB005A
:1004440010758800217588002E00900030079800F0
:100454003E0090000080FA00000006000600FA004A
:10046400004F7800110798009E0090004200200081
:100474001E40780071FF07008000EB002107980000
:10048400E40F500002003A001000200020079800FA
:100494002E0090000080FA00000006001000FA0010
:1004A400881F780040479800320798004307980057
:1004B400510798004E409000E74F5000030036006B
:1004C4000000EB0060079800DE0037004E4090000B
:1004D4000080FB006A00B9008000780060E320001F
:1004E400008040001001BE000080EB008080EB0023
:1004F400800F5100818F590003003A000001EB0086
:1005040062079800CF003700DE019000730798005F
:100514007E029000E10F5200A3003200FE02900020
:10052400E18F5200070039007E009000E20F500076
:100534002B0032007E019000E30F51005E00320078
:10054400BE0037004E409000FF010700008FBE0040
:100554003E009000CE009000BE0F5000AE8F5800B9
:10056400030036008001EB0063079800B5003700F4
:100574004E4090000084FB004E4090003D02070076
:100584000001BE003E009000CE0090000201400039
:10059400838148006A40B9008000780060E320004D
:1005A400008040000288BE004E4090000081FB00A5
:1005B4003E009000CE0090003E021000AE82180073
:1005C4006A10B900E400400060E3200000804000AD
:1005D4000488BE00140020006407980099003700C6
:1005E4004E4090000080FB006A00B900E400400027
:1005F40060E32000008040001001BE003E00900037
:10060400CE009000800F5100818F5900030031000B
:100614008002EB00650798008A0037004E40900086
:100624000082FB004E4090000080FB006A00B9008D
:100634008000780060E32000008040001001BE00CC
:100644003E009000CE0090000201400083814800EB
:100654006A20B9008000780060E320000080400038
:100664000288BE004E4090000082FB004E40900085
:100674000080FB006A00B900E400400060E3200051
:10068400008040001001BE003E009000CE009000AB
:1006940000015100818159006A20B900E400400042
:1006A40060E32000008040000288BE0010002000AB
:1006B40060079800630037004E409000ED0107008A
:1006C400008FBE004E4090000080FB006A00B9001D
:1006D4008000780060E32000008040001001BE002C
:1006E4003E009000CE0090003E024000AE824800E2
:1006F4000400BE00800F5100818F590003003100B7
:100704008002EB00650798004E0037004E409000D1
:100714000082FB004E4090000080FB006A00B9009C
:100724008000780060E32000008040001001BE00DB
:100734003E009000CE0090000001510081815900DC
:100744006A20B9008000780060E320000080400047
:100754000288BE004E4090000082FB004E40900094
:100764000080FB006A00B900E400400060E3200060
:10077400008040001001BE003E009000CE009000BA
:1007840002014000838148006A20B900E40040006F
:1007940060E32000008040000288BE0010002000BA
:1007A40060079800270037004E409000660107005C
:1007B400008FBE003E009000CE009000BE0F50009F
:1007C400AE8F5800030036000001EB00620798006A
:1007D4001C0037004E4090000084FB004E40900007
:1007E400CC0107000001BE003E009000CE00900046
:1007F40000015100818159006A40B90080007800ED
:1008040060E32000008040000288BE004E4090005B
:100814000080FB006A00B900E400400060E32000AF
:10082400008040003E029000CE0290000488BE008A
:100834001500200065079800020037000000EB0057
:10084400600798006E0090004F0478000080FA0062
:10085400000006000800FA000040EB00004F78009A
:10086400090037001E80FB006A00B9008000780090
:1008740060E32000008140000080EB008080EB00FA
:100884000089BE001E4FE80060C0B3009E4F1000F8
:10089400F4FF360010002000307488006000B800B7
:1008A400B0718800C17188000080EB00F07188008D
:1008B400B0718000C17180000080FB000100200045
:1008C4009008B0000180B000F20320000300200073
:1008D400000278008102780002007800830078002A
:1008E40000016200018062006102B80024079800E0
:1008F400350798002E009000BE009000C000DD0077
:100904000000200020079800310798002E00900076
:10091400BE0090006112B8002407980035079800C3
:100924002E019000BE0190000200700083807000D0
:1009340002042000030020000000510081805900BF
:10094400D0718800E1718800B0718000C1718000AD
:100954009008B0000180B00058E3020000000000DD
:100964000000E00003003A008001EB001307980048
:1009740002003700F40F2000140798001E009000B6
:100984000080FA00000006000800FA0020479800E2
:1009940021079800320798000000EB00000F780050
:1009A400450037009E0078002E0090000080400033
:1009B400104078006CE30200000000002E4090001C
:1009C4000082FB006A20B9008000780060E3200008
:1009D400008040001000BE0061014000E08148003A
:1009E4006A20B9008000780060E3200000804000A5
:1009F4000288BE002E4090000082FB006A20B900ED
:100A0400E400400060E32000008040001000BE00CD
:100A140061015000E08158006A20B900E400400000
:100A240060E32000008040000288BE002E40900059
:100A34000080FB006A00B900E400400060E320008D
:100A4400008040001000BE00E00F5000E08F58000E
:100A540018003A000000EB001D0007001000200001
:100A6400307488002E4090000080FB006A00B900BA
:100A74008000780060E32000008040001000BE0089
:100A84009008B0000180B00058E3020000000000AC
:100A94002E4090000080FB006A00B900E400400092
:100AA40060E32000008140000004200001002000D9
:100AB4000089BE001E0FE8003E0090009E0F10004B
:100AC400B8FF39001E0078000080FA00000006001C
:100AD4000200FA00000F78000000EB003074880078
:100AE400CAE3020000000000D6E402000000000097
:100AF4000000E000FCFF3A001E00E00001003200AC
:100B04007F0107000080FA00000006000200FA00DE
:100B1400000F7800F07480009E0F1000180032005F
:100B2400007580009E0F100001003900140037008A
:100B34006001200001002000D0718800E17188006C
:100B44001E0078006B00B9008000780000758000FA
:100B540000804000000040006800400001002000C8
:100B6400B0718800C171880081E820006201200012
:100B74000040EB00B1FD07001E007800F07488000F
:100B84000080FA00000006000600FA00004F78001A
:100B940070C0B3009E4F1000040036006000B8001F
:100BA40010079800210798001A0037001E80FB00E8
:100BB4006A00B9008000780060E3200000804000F3
:100BC4001001BE000080EB008080EB00800F51001C
:100BD400818F590004003A006000B80010079800A3
:100BE400210798000B0037001E80FB006A00B90043
:100BF400E800400060E3200000804000100078001E
:100C0400C2FF0700A0748000B17480001007980030
:100C1400210798001E009000AE0090000080FA00AA
:100C2400000006000600FA00004F780070C0B30010
:100C34009E4F1000040036006000B80010079800B2
:100C4400210798001A0037001E80FB006A00B900D3
:100C54008000780060E32000008040001001BE00A6
:100C64000080EB008080EB00800F5100818F5900E1
:100C740004003A006000B8001007980021079800AB
:100C84000B0037001E80FB006A00B900E80040003A
:100C940060E3200000804000100078009BFF070004
:100CA400C0748000D1748000100798002107980058
:100CB4001E009000AE0090000080FA0000000600C4
:100CC4000400FA00004F780070C0B3009E4F10007B
:100CD400030036000000EB001007980017003700EF
:100CE4001E80FB006A00B9008000780060E32000E9
:100CF400008040001001BE000080EB008080EB000B
:100D0400800F5100818F590003003A000000EB006E
:100D140010079800090037001E80FB006A00B90024
:100D2400E800400060E320000080400010007800EC
:100D340076FF0700E0748000100798001E00900002
:100D44000080FA00000006000600FA00004F780058
:100D540070C0B3009E4F1000040036006000B8005D
:100D640010079800210798001A0037001E80FB0026
:100D74006A00B9008000780060E320000080400031
:100D84001001BE000080EB008080EB00800F51005A
:100D9400818F590004003A006000B80010079800E1
:100DA400210798000B0037001E80FB006A00B90081
:100DB400E800400060E3200000804000100078005C
:100DC40052FF07008074800091748000100798001F
:100DD400210798001E009000AE0090000080FA00E9
:100DE400000006000600FA00004F780070C0B3004F
:100DF4009E4F1000040036006011B80012079800DE
:100E040023079800170037001E80FB006A00B90012
:100E14008000780060E32000008040001001BE00E4
:100E24000080EB008080EB00800F5100818F59001F
:100E340004003A006000B8001007980021079800E9
:100E4400080037001E80FB006A00B900E40040007F
:100E540060E32000008040001001BE0012079800EB
:100E6400230798001E009000AE0090000080FA0056
:100E7400000006000600FA00004F780070C0B300BE
:100E84009E4F1000040036006000B8001007980060
:100E9400210798001B0037001E80FB006A00B90080
:100EA4008000780060E32000008040001001BE0054
:100EB4000080EB008080EB00800F5100818F59008F
:100EC40005003A000080EB008080EB0010079800DA
:100ED400210798000B0037001E80FB006A00B90050
:100EE400E800400060E3200000804000100078002B
:100EF40006FF07006074800071748000100798007A
:100F0400210798001E009000AE0090000080FA00B7
:100F1400000006000600FA00004F780070C0B3001D
:100F24009E4F1000050036000080EB008080EB002F
:100F340010079800210798001F0037001E80FB004F
:100F44006A00B9008000780060E32000008040005F
:100F54001001BE000080EB008080EB00800F510088
:100F6400818F590005003A000080EB008080EB007F
:100F740010079800210798000F0037001E80FB001F
:100F84006A00B900E800400060E3200000804000EF
:100F940010007800DDFE0700627480007374800026
:100FA40080748000917480000201400083814800B5
:100FB40012079800230798001E009000AE009000CE
:100FC4000080FA00000006000C00FA004047980078
:100FD40031079800420798004E409000E74F5000B8
:100FE400030036000000EB0050079800270037008C
:100FF4004E4090000080FB006A00B9008000780039
:1010040060E32000008040001001BE000080EB007F
:101014008080EB00800F5100818F590003003A005B
:101024008000EB0051079800180037004E409000F4
:101034000080FB006A00B900E800400060E3200083
:101044000080400010007800B0FE0700407480006B
:1010540051748000008FBE001E00BE00B071880075
:10106400C1718800F00F200001002000D0718800B9
:10107400E17188004E019000BE0090000040EB003A
:101084006EFC070011002000510798005E009000DC
:101094000080FA00000006000200FA00889FBE00EB
:1010A400004F78001E80FB006A00B90080007800C1
:1010B40060E32000008040001004BE001E40780061
:1010C4006CFF07000000540081805C004F04BE00E8
:1010D4000080FA00000006000200FA00004F7800C9
:1010E4001E80FB006A00B900E800400060E32000B5
:1010F40000804000100078000080FA000000060024
:101104000000FA006000B800B0718800C171880066
:101114008000200001002000D0718800E171880067
:1011240081E82000620020000040EB0043FC07003F
:101134006200200021A42A0080E820009407020015
:10114400000000000000E00005003A0001EA200071
:10115400220020000040EB0038FC070002003700AA
:101164000000EB00007588000080EB00F07488003C
:101174000080FA00000006000400FA0020479800EE
:10118400008680000000E0000A003A001000200001
:10119400008688000040EB00004F78000300370011
:1011A40000C0EB00C2EFB7001E4FE8001E04E000D1
:1011B400FBFF3200C2CFBF00E14F40000500320008
:1011C400C2CFBF00A4B802000000000000C0EB00C2
:1011D400C2EFB7002000200001002000607E8800DC
:1011E400717E880010002000207E88000040EB0003
:1011F400C6EFB700C68FA800C62FA8000080FA006B
:10120400000006000200FA00004F7800C2CFBF00C1
:10121400E14F400005003200C2CFBF00A4B8020075
:101224000000000000C0EB00C2EFB7000000EB00BC
:10123400207E88000080FA00000006000200FA0008
:10124400004F7800207E80000000E00007003A0094
:101254002000200001002000607E8800717E88004C
:1012640010002000207E8800C60FA9000080FA002C
:10127400000006000400FA00004F7800207E800081
:10128400100798001E0090000000E00002003200E9
:1012940010002000100798001E0090000080FA0043
:1012A400000006000200FA00004F7800307E800043
:1012B400614060000080FB000080FA00000006002E
:1012C4000400FA00004F7800307E80006200600065
:1012D4000000E00004003200C62FA9001000200026
:1012E40010079800020037000000EB001007980078
:1012F4001E0090000080FA00000006000200FA00C0
:10130400004F7800307E80004300DE0061406000C2
:101314000080FB000080FA00000006000000FA00D4
:10132400C27E8000D37E8000F00F20008000610028
:101334005ACBBF0060406000014070005AEBB70018
:10134400C810DE005BCBBF0060406000014070004D
:101354005BEBB700F00F2000808061005CCBBF0026
:1013640060406000014070005CEBB700C818DE000C
:101374005DCBBF0060406000014070005DEBB700D2
:101384000080FA00000006000A00FA00889FBE00F0
:101394008A9FBE000040EB00004F78003D023700FA
:1013A400207E80006101B80032079800430798004E
:1013B400C0002000010020003E019000CE019000FA
:1013C400800F5100818F590031023E003E00900091
:1013D400CE009000006001002D0237000B003700A2
:1013E400160037006300370089003700BD0037005E
:1013F40090013700C6013700F2013700C4013700FD
:10140400F0013700C2013700EE0137003404200038
:10141400430420000041EB006000B8007EB50200E8
:1014240000000000C2EFB700C2CFBF00E14F400090
:101434001702320020002000207E8800C003200014
:1014440001002000807E8800917E88000040EB002F
:10145400ECEFB700C60FA900C64FA900BE66020094
:10146400000000000000E00009023200C2CFBF000B
:1014740004B902000000000080007800B0122000CF
:10148400808F500002023600307E80004400DE006F
:10149400614060000004A200614060000080FB0025
:1014A400610060004401DD00317E8000F0FE2F0009
:1014B4000080600002007000307E8800C2CFBF0050
:1014C4000080FB007800B90080007800C0EA2000AA
:1014D40000804000A2002000F10F2000D807020085
:1014E400000000008000EB0010C0B3004A030700B6
:1014F400F6FC0200000000000005BE00647E8000CF
:10150400757E80000400BE000001EB008001EB004A
:10151400A4252600250020006033B800DE04020064
:10152400000000000004BE00BAA502000000000094
:10153400010020000200200003002000A425260052
:10154400250020006033B8003C06020000000000C3
:1015540008004000898048000A0040008B80480051
:10156400407E8800517E880030002000207E880064
:10157400C7013700C2CFBF0018BA02000000000044
:1015840080007800900F2000808F50001A003E00E9
:10159400F6FC0200000000000001BE00407E800056
:1015A400517E80000000510081805900E00F5000FE
:1015B400E08F5800B6013400627E8000737E8000A4
:1015C400F003200001002000800F5100818F59009A
:1015D40006003E00607E8000717E800000004000B6
:1015E40081804800607E8800717E88002000200091
:1015F400207E8800A6013700C66FA800AB01070053
:10160400E24F5000A2013A0040002000207E8800F2
:10161400C2CFBF0004B902000000000080007800BF
:1016240010102000808F500099013600C2CFBF00F7
:101634000080FB007800B90080007800C0EA200038
:1016440000804000A2002000F10F2000D807020013
:10165400000000008000EB0030C0B300EE02070081
:10166400F6FC0200000000000005BE00647E80005D
:10167400757E80000400BE000001EB008001EB00D9
:10168400A4252600250020006033B800DE040200F3
:10169400000000000004BE00BAA502000000000023
:1016A400010020000200200003002000A4252600E1
:1016B400250020006033B8003C0602000000000052
:1016C40008004000898048000A0040008B804800E0
:1016D400407E8800517E880050002000207E8800D3
:1016E4006B013700C2CFBF0018BA0200000000002F
:1016F40080007800900F2000808F50001A003E0078
:10170400F6FC0200000000000001BE00407E8000E4
:10171400517E80000000510081805900E00F50008C
:10172400E08F58005A013400627E8000737E80008E
:10173400F003200001002000800F5100818F590028
:1017440006003E00607E8000717E80000000400044
:1017540081804800607E8800717E8800200020001F
:10176400207E88004A013700500107000080FB00FA
:1017740020079800AE009000E58F5000040032006E
:101784002E019000E60F5100A700320040013700FF
:10179400C2CFBF00A4B802000000000000C0EB00EC
:1017A400C2EFB700F6FC020000000000407E880093
:1017B400517E880060002000207E8800C62FA8008B
:1017C400C60FA800607F8000610060000000E00098
:1017D40018003200C27E8000D37E8000F00F20000B
:1017E400800061005ACBBF0060406000014070007F
:1017F4005AEBB700C810DE005BCBBF00604060004E
:10180400014070005BEBB700F00F200080806100A6
:101814005CCBBF0060406000014070005CEBB7002F
:10182400C818DE005DCBBF0060406000014070005E
:101834005DEBB700607F8000640060000000E000A2
:1018440018003200027F8000137F8000F00F200018
:10185400800061005ECBBF0060406000014070000A
:101864005EEBB700C810DE005FCBBF0060406000D5
:10187400014070005FEBB700F00F20008080610032
:1018840060CBBF00604060000140700060EBB700B7
:10189400C818DE0061CBBF006040600001407000EA
:1018A40061EBB700607F8000620060000000E00030
:1018B40018003200E27E8000F37E8000F00F2000EA
:1018C4008000610062CBBF00604060000140700096
:1018D40062EBB700C810DE0063CBBF00604060005D
:1018E4000140700063EBB700F00F200080806100BE
:1018F40064CBBF00604060000140700064EBB7003F
:10190400C818DE0065CBBF00604060000140700075
:1019140065EBB700607F8000680060000000E000B5
:1019240018003200227F8000337F8000F00F2000F7
:101934008000610066CBBF00604060000140700021
:1019440066EBB700C810DE0067CBBF0060406000E4
:101954000140700067EBB700F00F20008080610049
:1019640068CBBF00604060000140700068EBB700C6
:10197400C818DE0069CBBF00604060000140700001
:1019840069EBB7006ACBBF00604060006AEBB70048
:101994006BCBBF00604060006BEBB7006CCBBF004B
:1019A400604060006CEBB7006DCBBF00604060002E
:1019B4006DEBB700607F8000700060000000E00005
:1019C400B3003200427F8000537F8000F00F20007C
:1019D400800061006ACBBF0060406000014070007D
:1019E4006AEBB700C810DE006BCBBF00604060003C
:1019F400014070006BEBB700F00F200080806100A5
:101A04006CCBBF0060406000014070006CEBB7001D
:101A1400C818DE006DCBBF0060406000014070005C
:101A24006DEBB7009A00370020002000207E88006C
:101A340097003700F6FC0200000000000001BE0021
:101A4400407E8000517E8000000151008181590058
:101A54009025260021002000800F5100818F59001D
:101A64008B003600887E8000997E8000667E800030
:101A7400777E80008600780030002000000AB800DD
:101A84006030B90005017800000141006338B900F5
:101A94000001410082027800840F5400858F5C00AD
:101AA4000F003600427E8000537E8000A025260071
:101AB400210020000200400083804800407E88000E
:101AC400517E8800807E8000917E800061005000FD
:101AD400E0805800807E8800917E88006C0037008A
:101AE40034042000430420000041EB006000B800EF
:101AF4007EB5020000000000C2EFB700C2CFBF00F5
:101B0400E14F40006200320070002000207E880017
:101B1400C2CFBF0004B902000000000080007800BA
:101B240010102000808F5000590036001100200052
:101B340030C0B300B8010700C64FA900F6FC02008C
:101B4400000000000005BE00647E8000757E8000F9
:101B54000400BE000001EB008001EB00A425260078
:101B6400250020006033B800DE04020000000000FD
:101B74000004BE00BAA5020000000000010020001D
:101B84000200200003002000A425260025002000D8
:101B94006033B8003C06020000000000080040006A
:101BA400898048000A0040008B804800407E8800FD
